:100000000C9424090C9443090C9443090C94D709CB
:100010000C940D0A0C9443090C9443090C94430965
:100020000C9443090C9443090C9443090C94430920
:100030000C9443090C9443090C9443090C942D0D22
:100040000C9443090C9443090C9443090C94430900
:100050000C94A66C0C9457640C9443090C944309BB
:100060000C9443090C942C650C9443090C94206562
:100070000C9443090C9443090C9443090C944309D0
:100080000C94D9770C9443090C9443090C944309BC
:100090000C946A650C9443090C945E650C944309B6
:1000A0000C9443090C9443090C9443090C944309A0
:1000B0000C9443090C9443090C9443090C94430990
:1000C0000C9443090C9443090C9443090C94430980
:1000D0000C9443090C9443090C9443090C94430970
:1000E0000C9443090C945F6C0C94696C0C94556CE3
:1000F0000C94156C0C949A6C0C948B6C0C947F6C17
:100100000C94736C0C9443090C9443090C944309AC
:100110000C9443090C9443090C9443090C9443092F
:1001200012813181B0819F82BF82DF82E782948217
:10013000084AD73B3BCE016E84BCBFFDC12F3D6C4E
:1001400074319ABD56833DDA3D00C77F11BED9E4B4
:10015000BB4C3E916BAAAABE000000803F076342E1
:1001600036B79BD8A71A39685618AEBAAB558C1D4E
:100170003CB7CC5763BD6DEDFD753EF6177231BFD0
:10018000000000803F08000000BE922449123EABF0
:10019000AAAA2ABECDCCCC4C3E00000080BEABAAA1
:1001A000AAAA3E00000000BF000000803F0000003F
:1001B0000000084178D3BB4387D1133D190E3CC3DF
:1001C000BD4282AD2B3E68EC8276BED98FE1A93E5E
:1001D0004C80EFFFBE01C4FF7F3F00000000002500
:1001E000730A005854414C5F5452494D3D256400F8
:1001F00025730A0025730A00546573742036202580
:10020000730A005465737420352025730A00546501
:10021000737420342025730A0054657374203320CE
:1002200025730A005465737420322025730A005424
:1002300065737420312025730A006368616E3D2563
:10024000640A0074787077723D25640A0035303096
:100250006B0A003235306B0A003131356B0A0035DC
:10026000366B0A0033386B0A0025730A00765F6C20
:100270006F773D252D332E32660A0025730A0073F1
:10028000656E743D252D75206475703D252D752096
:1002900069676E6F7265643D252D752074746C5F9F
:1002A0007A65726F3D252D750A0025372E3366203D
:1002B00025372E33660025352E32662000457272B2
:1002C0006F72203020566F6C74004E6F74207375FF
:1002D00070706F727465640A004572726F722030BC
:1002E00020566F6C74004572726F72203020566F0A
:1002F0006C7400256C7500416C6C6F7765642073BD
:100300007065656420312F31302F3130302F34301B
:1003100030206B6269742F730025630074746C3D28
:10032000252D64200074746C3D252D6420004E65DD
:10033000772074746C3D252D6420002563004D5397
:100340003536313120503D252D372E326620252D72
:10035000372E32666D0A00424D5030383520256CFC
:10036000642050612020252D372E32666D002563D4
:1003700000545F484541545F4944583D252D352E72
:1003800032662000545F4445573D252D352E326698
:10039000200041483D252D352E32662000545F5304
:1003A000485432583D252D352E3266200052485F84
:1003B00053485432583D252D352E32662000545F67
:1003C00052483D252D342E3166200052483D252DC2
:1003D000342E316620002563002563002563002547
:1003E00063002563007265706F72745F616C6C3DB1
:1003F000007265706F72743D0025630025630025EF
:100400006300256300204F534343414C3D25642046
:100410000020467573653A2065653D2530327820A9
:1004200068663D25303278206C663D253032782074
:100430006C623D25303278004D43553D2530366C99
:10044000780025630074785F6C656E3D252D6C75B2
:100450002C765F6C6F773D252D6C752C736874322C
:10046000783D252D6C750A002563004F4B0A002549
:100470006300256300256300256300256300256371
:100480000025630025630064656275675F616C6CBD
:100490003D0064656275673D0064656275673D0097
:1004A00025730A00646565700A006E6F6E650A0048
:1004B000707772733D00696E74725F7365635F700D
:1004C000313D252D372E33660A00696E74725F70D8
:1004D000313D252D6C640A00696E74725F7365632B
:1004E0005F70303D252D372E33660A00696E7472B9
:1004F0005F70303D252D6C640A00765F6D63753D3D
:10050000252D352E32660A00745F6D63753D252DED
:10051000352E32660A00707077723D25730A0064CA
:10052000656275673D0072636D643D25730A002541
:10053000730A006175746F0A006C6F675F6D6F649A
:10054000653D007573625F7077723D25730A0072B6
:10055000656C61793D25730A0074746C3D252D64CA
:100560000A0052494D455F616464723D252D642E39
:10057000252D640A006E65696768626F725F746139
:10058000626C655F73697A653D25640A00765F6C0D
:100590006F773D252D332E32660A00747870773DD3
:1005A00025640A006368616E3D25640A0069643D44
:1005B000006932635F6275733D006932635F737017
:1005C0006565643D252D6C750A007478743D25734E
:1005D0000A0053797374656D2053756D6D6172797E
:1005E0000A006D61736B3D002C00696E7465727654
:1005F000616C3D252D750023252D642C00745F68EA
:100600006561745F69647800745F64657700616830
:1006100000705F6D73353631310072685F736874D6
:10062000327800745F736874327800706100700013
:1006300061643400616433006164320061643100DC
:10064000613300613200613100765F696E0072686B
:100650000065727200757074696D650070315F6C51
:1006600073740070315F740070310070305F6C73B0
:10067000740070305F7400703000765F6D637500D9
:10068000745F6D63750074310074006964006536D1
:100690003400747874002D002B006175746F006E47
:1006A0006F6E6500706F7765725F736176655F6C02
:1006B000656472790072656C61795F6C656479005C
:1006C000636F6D7061737300616363656C0070725A
:1006D000657300705F707772006165730070315FE1
:1006E0006C6564790070305F6C6564720065766576
:1006F0006E74006C6564006F7700706B74007478C2
:100700005F6C6564790072785F6C656472006F700D
:100710006572006E6F6E65002530327800765F611D
:1007200064343D252D382E3666002000765F6164E6
:10073000333D252D382E3666002000765F61643209
:100740003D252D382E3666002000765F6164313DF0
:10075000252D382E3666002000765F6C6967687438
:100760003D252D382E3666002000765F61323D250E
:100770002D372E3366002000765F61313D252D3701
:100780002E3366002000765F696E3D252D352E32B2
:100790006600204E657665722D75736564207374EE
:1007A00061636B203E2025642062797465730A00C2
:1007B000757074696D653D252D642D646179732DA7
:1007C000253032643A253032643A253032642D685F
:1007D0006F7572730A0074657374205B6F66667C54
:1007E000317C327C337C347C355D202020202020FD
:1007F00020202D2074657374206D6F6465730A0D5D
:10080000007478205B706B74207061796C6F616428
:100810005D2020202020202020202020202D20733B
:10082000656E6420726164696F20706B74206B6503
:1008300079626F6172640A0D00776474205B6F6E79
:100840007C6F66667C746573745D20202020202098
:1008500020202020202D207761746368646F670A50
:100860000D00765F6C6F77205B765F6C6F775D2035
:1008700020202020202020202020202020202D206B
:100880006C6F77657374207265706F727420766F09
:100890006C746167650A0D007570677220202020F6
:1008A0002020202020202020202020202020202048
:1008B000202020202D207265626F6F742076696180
:1008C00020626F6F746C6F616465720A0D007561F0
:1008D0007274205B33386B7C35366B7C3131356B11
:1008E0007C3235306B7C3530306B5D202D2073656C
:1008F00074207465726D2F756172742073706565F4
:10090000640A0D00626F6F742020202020202020B8
:1009100020202020202020202020202020202020D7
:100920002D207265626F6F740A0D007077727320EC
:100930005B646565707C6E6F6E655D202020202095
:10094000202020202020202D206D637520736C65D1
:100950006570206D6F64650A0D00726573742065A3
:100960006570726F6D202020202020202020202004
:100970002020202020202D20726573746F72652046
:10098000656570726F6D0A0D0070707772205B6F15
:100990006E7C6F66665D2020202020202020202095
:1009A00020202020202D2070726F6772616D6D6194
:1009B000626C65207077720A0D00747874205B7326
:1009C0007472696E675D2020202020202020202066
:1009D0002020202020202D20536574207265706F08
:1009E0007274207465787420737472696E670A0D6E
:1009F0000074787077205B31352D305D2020202009
:100A0000202020202020202020202020202D2054A5
:100A100058205077722E20486967686573742030BB
:100A200020283364426D290A0D0074746C205B30F9
:100A30002D31355D20202020202020202020202046
:100A40002020202020202D2074696D652D746F2DAD
:100A50006C69766520666F72207061636B65747374
:100A60000A0D007373202020202020202020202029
:100A70002020202020202020202020202020202D69
:100A80002073797374656D2073756D6D6172790A69
:100A90000D007273202020202020202020202020E4
:100AA00020202020202020202020202020202D2039
:100AB000726164696F2073746174730A0D007269E6
:100AC000205B236E5D205B696E745D2020202020FA
:100AD000202020202020202020202D207265706FD3
:100AE000727420696E74657276616C0A0D007263AF
:100AF0006D64205B6F6E7C6F66665D202020202019
:100B0000202020202020202020202D20616C6C6FB0
:100B10007720636D642066726F6D206E65746F72EE
:100B20006B0A0D007265205B236E5D205B2B7C2DB4
:100B30005D205B6D61736B7C6175746F2C6D61738F
:100B40006B5D202D206D6F7465207265706F7274FF
:100B5000207365742F6D6F646966790A0D006F7775
:100B60002020202020202020202020202020202085
:100B7000202020202020202020202D206F6E652D79
:100B8000776972652073656E736F72730A0D006CFE
:100B90006F67205B6175746F7C6F6E7C6F66665DDE
:100BA00020202020202020202020202D206D6F7448
:100BB00065732064617461206F6E205553420A0D85
:100BC000006E65205B666C7573685D2020202020B8
:100BD000202020202020202020202020202D206EBA
:100BE00065696768626F72207461626C650A0D00E6
:100BF000657272202020202020202020202020200C
:100C00002020202020202020202020202D20657240
:100C1000726F722073746174730A0D006D637520B6
:100C200020202020202020202020202020202020C4
:100C300020202020202020202D206D637520696E2B
:100C4000666F0A0D00693263205B70726F62657CAB
:100C5000737065656420236E5D2020202020202095
:100C6000202D206932632070726F62652062757377
:100C70007C736574206275732073706565640A0DFA
:100C8000006964205B72657365745D2020202020FC
:100C9000202020202020202020202020202D2069FE
:100CA000642068616E646C696E670A0D0068756D1A
:100CB0002020202020202020202020202020202034
:100CC0002020202020202020202D2068756D6964A0
:100CD0006974792073656E736F720A0D0072656CAA
:100CE0006179205B6F6E7C6F66667C737461747370
:100CF0005D20202020202020202D2072656C61792D
:100D0000206E6574776F726B207265706F7274738A
:100D10000A0D006465205B6D61736B5D20202020EF
:100D20002020202020202020202020202020202DB6
:100D30002064656275670A0D006368616E205B312F
:100D4000312D32365D202020202020202020202020
:100D500020202020202D206368616E2031312D322B
:100D6000362028322E3430352D32343830204D683C
:100D70007A290A0D0063616C69205B5B765F696E9E
:100D80007C61317C61325D20766F6C747C7265733E
:100D900065747C6E6F6E655D202D2063616C696289
:100DA000726174650A0D0061646320202020202098
:100DB0002020202020202020202020202020202033
:100DC0002020202D2073686F7720765F696E2C209D
:100DD00061312C20613220766F6C74616765730A13
:100DE0000D007520202020202020202020202020E1
:100DF00020202020202020202020202020202D20E6
:100E0000757074696D650A0D007620202020202001
:100E100020202020202020202020202020202020D2
:100E200020202020202D2076657273696F6E0A0DB8
:100E3000006820202020202020202020202020208A
:100E4000202020202020202020202020202D20684D
:100E5000656C700A0D00256300756E6B6E6F776EA2
:100E600020636D640A00484D4335383833002573DC
:100E700000257300202573002025362E32662000C1
:100E8000253032780074656D705F65787465726EB8
:100E90003D252D362E326600202573002025362E66
:100EA0003266204F6E2D426F6172640025303278B9
:100EB0000074656D705F626F6172643D252D362E22
:100EC0003266000A00503A20256C642050612020D0
:100ED000252D372E3266206D0A002563002563001C
:100EE0004932433A2000452025642E256420636C56
:100EF0006F636B20256C752063707520256C7520E1
:100F00006C706D20256C752069727120256C7520C0
:100F1000676C656420256C7520796C656420256C90
:100F20007520726C656420256C7520747820256CA2
:100F300075206C697374656E20256C752073656E01
:100F4000736F727320256C752073657269616C20F4
:100F5000256C750A00532025642E256420636C6F70
:100F6000636B20256C7520747820256C7520727851
:100F700020256C752072747820256C75207272782B
:100F800020256C75207265786D697420256C75203C
:100F900061636B747820256C75206E6F61636B7470
:100FA0007820256C752061636B727820256C752024
:100FB00074696D65646F757420256C752062616459
:100FC00061636B727820256C7520746F6F6C6F6E27
:100FD0006720256C7520746F6F73686F727420259D
:100FE0006C752062616473796E636820256C75206E
:100FF00062616463726320256C7520636F6E746533
:101000006E74696F6E64726F7020256C75207365E5
:101010006E64696E6764726F7020256C75206C6CED
:10102000747820256C75206C6C727820256C750A9C
:1010300000257325730A004F6E6C696E650A000AFD
:10104000002C20636865636B2072617465202575D0
:1010500020487A0025732025732C206368616E6E0A
:10106000656C20257520706F776572202575000AE4
:101070000025783A004D41432061646472657373C2
:10108000200052616E646F6D2045554936342061F1
:101090006464726573732067656E657261746564FC
:1010A0000A000A2A2A2A2A2A2A2A426F6F74696E9B
:1010B000672025732A2A2A2A2A2A2A0A0045455007
:1010C000524F4D20697320636F72727570742C20BB
:1010D000726577726974696E6720776974682064D5
:1010E000656661756C74732E0A006C6F63616C6861
:1010F0006F73740041544D45474131323872666117
:101100003100020000FFFE0000016E616E00696E9A
:10111000660000407A10F35A00A0724E18090010C1
:10112000A5D4E80000E87648170000E40B5402005C
:1011300000CA9A3B000000E1F50500008096980087
:10114000000040420F000000A086010000001027B0
:1011500000000000E8030000000064000000000040
:101160000A00000000000100000000002C76D88872
:10117000DC674F0823DFC1DFAE59E1B1B796E5E385
:10118000E453C63AE651997696E8E6C28426EB899E
:101190008C9B62ED407C6FFCEFBC9C9F40F2BAA53B
:1011A0006FA5F490055A2AF75C936B6CF9676DC1D3
:1011B0001BFCE0E40D47FEF520E6B500D0ED902ED7
:1011C0000300943577050080841E080000204E0A35
:1011D000000000C80C333333330F986E1283114173
:1011E000EF8D2114893BE65516CFFEE6DB18D1843E
:1011F0004B381BF77C1D901DA4BBE4242032847265
:101200005E228100C9F124ECA1E53D274E414E4903
:101210004E495459494E46CDCCCC3D0AD7233C17B4
:10122000B7D13877CC2B329595E6241FB14F0A0001
:101230000020410000C84200401C4620BCBE4CCAF1
:101240001B0E5AAEC59D740011241FBECFEFD1E412
:10125000DEBFCDBF19E0A0E0B2E0E4EBFBE201E0CD
:101260000BBF02C007900D92AE3BB107D9F711E357
:10127000AEEBB9E001C01D92A337B107E1F70E94C0
:10128000B6830C94D8950C94000080EB94E09F9367
:101290008F930E94B1928091580290915902A0912F
:1012A0005A02B0915B020F900F9093FF03C08AEA3D
:1012B00094E002C084EA94E09F938F930E94B192DD
:1012C0000F900F900895E091771BEF71F0E0E453D9
:1012D000F44E80838091771B8F5F8093771B809182
:1012E000AD2888608093AD284EE352E061E1CA01E9
:1012F0000E94375480E090E00895CF93DF93EC0193
:101300008091C5099091C60986FF1DC08E811F92EC
:101310008F938D811F928F938C811F928F938B81DE
:101320001F928F938A811F928F9385E693E09F93FC
:101330008F930E949F928DB79EB70C960FB6F8942C
:101340009EBF0FBE8DBFBE018CEF99E00E94695514
:10135000BE0184E092E0DF91CF910C94DE5487EEE1
:1013600093E08115910511F00197F1F70895882315
:10137000B9F052985A981DBA8091690080628093A2
:101380006900EA9A53985B98EB9A809169008068AB
:10139000809369008091680081608093680008955F
:1013A000109269005A9AEA985B9AEB9808951F92F6
:1013B0000F920FB60F9211248F939F93AF93BF9309
:1013C0008091680080FF20C08091882890918928B2
:1013D000A0918A28B0918B280196A11DB11D809300
:1013E000882890938928A0938A28B0938B2880918D
:1013F000C5099091C60987FF07C0749882E090E004
:101400009093850280938402BF91AF919F918F91B9
:101410000F900FBE0F901F9018951F920F920FB64E
:101420000F9211248F939F93AF93BF938091680085
:1014300080FF20C080918C2890918D28A0918E28CB
:10144000B0918F280196A11DB11D80938C28909397
:101450008D28A0938E28B0938F288091C5099091F4
:10146000C60990FF07C0739882E090E090938502D0
:1014700080938402BF91AF919F918F910F900FBE87
:101480000F901F90189580937C0080917B00877F40
:1014900080937B0080917C00806C80937C0085E051
:1014A00080937A0080917A00806880937A0080919E
:1014B0007B0087FFFCCF80917B0085FFFCCF809174
:1014C0007A00806480937A0080917A0086FDFCCF58
:1014D000109279001092780084E090E060E070E073
:1014E00020917A00206420937A0020917A0026FDD2
:1014F000FCCF2091780030917900620F731F019723
:10150000009771F710927C0080917A008F7780931A
:101510007A00769567957695679580E090E00E94D1
:101520000C89089580E00E94430A20917C0230914A
:101530007D0240917E0250917F020E94F08A21EE4E
:101540003AE744E95EE30E94A587089580E180932D
:10155000510160E1609351018091510185FF03C009
:101560006F5F6F31B9F78BE4689FB0011124882752
:1015700077FD8095982F0E940E8920E030E64FE994
:1015800054E40E94A58720E030E04AE754E40E943A
:101590006F880895CF93DF93EC018881998100973C
:1015A00099F08136904121F01982188283E011C0B0
:1015B000623171F40E94A60A60931F247093202464
:1015C000809321249093222481E690E1998388835B
:1015D00081E0DF91CF91089580917B0088608093B6
:1015E0007B0089EC80937C0085E080937A00809179
:1015F0007A00806880937A0080917B0087FFFCCF1F
:1016000080917B0085FFFCCF80917A00806480937D
:101610007A0080917A0086FDFCCF80917A00806408
:1016200080937A0080917A0086FDFCCF60917800EB
:101630007091790080917A008F7780937A0080E0B2
:1016400090E00E940C8927ED33EA40E95FE30E94B5
:10165000F08A26E636E648E853E40E94A487089517
:10166000BF92CF92DF92EF92FF920F931F93CF938F
:10167000DF93CDB7DEB729970FB6F894DEBF0FBE64
:10168000CDBF6C011092BE098FEF898708E81BE17E
:10169000B12C7E0189E0E80EF11C89858823E9F1EF
:1016A000E8E0BE16E1F1BE016F5F7F4FC7010E9407
:1016B000D25D89858F3F11F08E3F19F48093BE096A
:1016C0002CC0CE010196C114D10471F40E94EB5DCF
:1016D0008093AA28FE013196A2EAB8E281918D9307
:1016E000EE15FF05D9F71DC00E94EB5DF801808360
:1016F000FE01319620E030E0A80148505109819167
:10170000DA01A20FB31F8C932F5F3F4F28303105B2
:10171000B1F7B394075F1F4FC0CF8B2D03C088E094
:1017200001C081E029960FB6F894DEBF0FBECDBF91
:10173000DF91CF911F910F91FF90EF90DF90CF90AD
:10174000BF90089583EC9EE09F938F930E94B19287
:101750000F900F9008952F923F924F925F926F9249
:101760007F928F929F92AF92BF92CF92DF92EF9231
:10177000FF920F931F93CF93DF93EC014B010097E0
:1017800011F427E004C08130910549F426E04AE2D3
:1017900050E06BE270E089E290E00E94B25CCE0122
:1017A0000E94300B9E012154364F5901D9018C9370
:1017B000CD2B69F098E8C92E9BE1D92EC0E8DBE17A
:1017C000E12CF12C24E7222E2EE0322EA6C082EA54
:1017D00098E20E94205FBC01882777FD8095982FB2
:1017E0000E940E896B017C01892869F020E030E0BD
:1017F00048EC52E40E946F889F938F937F936F937E
:1018000081EB9EE0ACC0C2EAD8E20CEA1EE089910E
:101810001F928F931F930F930E94B1920F900F907E
:101820000F900F90B8E2CA3ADB0789F720E030E06A
:1018300048EC52E4C701B6010E946F889F938F93D2
:101840007F936F938CE99EE09F938F930E94B19258
:101850000F900F900F900F900F900F908091AA28EB
:10186000882319F084E993E002C088E094E09F9314
:101870008F9388E99EE09F938F930E94B1920F907F
:101880000F900F900F9075C000E010E0FE01E00F88
:10189000F11F80811F928F93A0E8BEE0BF93AF93AA
:1018A0000E94B1920F5F1F4F0F900F900F900F90FB
:1018B0000830110559F720E030E048EC52E4C3014C
:1018C000B2010E946F889F938F937F936F93A8E7D5
:1018D000BEE0BF93AF930E94B1920F900F900F9014
:1018E0000F900F900F90D6018C91882309F455C06A
:1018F00084E993E09F938F933F922F920E94B1923D
:101900000E94A20BBFEFEB1AFB0AE9E0CE0ED11C3E
:1019100029960F900F900F900F90D5018C9190E029
:10192000E816F906ECF5CE010E94205FBC0188277D
:1019300077FD8095982F0E940E892B013C01811420
:10194000910409F4A1CF20E030E048EC52E40E9479
:101950006F889F938F937F936F9385E89EE09F930B
:101960008F930E94B1920F900F900F900F900F9055
:101970000F90DF91CF911F910F91FF90EF90DF902B
:10198000CF90BF90AF909F908F907F906F905F901F
:101990004F903F902F900C94A20B88E094E0AACF38
:1019A000DF91CF911F910F91FF90EF90DF90CF903B
:1019B000BF90AF909F908F907F906F905F904F906F
:1019C0003F902F900895CF93DF9300D0CDB7DEB72F
:1019D0008091A32889838091A9288A83CE010196CA
:1019E0000E942B520F900F90DF91CF910895CF93CB
:1019F000DF93EC012091A2283091A3284091A428E4
:101A00005091A5286091A6287091A7288091A828B8
:101A10009091A928AFEF0E94208EE1F427E04AE2DE
:101A200050E06BE270E089E290E00E94B25C80E0FE
:101A300090E00E94300BC154D64F888349E050E0BB
:101A40006AE070E082EA98E20E942394DF91CF91ED
:101A50000C94E30CDF91CF9108951F920F920FB673
:101A60000F9211240BB60F92DF92EF92FF920F9319
:101A70001F932F933F934F935F936F937F938F9316
:101A80009F93AF93BF93CF93DF93EF93FF93809197
:101A9000AD2882608093AD288091580286FD2B9AF4
:101AA0008091580287FD2B9A809184029091850243
:101AB0001816190614F4749A739A8091C5099091B6
:101AC000C60985FF02C074987398809102029091B4
:101AD000030201979093030280930202892B09F07D
:101AE0003DC18091D3099091D40901969093D40976
:101AF0008093D3098091232490912424A0912524BC
:101B0000B09126240196A11DB11D809323249093AA
:101B10002424A0932524B093262480E190E0909380
:101B20000302809302028091580280FD02C01D9B37
:101B300007C01092C3091092C20983B7817F09C000
:101B400081E090E09093C3098093C20983B7817FBD
:101B5000866083BF8091C5099091C60997FF08C030
:101B60008091C2099091C309892B61F0749A73988E
:101B700007E21BE1C4E3D4E234E0E32EF12CDD24E0
:101B8000D3941FC0739A7498F3CF8091D309909126
:101B9000D40901960E94F18B892BD1F0F801608560
:101BA00071856115710509F5F8016085718561150B
:101BB000710569F5065F1F4F2596FBE10F341F077E
:101BC000D1F1F801608571856115710539F3DDCFBB
:101BD00077988091C5099091C60992FFDFCF7498DC
:101BE000F0928502E0928402D9CF8091D30990913E
:101BF000D40901960E94F18B892BB1F61C821B82BD
:101C0000AE0162E186E192E00E943754CDCF80912F
:101C1000D3099091D4090E94F18B892B59F6D8826F
:101C20001A8309831C821B82AE0162E184E392E085
:101C30000E943754BFCF60915E0270915F026115C0
:101C40007105A1F18091D3099091D4090E94F18B83
:101C5000892B61F58091882890918928A0918A2804
:101C6000B0918B284091151C5091161C6091171C47
:101C70007091181C841B950BA60BB70B80934F1B00
:101C80009093501BA093511BB093521B80918828B6
:101C900090918928A0918A28B0918B288093151C57
:101CA0009093161CA093171CB093181C60915C02B3
:101CB00070915D0261157105A1F18091D309909138
:101CC000D4090E94F18B892B61F580918C28909129
:101CD0008D28A0918E28B0918F284091191C509189
:101CE0001A1C60911B1C70911C1C841B950BA60B6D
:101CF000B70B8093531B9093541BA093551BB09329
:101D0000561B80918C2890918D28A0918E28B0919F
:101D10008F288093191C90931A1CA0931B1CB093BE
:101D20001C1C8091580286FD2B988091580290913E
:101D30005902A0915A02B0915B0291FF0FC00E941C
:101D4000D1688A3119F0C1E0C80F01C0CBE00E9410
:101D50008B678C2F0E94E9680E94D36740E050E0B7
:101D600060E086E892E00E943754FF91EF91DF91A6
:101D7000CF91BF91AF919F918F917F916F915F9123
:101D80004F913F912F911F910F91FF90EF90DF9016
:101D90000F900BBE0F900FBE0F901F901895809163
:101DA000771B90913324891B08950E94CF0E8823BE
:101DB00071F0E0913324EF71F0E0E453F44E808150
:101DC00090E0209133242F5F2093332408958FEFE8
:101DD0009FEF0895CF93DF93EC011092F0091092DA
:101DE000EF09888199810097C1F08437934021F0F1
:101DF0001982188283E0B6C0613109F0B2C0F8944C
:101E000078940E94D50E99279093EB098093EA0964
:101E10008D3009F441C08F3F49F40E94CF0E8111EB
:101E2000EECF84E793E0998388839BC0823191054C
:101E300009F458C08F37910509F050C08091E80926
:101E40009091E909181619060CF560916D317091A1
:101E50006E3188E090E00E946D9260916D317091DA
:101E60006E3180E290E00E946D9260916D317091D0
:101E70006E3188E090E00E946D928091E809909127
:101E8000E90901979093E9098093E8098091E809AD
:101E90009091E909CF9709F6109233241092771B9D
:101EA0008091E8099091E909FC01E85BFB4D108203
:101EB0009093F0098093EF091092E9091092E809D4
:101EC0008091AB289091AC28009709F4A6CF40E010
:101ED00050E06091FE110E9437549FCF88309105E9
:101EE00071F5ACCF60916D3170916E318DE090E005
:101EF0000E946D921092E7091092E6098091E6091E
:101F00009091E7092091E8093091E9098217930738
:101F10000CF0BCCFFC01E85BFB4D808160916D3122
:101F200070916E3190E00E946D928091E6099091DF
:101F3000E70901969093E7098093E609DFCF609166
:101F40006D3170916E310E946D928091E80990918F
:101F5000E9092091EA09FC01E85BFB4D2083019629
:101F600091CF81E0DF91CF9108958091C209909146
:101F7000C309892BD1F08091580290915902A09108
:101F80005A02B0915B0293FD10C00E948B6783B729
:101F9000817F866083BFF89483B7816083BF789424
:101FA000889583B78E7F83BF78940895CF93DF930E
:101FB000EC0188819981009719F08439904199F456
:101FC0000E9448660E94B50F40E050E065E88091AD
:101FD0000212909103120E94375484E990E1998390
:101FE000888381E003C01982188283E0DF91CF915A
:101FF0000895CF93DF9300D0CDB7DEB7892B81F062
:102000005F934F9381E79EE09F938F9369837A83D9
:102010000E94B1920F900F900F900F907A8169817A
:102020007F936F938EE69EE09F938F930E94B19271
:102030000F900F900F900F900F900F90DF91CF9116
:102040000895FF920F931F93CF93DF930E944866EA
:1020500080EB0E94AD5F81111CC00E9411608091D5
:102060001D2090911E20816090931E2080931D2042
:102070008DE993E09F938F938EE69EE09F938F93DD
:102080000E94B1920F900F900F900F90C1E0D0E09E
:1020900002C0C0E0D0E0FEB08F2D8470F82E729A9E
:1020A0000E9448668EE40E94AD5F811116C00E94B6
:1020B000116080911D2090911E20826090931E20BF
:1020C00080931D208E010F5F1F4F43E259E065EAA8
:1020D00073E0CE010E94F90FE801F11001C072987F
:1020E0000E9448668EEE0E94AD5F811116C00E946C
:1020F000116080911D2090911E20846090931E207D
:1021000080931D208E010F5F1F4F43E259E06DEA5F
:1021100073E0CE010E94F90FE8010E94486686EA4A
:102120000E94AD5F811116C00E94116080911D2038
:1021300090911E20886090931E2080931D208E0118
:102140000F5F1F4F43E259E064EB73E0CE010E9442
:10215000F90FE8010E9448668CE30E94AD5F81118F
:102160001EC00E94116080911D2090911E208061F0
:1021700090931E2080931D208E010F5F1F4F43E21E
:1021800059E06CEB73E0CE010E94F90F86E69EE009
:102190009F938F930E94B1920F900F90E8010E943D
:1021A000486682ED0E94AD5F811116C00E941160E9
:1021B00080911D2090911E20806290931E2080931C
:1021C0001D208E010F5F1F4F43E259E064EC73E066
:1021D000CE010E94F90FE8010E94486680E80E9443
:1021E000AD5F811116C00E94116080911D209091F9
:1021F0001E20916090931E2080931D208E010F5F02
:102200001F4F43E259E06DEC73E0CE010E94F90FDD
:10221000E8010E94486680ED0E94AD5F811116C002
:102220000E94116080911D2090911E2080689093E3
:102230001E2080931D208E010F5F1F4F43E259E047
:1022400063ED73E0CE010E94F90FE8010E94486639
:102250008CEE0E94AD5F811116C00E9411608091CA
:102260001D2090911E20926090931E2080931D202F
:102270008E010F5F1F4F43E259E06BED73E0CE011B
:102280000E94F90FE80107E010E00E9448668CE721
:102290000E94AD5F811113C00E94116080911D20CA
:1022A00090911E20806490931E2080931D2043E215
:1022B00059E062EE73E0CE010E94F90F05C00150B3
:1022C00011090115110509F70E941160DF91CF91E5
:1022D0001F910F91FF900C94A20BCF93DF9300D02E
:1022E000CDB7DEB74A8369830E94E85F6981862F94
:1022F0000E9419604A81842F0E9419600F900F90EC
:10230000DF91CF910C941160AF92BF92DF92EF9268
:10231000FF920F931F93CF93DF9300D01F92CDB7FF
:10232000DEB7182FD22E4A835B8369830E94E85F51
:102330006981862F0E941960812F81600E940F6041
:102340004A81A42E5B81B52E00E010E0ED2CF12C2B
:1023500081E0E81AF1080D1580F40E151F0519F437
:102360000E94346002C00E942A60F50180830F5FE2
:102370001F4FFFEFAF1ABF0AEECF0F900F900F90D5
:10238000DF91CF911F910F91FF90EF90DF90BF9061
:10239000AF900C941160AF92BF92CF92DF92EF9208
:1023A000FF920F931F93CF93DF93CDB7DEB7609764
:1023B0000FB6F894DEBF0FBECDBFB82EA42E662395
:1023C000E9F18E010F5F1F4F80E1F80111928A95AC
:1023D000E9F728E0A80168E980EB0E948411BB209E
:1023E00041F02BEE33E03F932F930E949F920F908A
:1023F0000F906E01F8E0CF0ED11C52EFE52E53E0A6
:10240000F52EF80181918F011F928F93FF92EF9229
:102410000E949F920F900F900F900F900C151D052A
:1024200081F788851F928F9327E434E03F932F93A1
:102430000E949F920F900F900F900F90AA20E9F1A9
:102440008E010F5F1F4F80E1F80111928A95E9F725
:1024500028E0A80160E880EB0E948411BB2041F0D5
:1024600087EF93E09F938F930E949F920F900F901E
:102470006E01F0E1CF0ED11C42EFE42E43E0F42ECA
:10248000F80181918F011F928F93FF92EF920E942A
:102490009F920F900F900F900F900C151D0581F7D4
:1024A00088851F928F9387E494E09F938F930E9477
:1024B0009F920F900F900F900F9060960FB6F89428
:1024C000DEBF0FBECDBFDF91CF911F910F91FF9067
:1024D000EF90DF90CF90BF90AF900895CF93DF93B0
:1024E00000D0CDB7DEB71A82198222E0AE014F5F6D
:1024F0005F4F6AEA8EEE0E948411898190E0982FE6
:1025000088272A81822B9093ED1B8093EC1B22E07D
:10251000AE014F5F5F4F6CEA8EEE0E94841189819D
:1025200090E0982F88272A81822B9093EF1B80932D
:10253000EE1B22E0AE014F5F5F4F6EEA8EEE0E940F
:102540008411898190E0982F88272A81822B90938B
:10255000F11B8093F01B22E0AE014F5F5F4F60EBF9
:102560008EEE0E948411898190E0982F88272A811D
:10257000822B9093FF1B8093FE1B22E0AE014F5FE6
:102580005F4F62EB8EEE0E948411898190E0982F5C
:1025900088272A81822B9093011C8093001C22E0C3
:1025A000AE014F5F5F4F64EB8EEE0E948411898114
:1025B00090E0982F88272A81822B9093031C809388
:1025C000021C22E0AE014F5F5F4F66EB8EEE0E9471
:1025D0008411898190E0982F88272A81822B9093FB
:1025E000F31B8093F21B22E0AE014F5F5F4F68EB5D
:1025F0008EEE0E948411898190E0982F88272A818D
:10260000822B9093F51B8093F41B22E0AE014F5F69
:102610005F4F6AEB8EEE0E948411898190E0982FC3
:1026200088272A81822B9093F91B8093F81B22E044
:10263000AE014F5F5F4F6CEB8EEE0E94841189817B
:1026400090E0982F88272A81822B9093FB1B809300
:10265000FA1B22E0AE014F5F5F4F6EEB8EEE0E94E1
:102660008411898190E0982F88272A81822B90936A
:10267000FD1B8093FC1B0F900F90DF91CF9108956D
:102680002F923F924F925F926F927F928F929F9282
:10269000AF92BF92CF92DF92EF92FF920F931F9370
:1026A000CF93DF93CDB7DEB76A970FB6F894DEBF4E
:1026B0000FBECDBF182F488F298F19821A821B8217
:1026C0008091101C811107C06A8F0E946E1281E0F8
:1026D0008093101C6A8D662309F46CC04EE264EF8F
:1026E0008EEE0E946D1169E07AE180E090E00E9438
:1026F0008B5F22E0AE014F5F5F4F66EF8EEE0E9470
:1027000084112981822F90E0A0E0B0E02227382FA9
:10271000492F5A2F8A81282B8091021C9091031CEB
:10272000281B390B41095109A091001CB091011CD3
:102730000E94CE8B6B017C018FE0F594E794D794D7
:10274000C7948A95D1F76091FA1B7091FB1B88277B
:1027500077FD8095982F2BE0660F771F881F991FB4
:102760002A95D1F72091FC1B3091FD1B442737FDA2
:102770004095542F2C0D3D1D4E1D5F1D0E943B8C1E
:10278000C20ED31ED092F71BC092F61B88E0C80E73
:10279000D11C34E0D594C7943A95E1F7EE24D7FCE8
:1027A000E094FE2CC092041CD092051CE092061C02
:1027B000F092071C012F0295000F000F007C0C5CAB
:1027C000A12FB0E0BD8BAC8BA3E0B0E0012E02C026
:1027D000AA0FBB1F0A94E2F725E335E00E94C78BDE
:1027E000DC01CB010296A11DB11D8C879D87AE87B0
:1027F000BF8780E593ECA0E0B0E004C0B595A79555
:10280000979587951A95D2F7888B998BAA8BBB8B56
:1028100010E0188619861A861B86A8E02A2E312C0D
:10282000AC89BD892A1A3B0A988D191709F436C15B
:10283000402F64EF8EEE0E946D116C857D858E8534
:102840009F850E948B5F23E0AE014F5F5F4F66EF75
:102850008EEE0E948411E091F61BF091F71BE05A76
:10286000FF409F01DF010E94B08B6B017C018091D2
:10287000EE1B9091EF1B9F8B8E8BA090EC1BB0906A
:10288000ED1B2091F01B3091F11B0E94B08B2B01AE
:102890003C013DE075946794579447943A95D1F77D
:1028A000A091F21BB091F31BA70196016CE0559526
:1028B0004795379527956A95D1F70E94D98BBB2705
:1028C00097FDB095AB2F480E591E6A1E7B1E92E0F5
:1028D000490E511C611C711CB2E0759467945794A9
:1028E0004794BA95D1F7A0E85A0E611C711CA091CB
:1028F000FE1BB091FF1BA30192010E94CE8BDC0155
:10290000CB012FE0B695A795979587952A95D1F796
:102910008C839D83AE83BF8329818A8190E0A0E070
:10292000B0E04424582E692E7A2E622A8B81482AE0
:10293000022C04C075946794579447940A94D2F774
:102940004501AA2497FCA094BA2C42E0880C991C5B
:10295000AA1CBB1C4A95D1F7A091F41BB091F51BA2
:10296000A70196010E94D98B6B017C0157E1F59478
:10297000E794D794C7945A95D1F72E893F89DF0100
:102980000E94B08BEBE09595879577956795EA95D2
:10299000D1F7C60ED71EE81EF91E8C0C9D1CAE1C6E
:1029A000BF1C0C8804C0880C991CAA1CBB1C0A9470
:1029B000D2F792E0890E911CA11CB11CF2E0B594F3
:1029C000A79497948794FA95D1F7481859086A08FC
:1029D0007B08A3019201688979898A899B890E9471
:1029E000E18B97FD0DC0660F771F881F991F2C8103
:1029F0003D814E815F810E94198C49015A010CC0B2
:102A00002C813D814E815F810E94198C49015A01C0
:102A1000880C991CAA1CBB1C9927B7FC9A958B2D76
:102A20007A2D692D9B01AC010E94E18B9B01AC01C9
:102A3000AEEDBBE00E94CE8B6C01FF24D7FCF0947E
:102A4000EF2CA3E4B3EEA50194010E94DC8BBB271D
:102A500097FDB095AB2FC80ED91EEA1EFB1EAFEC3A
:102A6000CA0EAEE0DA1EE11CF11CA4E0F594E79476
:102A7000D794C794AA95D1F7C80CD91CEA1CFB1CA3
:102A800088859985AA85BB858C0D9D1DAE1DBF1DB2
:102A900088879987AA87BB871F5FC6CE112391F0CD
:102AA000212F30E040E050E0688579858A859B855C
:102AB0000E94198C2093081C3093091C40930A1C17
:102AC00050930B1CA98DAA2389F16091081C709169
:102AD000091C80910A1C90910B1C611571058105E0
:102AE000910521F10E940E8920E836EE45EC57E46D
:102AF0000E946F8821E03EED42E45EE30E94538B2A
:102B00009B01AC0160E070E080E89FE30E94A48735
:102B10002BE43AE34DEB57E30E946F8860930C1C63
:102B200070930D1C80930E1C90930F1C6A960FB629
:102B3000F894DEBF0FBECDBFDF91CF911F910F91F3
:102B4000FF90EF90DF90CF90BF90AF909F908F90CD
:102B50007F906F905F904F903F902F9008950F93CC
:102B60001F93CF93DF9300D000D000D0CDB7DEB756
:102B70008E010F5F1F4F86E0F80111928A95E9F7E9
:102B800080911E1B811113C040E061E386EA0E9420
:102B90006D114AE06CE286EA0E946D1181E080933B
:102BA0001E1B6CE77EE380E090E00E948B5F48E0B4
:102BB0006DE286EA0E946D116CE77EE380E090E0B2
:102BC0000E948B5F26E0A80162E386EA0E948411DE
:102BD00047E06DE286EA0E946D118A8190E0982FAD
:102BE00088272981822B9093191B8093181B2C8195
:102BF00030E0322F22274B81242B30931B1B209354
:102C00001A1B4E8150E0542F44276D81462B509360
:102C10001D1B40931C1B5F934F933F932F939F93D8
:102C20008F938BEF93E09F938F930E949F920FB6A9
:102C3000F894DEBF0FBECDBF26960FB6F894DEBF68
:102C40000FBECDBFDF91CF911F910F910895CF920D
:102C5000DF92EF92FF920F931F93CF93DF93CDB745
:102C6000DEB72A970FB6F894DEBF0FBECDBF8E0138
:102C70000F5F1F4F86E0F80111928A95E9F741E056
:102C800062E08CE30E946D1148E560E08CE30E94F5
:102C90006D1162E174E380E090E00E948B5F26E0BA
:102CA000A80163E08CE30E94841143E062E08CE3BE
:102CB0000E946D11098110E0102F00278A81082BD6
:102CC0001093F91A0093F81AEB80F12CFE2CEE24E5
:102CD0008C81E82AF092FB1AE092FA1ACD80D12C6E
:102CE000DC2CCC248E81C82AD092FD1AC092FC1A0A
:102CF000B801882777FD8095982F0E940E899B0147
:102D0000AC01B701882777FD8095982F2F833887EE
:102D100049875A870E940E892F81388549855A85AF
:102D20000E94188820EE3EE245E652E40E94F08AB6
:102D300020E030E044E353E40E94A5879F938F9303
:102D40007F936F93DF92CF92FF92EF921F930F9337
:102D500089E094E09F938F930E949F920FB6F8941E
:102D6000DEBF0FBECDBF2A960FB6F894DEBF0FBEF2
:102D7000CDBFDF91CF911F910F91FF90EF90DF902A
:102D8000CF900895CF93DF93EC01888199810097CC
:102D9000F9F08D37904121F01982188283E063C0E9
:102DA00085ED99E00E94DD56892BE1F08091C509FF
:102DB0009091C60993FD18C08091C5099091C609EC
:102DC00094FD43C08091C5099091C60995FD44C00A
:102DD00060E870E085ED99E00E94B6568DE790E1DD
:102DE0009983888381E03FC080911D2082FFE4CFDA
:102DF00021E048E061E083E00E94401380910F1CD5
:102E00008F9380910E1C8F9380910D1C8F938091D6
:102E10000C1C8F9380910B1C8F9380910A1C8F93B5
:102E20008091091C8F938091081C8F9385EC9EE004
:102E30009F938F930E94B1928DB79EB70A960FB65B
:102E4000F8949EBF0FBE8DBFB7CF80911D2083FF2A
:102E5000B9CF0E94AF15B6CF80911D2084FFB8CFA7
:102E60000E942716B5CFDF91CF910895CF93C82F39
:102E70008CEE0E940F608C2F0E94196065E375E054
:102E800080E090E00E948B5F8DEE0E940F600E94B8
:102E90002A60C82F0E9434602C2F30E0322F222766
:102EA000A901482BCA01CF910895CF93DF93C82F72
:102EB0008CEE0E940F608C2F0E94196062E174E317
:102EC00080E090E00E948B5F8CEE0E940F6080E0BB
:102ED0000E94196065E375E080E090E00E948B5FDE
:102EE0008DEE0E940F600E942A60C82F0E942A6007
:102EF000D82F0E9434604D2F50E060E070E0762FB4
:102F0000652F542F44276C2B482BCB01BA01DF913E
:102F1000CF9108952F923F924F925F926F927F923E
:102F20008F929F92AF92BF92CF92DF92EF92FF92D9
:102F30000F931F93CF93DF93CDB7DEB7CD54D10955
:102F40000FB6F894DEBF0FBECDBF80910002909106
:102F50000102892BD1F110920102109200028CEE35
:102F60000E940F608EE10E9419606BE17EE480E0B8
:102F700090E00E948B5F82EA0E9436179093D209FC
:102F80008093D10984EA0E9436179093D0098093E8
:102F9000CF0986EA0E9436179093CE098093CD0917
:102FA00088EA0E9436179093CC098093CB098AEA6D
:102FB0000E9436179093CA098093C9098CEA0E942F
:102FC00036179093C8098093C70988E40E94551763
:102FD0006FAB78AF89AF9AAF88E50E9455174B0168
:102FE0005C018091C9099091CA0920E030E040E07D
:102FF00050E0BA0126962FAF269727963FAF279726
:1030000028964FAF289729965FAF29972A966FAFDA
:103010002A972B967FAF2B979C0140E050E060E011
:1030200070E080E090E008E00E94C28D0E946E8D0A
:103030003901B42FA52FF62FE72F8C019401A5019C
:1030400060E070E080E090E05301CB2EDA2EEF2EAE
:10305000FE2E0E94F98D29833A832A011B014C011F
:10306000B101C401315041095F4F6F4F7F4F8F4F06
:103070009F4FA1E0B0E02596BFAFAEAF25972115D9
:103080003F4F4F4F5140610571058105910509F092
:1030900020F425961FAE1EAE259725966EAC7FAC0C
:1030A00025978091C7099091C8095C01C12CD12C4A
:1030B000E12CF12C00E010E029813A81A201B1015C
:1030C000C4010E94918CD22EE32EF42E052F162FD0
:1030D000B72FF82FE92FA0E00E94208E84F4215012
:1030E000310940485F4F6F4F7F4F8F4F9F4FD22E18
:1030F000E32EF42E052F162FB72FF82FE92F2D2DA5
:103100003E2D4F2D502F612F7B2F8F2F9E2F07E1AC
:103110000E94DB8D2B8F3C8F4D8F5E8F6F8F78A33E
:1031200089A39AA32053384F4F4F5F4F6F4F7F4F64
:103130008F4F9F4F2B8B3C8B4D8B5E8B6F8B788F84
:10314000898F9A8F2056304F4F4F5F4F6F4F7F4F71
:103150008F4F9F4F243D3043410551056105710557
:103160008105910541F038F025966EAC7FAC25972E
:10317000FFEF6F1A7F0A8091CF099091D0099C01CF
:1031800040E050E060E070E080E090E000E10E940C
:10319000C28D2B833C834D835E836A8779878F83BF
:1031A00098874091CB095091CC09A980BA806201DF
:1031B000710184019A0140E050E060E070E080E03D
:1031C00090E00E94918CD22EE32EF42E052F162F24
:1031D000B72FF82FE92FA0E00E94208E5CF4AFE714
:1031E0000E94028ED22EE32EF42E052F162FB72F1B
:1031F000F82FE92F2D2D3E2D4F2D502F612F7B2F96
:103200008F2F9E2F07E00E94DB8D59016A017B0101
:103210008C012B813C814D815E816A8579858F810E
:1032200098850E94F98D2B833C834D835E836F8349
:1032300078878F87988B2E5F3F4F434051096E4FA1
:103240007F4F8F4F9F4F22303105494F5F4F644072
:1032500071058105910521F018F01FEF611A710ABF
:103260008091D1099091D209BC0180E090E020E0EA
:1032700030E840E050E00E94EA8C29873A874B878B
:103280005C876A8B798B8D879E874091CD095091A1
:10329000CE09A980BA806201710184019A0140E0DF
:1032A00050E060E070E080E090E00E94918CD22ECF
:1032B000E32EF42E052F162FB72FF82FE92FA0E0BD
:1032C0000E94208E84F421503F4F4F4F5F4F6F4F2D
:1032D0007F4F8F4F9F4FD22EE32EF42E052F162FA8
:1032E000B72FF82FE92F2D2D3E2D4F2D502F612F69
:1032F0007B2F8F2F9E2F08E00E94DB8D59016A01E2
:103300007B018C0129853A854B855C856A897989A1
:103310008D859E850E94F98D29873A874B875C872A
:103320006D877E87898B9A8B2F5F3F4F4140510974
:103330006109710981099109213030484C4F5F477B
:10334000614071058105910521F018F0BFEF6B1AFE
:103350007B0A2B893C894D895E896F89788D898D9F
:103360009A8D2F3C37404105510561057105810556
:10337000910511F00CF0A5C1A980BA80620171011C
:1033800084019501A201B101C4010E94918CA12C7C
:10339000B12CC12C10E8D12EE12CF12C00E010E072
:1033A0000E94548C2BAF3CAF4DAF5EAF6FAF2196F8
:1033B0007FAF219722968FAF229723969FAF2397B7
:1033C000AB8CBC8CCD8CDE8CEF8CF8A009A11AA143
:1033D0009501A601B701C8010E94918C59016A01AB
:1033E0007B01E82F192F02E00E94C28D0E2F0E9450
:1033F000F98D69017A01162F272EF82FE92F322E29
:103400008D2C942EAF2CB62E072F582EB92FA0E05E
:103410000E94208E5CF4A1E00E94028E322E832E48
:10342000942EA52EB62E072F582EB92F232D382DCA
:10343000492D5A2D6B2D702F852D9B2F01E00E9459
:10344000DB8D2E962FAF2E972D963FAF2D9749A748
:103450005AA76BA77CA78DA79EA7522E432E4BA3DE
:103460005CA36DA37EA38FA398A7B22D9601A7019D
:10347000612F722D8F2F9E2FA0E00E94208E4CF482
:10348000A3E00E94028E69017A01162FB72FF82F50
:10349000E92F9601A701612F7B2F8F2F9E2F02E02E
:1034A0000E94DB8D2FA738AB49AB5AAB6BAB7CAB23
:1034B0008DAB9EAB19014A01B62FA72F24968FAF73
:1034C0002497F92F2B893C894D895E896F89788DE6
:1034D000898D9A8D24323A4F4F4F5F4F6F4F7F4FF8
:1034E0008F4F9F4F0CF08CC02B8D3C8D4D8D5E8D82
:1034F0006F8D78A189A19AA12455324F4F4F5F4F0C
:103500006F4F7F4F8F4F9F4F59016A017B018C0195
:103510000E94918C19014A01B62FA72FFC0103E0EC
:103520000E94C28D51016401EB2EFA2E8F010E9480
:103530000E8E59016A017B018C012E962FAD2E97BC
:103540002D963FAD2D9749A55AA56BA57CA58DA5B8
:103550009EA50E94F98D522E432E4BA35CA36DA312
:103560007EA38FA398A79101A4016B2F7A2FCF017F
:1035700002E00E94C28D51016401EB2EFA2E8F01F0
:103580000E940E8E02E00E94C28D0E2F0E940E8EAF
:10359000F22E032F142FD52EE62EB72FF82FE92F5A
:1035A000A0E00E94208E5CF4A1E00E94028EF22E28
:1035B000032F142FD52EE62EB72FF82FE92F2F2DFE
:1035C000302F412F5D2D6E2D7B2F8F2F9E2F01E0F1
:1035D0000E94DB8D59016A017B018C012FA538A95E
:1035E00049A95AA96BA97CA98DA99EA90E94F98D08
:1035F00019014A01B62FA72F24968FAF2497F92FD0
:103600002B813C814D815E816F8178858F85988982
:10361000A52CB42CCBA0DCA0EDA0FEA00FA118A57A
:103620000E940E8E2B833C834D835E836F8378874D
:103630008F87988B29853A854B855C856D857E853E
:1036400089899A8951016401EB2EFA2E24960FADD7
:1036500024971F2F0E940E8E29873A874B875C87FD
:103660006D877E87898B9A8B2B893C894D895E89F2
:103670006F89788D898D9A8DABACBCACCDACDEAC4E
:10368000EFAC2196FFAC219722960FAD229723969F
:103690001FAD23970E940E8E2056304F4F4F5F4F25
:1036A0006F4F7F4F8F4F9F4F243D30434105510552
:1036B000610571058105910521F018F02FEF621A5F
:1036C000720A6FA978AD89AD9AADAB01BC0180E0FB
:1036D00090E0DC0124964FAF249725965FAF2597A5
:1036E00026966FAF269727967FAF279728968FAF9E
:1036F000289729969FAF29972A96AFAF2A972B969E
:10370000BFAF2B97A984BA84CB84DC84ED84FE847C
:1037100009891A899A01AB0160E070E080E090E0CD
:103720000E94918CF22E032F142FD52EE62EB72F48
:10373000F82FE92FA0E00E94208E84F42150310957
:10374000404E5F4F6F4F7F4F8F4F9F4FF22E032F93
:10375000142FD52EE62EB72FF82FE92F2F2D302F2F
:10376000412F5D2D6E2D7B2F8F2F9E2F05E10E9407
:10377000DB8DAB80BC80CD80DE80EF80F8840F8550
:1037800018890E940E8EF22E032F142FD52EE62EAE
:10379000B72FF82FE92FA0E00E94208E84F421504B
:1037A00030484F4F5F4F6F4F7F4F8F4F9F4FF22EDD
:1037B000032F142FD52EE62EB72FF82FE92F2F2DFC
:1037C000302F412F5D2D6E2D7B2F8F2F9E2F0FE0E1
:1037D0000E94DB8D69017A018B018A83998329011B
:1037E0001A014B015C01285E33404109510961090E
:1037F000710981099109283D304D4140510561050C
:1038000071058105910521F018F0BFEF6B1A7B0A55
:103810000E941160672859F09601A701B8018A81BA
:1038200099810E946E8D29011A014B015C01920160
:10383000A101B401C5010E94088920E030E048ECF4
:1038400052E40E946F88C35BDF4F0FB6F894DEBF6F
:103850000FBECDBFDF91CF911F910F91FF90EF90E1
:10386000DF90CF90BF90AF909F908F907F906F90A0
:103870005F904F903F902F9008954F925F926F927C
:103880007F928F929F92AF92BF92CF92DF92EF92F0
:10389000FF922B013C0169017A0123EC35EF4CE8E2
:1038A00051E4C701B6010E94F08A4B015C0128EB8C
:1038B0003EE143E753E4C701B6010E94A5879B019F
:1038C000AC01C501B4010E946F880E94DC884B01E5
:1038D0005C0120E030E048EC52E4C301B2010E94F8
:1038E0006F8821E835E943EC50E40E94F08AA50195
:1038F00094010E94F08A4B015C0123E333E948E81C
:1039000053E4C701B6010E94A5879B01AC01C50124
:10391000B4010E946F8823E333EB48E553E40E942F
:10392000F08AFF90EF90DF90CF90BF90AF909F9084
:103930008F907F906F905F904F9008954F925F921D
:103940006F927F928F929F92AF92BF92CF92DF92AF
:10395000EF92FF9269017A010E94728A20E030E0C2
:1039600040E050E40E94A48722E93CE54EED5EE38E
:103970000E946F884B015C0123EC35EF4CE851E469
:10398000C701B6010E94F08A2B013C0128EB3EE101
:1039900043E753E4C701B6010E94A5879B01AC0130
:1039A000C301B2010E946F889B01AC01C501B40143
:1039B0000E94A5876B017C0128EB3EE143E753E4BD
:1039C0000E94F08A4B015C01A701960163EC75EF40
:1039D0008CE891E40E94A4879B01AC01C501B4016D
:1039E0000E946F88FF90EF90DF90CF90BF90AF90D4
:1039F0009F908F907F906F905F904F9008954F921F
:103A00005F926F927F928F929F92AF92BF92CF926E
:103A1000DF92EF92FF922B013C0169017A0123ECC6
:103A200035EF4CE851E4C701B6010E94F08A4B0122
:103A30005C0128EB3EE143E753E4C701B6010E9475
:103A4000A5879B01AC01C501B4010E946F880E944B
:103A5000DC884B015C0120E030E048EC52E4C3011B
:103A6000B2010E946F88A50194010E94F08A20E0B3
:103A700030E040E251E40E94A48724EE38E34EE0B7
:103A80005FE30E94F08A9B01AC01C701B6010E946E
:103A9000A587FF90EF90DF90CF90BF90AF909F9061
:103AA0008F907F906F905F904F90089580E80E9474
:103AB0000F6081110DC08EEF0E941960811108C046
:103AC0006BE17EE480E090E00E948B5F0C941160DB
:103AD0000E94116080912F2490913024A091312474
:103AE000B09132240196A11DB11D80932F24909393
:103AF0003024A0933124B09332240895FC01DC01DA
:103B000082E020E041E39D91292798E0322F330F96
:103B100027FF03C0232F242701C0232F9150B1F783
:103B2000815089F781E090E03281231711F080E025
:103B300090E00895DF92EF92FF920F931F93CF933F
:103B4000DF930E94561D80E80E940F6081116DC0B6
:103B50008AEF0E941960811168C08FE00E9419608D
:103B6000811163C065E375E080E090E00E948B5FA7
:103B700081E80E940F60811158C00E942A60C82FFE
:103B80000E942A600E942A60D82F0E942A600E9408
:103B90002A60182F0E942A600E943460082F80E853
:103BA0000E940F60811141C08CEF0E941960811149
:103BB0003CC089EC0E941960811137C065E375E053
:103BC00080E090E00E948B5F81E80E940F600E947D
:103BD0002A60E82E0E942A60D82E0E942A600E9445
:103BE0002A60F82E0E9434601F92DF921F92EF929B
:103BF0001F920F931F921F931F92DF931F92CF93D9
:103C00001F928F931F92FF928EE194E09F938F9368
:103C10000E949F920E9411608DB79EB742960FB688
:103C2000F8949EBF0FBE8DBF17C00E941160809197
:103C30002F2490913024A0913124B0913224019608
:103C4000A11DB11D80932F2490933024A093312483
:103C5000B09332240E94561D20E030E040E050E056
:103C600060E070E080E090E0DF91CF911F910F91D4
:103C7000FF90EF90DF900895EF92FF920F931F93C4
:103C8000CF93DF9300D01F92CDB7DEB78C0180E8D1
:103C90000E940F60811154C00115110551F085EE8D
:103CA0000E94196081114CC061E077E980E090E0EA
:103CB00009C083EE0E941960811142C069E97AEB64
:103CC00081E090E00E948B5F81E80E940F6081118B
:103CD00037C00E942A60F82E89830E942A60E82E4D
:103CE0008A830E9434608B830E941160CE0101960A
:103CF0000E947E1D892B21F16E2D70E07F296C7F43
:103D000080E090E0012B69F00E940C8920E030E017
:103D10004AEF5AE30E94F08A20E030E040EC50E4A1
:103D20000CC00E940C8922E538EB4FE25BE30E9455
:103D3000F08A26E636E64BE352E40E94A4871BC0D5
:103D40000E94116080912F2490913024A091312401
:103D5000B09132240196A11DB11D80932F24909320
:103D60003024A0933124B09332240E94561D60EF7A
:103D70007FEF89E794E40F900F900F90DF91CF9140
:103D80001F910F91FF90EF9008950F931F93CF9382
:103D9000DF93729A8091580283FF08C08EE40E94DC
:103DA000AD5F811163C0C0E5D0E008C0C0E5D0E0E0
:103DB0000E94AF0921972097D9F7F0CF0E94AF0951
:103DC00021972097D9F78FE40E94AD5F0E942A6067
:103DD000082F0F730E942A60182F0E942A60D82F84
:103DE0000E943460C82F0E9411608091580283FFA6
:103DF0007298602F70E0762F6627610F711D80E04A
:103E000090E00E940C8920E134E048EC5BE30E94E2
:103E1000F08A6093111C7093121C8093131C909372
:103E2000141C6D2F70E0762F66276C0F711D769530
:103E300067957695679580E090E00E940C8924EA6A
:103E40003CEF44E25CE30E94F08A20E030E040E294
:103E500052E40E94A4876093AE287093AF288093A9
:103E6000B0289093B12880E090E002C081E090E01B
:103E7000DF91CF911F910F9108957298729A8EE4FD
:103E80000E94AD5F80EA0E94196080E00E94196084
:103E900080E00E9419608FE40E94AD5F0E942A605A
:103EA0008EE40E94AD5F80E80E94196080E00E946D
:103EB000196080E00E9419600E94116080E090E02B
:103EC000089589E59EE09F938F930E94B19280911F
:103ED00073020F900F90882361F01F928F9386E5F5
:103EE0009EE09F938F930E94B1920F900F900F903E
:103EF0000F90089581E39EE09F938F930E94B1926B
:103F000089E09EE09F938F930E94B19282EE9DE0A4
:103F10009F938F930E94B19287EA9DE09F938F9326
:103F20000E94B19285E79DE09F938F930E94B1928A
:103F300089E39DE09F938F930E94B19283E19DE07E
:103F40009F938F930E94B1928DED9CE09F938F93EE
:103F50000E94B19280911D2090911E2082709170DC
:103F60002DB73EB7205F3F4F0FB6F8943EBF0FBE50
:103F70002DBF892B41F08DEA9CE09F938F930E9487
:103F8000B1920F900F9081E89CE09F938F930E94D5
:103F9000B19285E49CE09F938F930E94B1928CE153
:103FA0009CE09F938F930E94B19280EF9BE09F9340
:103FB0008F930E94B19281EC9BE09F938F930E941C
:103FC000B1928FE89BE09F938F930E94B1928EE510
:103FD0009BE09F938F930E94B19284E29BE09F931A
:103FE0008F930E94B1928EEE9AE09F938F930E94DE
:103FF000B1928EEB9AE09F938F930E94B19282E9E7
:104000009AE09F938F930E94B19283E69AE09F93E8
:104010008F930E94B1928AE29AE09F938F930E94BD
:10402000B19281EF99E09F938F930E94B1928AEBB6
:1040300099E09F938F930E94B19289E899E09F93B2
:104040008F930E94B1928DB79EB780960FB6F89469
:104050009EBF0FBE8DBF8AE599E09F938F930E940C
:10406000B1928BE299E09F938F930E94B19284E08A
:1040700099E09F938F930E94B1928EEC98E09F936A
:104080008F930E94B19288E998E09F938F930E944A
:10409000B19282E698E09F938F930E94B19289E358
:1040A00098E09F938F930E94B19281E098E09F9354
:1040B0008F930E94B19286ED97E09F938F930E9419
:1040C000B1922DB73EB72E5E3F4F0FB6F8943EBF6C
:1040D0000FBE2DBF08958DE494E00C94D5924F92BD
:1040E0005F926F927F928F929F92AF92BF92CF9288
:1040F000DF92EF92FF92CF93DF93CDB7DEB7289791
:104100000FB6F894DEBF0FBECDBF809123249091EF
:104110002424A0912524B091262489839A83AB83FB
:10412000BC834090232450902424609025247090D8
:1041300026248091232490912424A0912524B091B9
:1041400026248D839E83AF83B8876091232470914A
:10415000242480912524909126242CE3822E912CD6
:10416000A12CB12CA50194010E94198C7F936F930F
:1041700030E1C32E3EE0D32EE12CF12C6D817E8107
:104180008F819885A70196010E94198CA501940141
:104190000E94198C3F932F9340E8842E41E5942E82
:1041A000AA24A394B12CC301B201A50194010E94D9
:1041B000198CA70196010E94198C3F932F93698156
:1041C0007A818B819C81A50194010E94198C3F9377
:1041D0002F9380EB97E09F938F930E94B1920FB63D
:1041E000F894DEBF0FBECDBF28960FB6F894DEBFA1
:1041F0000FBECDBFDF91CF91FF90EF90DF90CF90BA
:10420000BF90AF909F908F907F906F905F904F90F6
:104210000895E3E7F1E3808191818234924479F05B
:10422000E357F143FF93EF9382E997E09F938F93D6
:104230000E94B1920F900F900F900F9008953A96B0
:10424000E53F81E4F80738F30895CF93DF93EC015D
:104250008C9A0E94920A9F938F937F936F9386E824
:1042600097E09F938F930E94B1920F900F900F90C1
:104270000F900F900F90209719F00E94A20B08C08A
:1042800084E897E09F938F930E94B1920F900F90D4
:1042900081E00E94430A2091780230917902409196
:1042A0007A0250917B020E94F08A9F938F937F93B2
:1042B0006F9388E797E09F938F930E94B1920F903E
:1042C0000F900F900F900F900F90209719F00E9471
:1042D000A20B08C086E797E09F938F930E94B1924C
:1042E0000F900F9082E00E94430A20917402309157
:1042F000750240917602509177020E94F08A9F9356
:104300008F937F936F938AE697E09F938F930E949A
:10431000B1920F900F900F900F900F900F902097E9
:1043200019F00E94A20B08C088E697E09F938F9334
:104330000E94B1920F900F9083E00E94430A9F93D6
:104340008F937F936F9389E597E09F938F930E945C
:10435000B1928C980F900F900F900F900F900F903C
:10436000209719F00E94A20B08C087E597E09F9361
:104370008F930E94B1920F900F9080911D2087FF24
:1043800083C021E042E161E080ED0E9471619F9372
:104390008F937F936F938AE497E09F938F930E940C
:1043A000B1920F900F900F900F900F900F90209759
:1043B00019F00E94A20B08C088E497E09F938F93A6
:1043C0000E94B1920F900F9021E042E162E080EDF7
:1043D0000E9471619F938F937F936F938BE397E01C
:1043E0009F938F930E94B1920F900F900F900F9018
:1043F0000F900F90209719F00E94A20B08C089E33C
:1044000097E09F938F930E94B1920F900F9021E0BD
:1044100042E163E080ED0E9471619F938F937F93EF
:104420006F938CE297E09F938F930E94B1920F90CD
:104430000F900F900F900F900F90CD2B19F00E94BE
:10444000A20B08C08AE297E09F938F930E94B192DB
:104450000F900F9021E042E164E080ED0E947161D5
:104460009F938F937F936F938DE197E09F938F93AB
:104470000E94B1920F900F900F900F900F900F909D
:10448000DF91CF910C94A20BCD2BD1F3DF91CF9183
:1044900008950F931F93CF93DF93882389F049E00A
:1044A00050E06FEF70E082EA98E20E94F39149E0F9
:1044B00050E06AE070E082EA98E20E94239413C020
:1044C000C2EAD8E208E117E089911F928F931F9307
:1044D0000F930E94B1920F900F900F900F9088E26F
:1044E000CA3AD80789F7DF91CF911F910F910C94A9
:1044F000A20BCF92DF92EF92FF92CF93DF936B01EB
:104500007C0160FF11C08AE894E09F938F938EE650
:104510009EE09F938F930E94B1920F900F900F9007
:104520000F9081E090E002C080E090E0C1FE09C001
:10453000EC01219643E259E06FE874E00E94F90F24
:10454000CE01C2FE09C0EC01219643E259E067E9C1
:1045500074E00E94F90FCE01C3FE09C0EC01219660
:1045600043E259E06FE974E00E94F90FCE01C4FE06
:1045700009C0EC01219643E259E063EA74E00E942D
:10458000F90FCE01C5FE09C0EC01219643E259E0C6
:1045900066EA74E00E94F90FCE01C6FE09C0EC0184
:1045A000219643E259E06AEA74E00E94F90FCE01D5
:1045B000C7FE09C0EC01219643E259E060EB74E0CC
:1045C0000E94F90FCE01D0FE09C0EC01219643E212
:1045D00059E068EB74E00E94F90FCE01D1FE09C0EA
:1045E000EC01219643E259E060EC74E00E94F90F7F
:1045F000CE01D2FE09C0EC01219643E259E064EC01
:1046000074E00E94F90FCE0120911D2030911E20F0
:1046100024703270232B59F0D3FE09C0EC0121968F
:1046200043E259E06AEC74E00E94F90FCE01209158
:104630001D2023FF0BC0D4FE09C0EC01219643E2EC
:1046400059E06FEC74E00E94F90FCE0120911D201B
:1046500024FF0BC0D5FE09C0EC01219643E259E0CE
:1046600065ED74E00E94F90FCE01D6FE09C0EC01A1
:10467000219643E259E06DED74E00E94F90FCE01FE
:10468000B701A60144275078452B462B472B61F0F4
:1046900043E259E068EE74E0DF91CF91FF90EF9034
:1046A000DF90CF900C94F90FCD28CE28CF2841F47D
:1046B00083E197E09F938F930E94B1920F900F90A8
:1046C000DF91CF91FF90EF90DF90CF9008950F93FF
:1046D0001F93CF93DF938C01C0E0D0E0011511054B
:1046E00009F48AC06EE077E0C8010E94D291892B5C
:1046F00009F4C16066E077E0C8010E94D291892B7D
:1047000009F4C2606EEF76E0C8010E94D291892B55
:1047100009F4C4606AEF76E0C8010E94D291892B47
:1047200009F4C86067EF76E0C8010E94D291892B36
:1047300009F4C06163EF76E0C8010E94D291892B31
:1047400009F4C0626DEE76E0C8010E94D291892B17
:1047500009F4C06465EE76E0C8010E94D291892B0D
:1047600009F4C0686DED76E0C8010E94D291892BF2
:1047700009F4D16069ED76E0C8010E94D291892BDD
:1047800009F4D26063ED76E0C8010E94D291892BD2
:1047900009F4D4606EEC76E0C8010E94D291892BB6
:1047A00009F4D86068EC76E0C8010E94D291892BA8
:1047B00009F4D06160EC76E0C8010E94D291892BA7
:1047C00009F4D06265EB76E0C8010E94D291892B92
:1047D00009F4D06464EA76E0C8010E94D291892B82
:1047E00009F4D068609171027091720280E090E0EB
:1047F0000E94E6918C0172CFCE01DF91CF911F9183
:104800000F910895AF92BF92CF92DF92EF92FF92F5
:104810000F931F93CF93DF93F22E032F142FE52EC8
:10482000D62EA72EB82EC92E217030E040E050E0E1
:1048300060E070E080E090E0A0E00E94208E89F0CF
:10484000E9EFF4E0FF93EF93EEE6FEE0FF93EF93E2
:104850000E94B1920F900F900F900F90E1E0F0E066
:1048600002C0E0E0F0E080911D2080FF17C02F2DF6
:10487000247030E040E050E060E070E080E090E0E4
:10488000A0E00E94208E51F0EF01219643E259E012
:104890006DEF74E0CF010E94F90FFE012F2D227001
:1048A00030E040E050E060E070E080E090E0A0E0C8
:1048B0000E94208E51F0EF01219643E259E061E021
:1048C00075E0CF010E94F90FFE012F2D287030E016
:1048D00040E050E060E070E080E090E0A0E00E9406
:1048E000208E51F0EF01219643E259E069E175E035
:1048F000CF010E94F90FFE012F2D207130E040E022
:1049000050E060E070E080E090E0A0E00E94208E47
:1049100051F0EF01219643E259E064E075E0CF01E8
:104920000E94F90FFE012F2D207230E040E050E090
:1049300060E070E080E090E0A0E00E94208E51F006
:10494000EF01219643E259E067E075E0CF010E9454
:10495000F90FFE012F2D207430E040E050E060E0C0
:1049600070E080E090E0A0E00E94208E51F0EF0126
:10497000219643E259E06DE075E0CF010E94F90F06
:10498000FE012F2D207830E040E050E060E070E044
:1049900080E090E0A0E00E94208E51F0EF0121968F
:1049A00043E259E063E175E0CF010E94F90FFE0197
:1049B00020E0302F317040E050E060E070E080E0B7
:1049C00090E0A0E00E94208E51F0EF01219643E29A
:1049D00059E066E175E0CF010E94F90FFE0120E089
:1049E000302F327040E050E060E070E080E090E016
:1049F000A0E00E94208E51F0EF01219643E259E0A1
:104A00006BE175E0CF010E94F90FFE0120E0302F2D
:104A1000347040E050E060E070E080E090E0A0E0C2
:104A20000E94208E51F0EF01219643E259E062E2AC
:104A300075E0CF010E94F90FFE0120E0302F3870A1
:104A400040E050E060E070E080E090E0A0E00E9494
:104A5000208E51F0EF01219643E259E065E275E0C6
:104A6000CF010E94F90FFE0120E0302F307140E0AD
:104A700050E060E070E080E090E0A0E00E94208ED6
:104A800051F0EF01219643E259E06AE275E0CF016F
:104A90000E94F90FFE0120E0302F307240E050E01C
:104AA00060E070E080E090E0A0E00E94208E51F095
:104AB000EF01219643E259E061E375E0CF010E94E6
:104AC000F90FFE0120E030E040E050E06D2D647011
:104AD00070E080E090E0A0E00E94208E51F0EF01B5
:104AE000219643E259E068E375E0CF010E94F90F97
:104AF000FE0180911D2081FF17C020E0302F30740F
:104B000040E050E060E070E080E090E0A0E00E94D3
:104B1000208E51F0EF01219643E259E06CE375E0FD
:104B2000CF010E94F90FFE0180911D2090911E205F
:104B300090FF17C020E030E040E05E2D507160E053
:104B400070E080E090E0A0E00E94208E51F0EF0144
:104B5000219643E259E06FE375E0CF010E94F90F1F
:104B6000FE0180911D2090911E2090FF17C020E033
:104B700030E040E05E2D507260E070E080E090E058
:104B8000A0E00E94208E51F0EF01219643E259E00F
:104B900062E475E0CF010E94F90FFE0180911D20B3
:104BA00090911E2090FF17C020E030E040E05E2D85
:104BB000507460E070E080E090E0A0E00E94208E01
:104BC00051F0EF01219643E259E068E475E0CF012E
:104BD0000E94F90FFE0120E0302F307840E050E0D5
:104BE00060E070E080E090E0A0E00E94208E51F054
:104BF000EF01219643E259E063E575E0CF010E94A1
:104C0000F90FFE0120E030E0412F417050E060E0FC
:104C100070E080E090E0A0E00E94208E51F0EF0173
:104C2000219643E259E068E575E0CF010E94F90F53
:104C3000FE0120E030E0412F427050E060E070E083
:104C400080E090E0A0E00E94208E51F0EF012196DC
:104C500043E259E06BE575E0CF010E94F90FFE01D8
:104C600020E030E0412F447050E060E070E080E0F0
:104C700090E0A0E00E94208E51F0EF01219643E2E7
:104C800059E06EE575E0CF010E94F90FFE018091B9
:104C90001D2087FF17C020E030E0412F487050E012
:104CA00060E070E080E090E0A0E00E94208E51F093
:104CB000EF01219643E259E061E675E0CF010E94E1
:104CC000F90FFE0180911D2087FF17C020E030E022
:104CD000412F407150E060E070E080E090E0A0E0A3
:104CE0000E94208E51F0EF01219643E259E065E6E3
:104CF00075E0CF010E94F90FFE0180911D2087FF12
:104D000017C020E030E0412F407250E060E070E0DA
:104D100080E090E0A0E00E94208E51F0EF0121960B
:104D200043E259E069E675E0CF010E94F90FFE0108
:104D300080911D2087FF17C020E030E0412F407494
:104D400050E060E070E080E090E0A0E00E94208E03
:104D500051F0EF01219643E259E06DE675E0CF0195
:104D60000E94F90FFE0180911D2082FF17C020E0F4
:104D700030E0412F407850E060E070E080E090E06B
:104D8000A0E00E94208E51F0EF01219643E259E00D
:104D90006DE376E0CF010E94F90FFE0180911D20A6
:104DA00082FF17C020E030E040E05E2D517060E0EF
:104DB00070E080E090E0A0E00E94208E51F0EF01D2
:104DC000219643E259E061E775E0CF010E94F90FB7
:104DD000FE0180911D2090911E2090FF17C020E0C1
:104DE00030E040E05E2D527060E070E080E090E0E6
:104DF000A0E00E94208E51F0EF01219643E259E09D
:104E000064E775E0CF010E94F90FFE0180911D203B
:104E100090911E2090FF17C020E030E040E05E2D12
:104E2000547060E070E080E090E0A0E00E94208E8E
:104E300051F0EF01219643E259E06CE775E0CF01B4
:104E40000E94F90FFE0180911D2090911E2091FF7C
:104E50001EC020E030E040E05E2D587060E070E061
:104E600080E090E0A0E00E94208E89F043E259E0CB
:104E700065E875E0CF01DF91CF911F910F91FF9011
:104E8000EF90DF90CF90BF90AF900C94F90F2F2D43
:104E9000302F412F5E2D6D2D7A2D8B2D9C2DA0E076
:104EA0000E94208E41F48FE996E09F938F930E9499
:104EB000B1920F900F90DF91CF911F910F91FF90C2
:104EC000EF90DF90CF90BF90AF9008958F929F9218
:104ED000BF92DF92EF920F931F93CF93DF93EC017A
:104EE0004B01FB0110826AE976E00E94D291892B86
:104EF00061F580911D207DE4D72EE0E8EE2E82FD45
:104F000002C004E001C004E810E0B12C81FF02C03F
:104F100060ECE62E26E04AE250E06BE270E089E2C7
:104F200090E00E94B25C81E090E00E94300B882308
:104F300011F05DE5D52E80911D2090911E2090FDF1
:104F400016E091FF07C0186005C0D12CE12C00E0ED
:104F500010E0B12C68E976E0CE010E94D291892B55
:104F600061F481E0F40180836091710270917202BA
:104F700080E090E00E94E691EC0166E976E0CE01E7
:104F80000E94D291892B61F48FEFF40180836091AC
:104F900071027091720280E090E00E94E691EC0153
:104FA000209709F424C162E976E0CE010E94D291F3
:104FB000892B19F4FD2DF160DF2E6EE876E0CE012D
:104FC0000E94D291892B19F48D2D8460D82E6BE824
:104FD00076E0CE010E94D291892B19F4ED2DE2608A
:104FE000DE2E69E876E0CE010E94D291892B19F479
:104FF000FD2DF860DF2E66E876E0CE010E94D291AA
:10500000892B19F48D2D8061D82E60E876E0CE01D1
:105010000E94D291892B19F4ED2DE062DE2E6AE711
:1050200076E0CE010E94D291892B19F4FD2DF06417
:10503000DF2E67E776E0CE010E94D291892B19F42A
:105040008D2D8068D82E62E776E0CE010E94D29145
:10505000892B19F4EE2DE160EE2E6BE676E0CE01A1
:105060000E94D291892B19F4FE2DF260EF2E68E692
:1050700076E0CE010E94D291892B19F48E2D8460A6
:10508000E82E63E676E0CE010E94D291892B19F4D6
:10509000EE2DE860EE2E6CE576E0CE010E94D29116
:1050A000892B19F4FE2DF061EF2E65E576E0CE0137
:1050B0000E94D291892B19F48E2D8062E82E61E531
:1050C00076E0CE010E94D291892B19F4EB2DE46099
:1050D000BE2E6EE476E0CE010E94D291892B19F4A7
:1050E000FE2DF064EF2E69E476E0CE010E94D291AD
:1050F000892B19F48E2D8068E82E66E476E0CE01C7
:105100000E94D291892B09F4016063E476E0CE011C
:105110000E94D291892B09F4026060E476E0CE010E
:105120000E94D291892B09F404606CE376E0CE01F1
:105130000E94D291892B09F4086068E376E0CE01E1
:105140000E94D291892B09F4006164E376E0CE01DC
:105150000E94D291892B09F4006260E376E0CE01CF
:105160000E94D291892B09F400646EE276E0CE01B0
:105170000E94D291892B09F400686BE276E0CE019F
:105180000E94D291892B09F4116063E276E0CE018E
:105190000E94D291892B09F412606AE176E0CE0177
:1051A0000E94D291892B09F4146061E176E0CE016E
:1051B0000E94D291892B09F418606EE076E0CE014E
:1051C0000E94D291892B09F4106168E076E0CE014B
:1051D0000E94D291892B09F410626DEF75E0CE0127
:1051E0000E94D291892B09F0D2CE1064D0CE2D2D01
:1051F0003E2DA8016B2D70E080E090E0DF91CF9113
:105200001F910F91EF90DF90BF909F908F90089526
:105210005F926F927F928F929F92AF92BF92CF9246
:10522000DF92EF92FF920F931F93CF93DF93782E2D
:10523000C7E2DBE100E010E0F7EFEF2EF5E0FF2E34
:105240008170582E872D8270682EA2EECA2EA5E09E
:10525000DA2EBAEEAB2EB5E0BB2E88EE882E85E0B6
:10526000982E772051F01F930F93FF92EF920E9498
:10527000B1920F900F900F900F905520A1F089855B
:105280008F9388858F93BF92AF920E94B1920F90B7
:105290000F900F900F906620C1F09F928F920E9406
:1052A000B1920F900F90662081F0DF92CF920E9412
:1052B000B192288139814A815B816C817D818E81A7
:1052C0009F810E9402240F900F900E94A20B0F5FFB
:1052D0001F4F2A960430110521F6DF91CF911F91BF
:1052E0000F91FF90EF90DF90CF90BF90AF909F9085
:1052F0008F907F906F905F90089582ED95E09F93DF
:105300008F930E94B1920E946B208EE09BE19F934D
:105310008F938AEC95E09F938F930E94B192609156
:10532000520270915302809154029091550228EEDE
:1053300033E040E050E00E94198C5F934F933F931D
:105340002F938AEB95E09F938F930E94B19281EB0C
:1053500095E09F938F930E94B1920E9421108091BB
:105360001D202DB73EB7225F3F4F0FB6F8943EBFCA
:105370000FBE2DBF80FF05C041E061E081E00E94CB
:10538000CB118DEA95E09F938F930E94B19280E0BC
:105390000E9449220E946F20809157021F928F9392
:1053A00084EA95E09F938F930E94B1928091C10906
:1053B0001F928F938BE995E09F938F930E94B192F8
:1053C000809183028F93809182028F9380918102DA
:1053D0008F93809180028F938DE895E09F938F93B8
:1053E0000E94B1921F9280E48F9385E795E09F938E
:1053F0008F930E94B1928091B3281F928F938091D6
:10540000B2281F928F9382E695E09F938F930E941C
:10541000B192809156021F928F9389E595E09F93F8
:105420008F930E94B1928091580290915902A0915D
:105430005A02B0915B022DB73EB7225E3F4F0FB6C6
:10544000F8943EBF0FBE2DBF96FF03C08EE895E0D7
:1054500002C081E995E09F938F938FE495E09F933D
:105460008F930E94B19283E00E9408290F900F90C1
:105470000F900F901D9B03C08EE895E002C081E95C
:1054800095E09F938F9383E495E09F938F930E9481
:10549000B19289E395E09F938F930E94B19280919E
:1054A00058020F900F900F900F900F900F9081FF68
:1054B00009C083E395E09F938F930E94B1920F9070
:1054C0000F9013C080FF03C08EE895E002C081E911
:1054D00095E09F938F938FE295E09F938F930E9427
:1054E000B1920F900F900F900F9080915802909171
:1054F0005902A0915A02B0915B0297FF03C08EE857
:1055000095E002C081E995E09F938F9386E295E054
:105510009F938F930E94B1928FE195E09F938F9319
:105520000E94B1926091C5097091C60980E090E037
:105530000E9479220E94A20B0F900F900F900F9063
:105540000F900F90779903C08EE895E002C081E933
:1055500095E09F938F9386E195E09F938F930E94B0
:10556000B1920E9445090E94EC0A9F938F937F930A
:105570006F9388E095E09F938F930E94B1920E9471
:10558000A60A9F938F937F936F938AEF94E09F93E4
:105590008F930E94B19281E090E00E94252180913A
:1055A000882890918928A0918A28B0918B28BF9350
:1055B000AF939F938F938CEE94E09F938F930E9471
:1055C000B19280919D288F9380919C288F93809198
:1055D0009B288F9380919A288F9388ED94E09F93D6
:1055E0008F930E94B19280918C2890918D28A091E8
:1055F0008E28B0918F28BF93AF939F938F938AEC9F
:1056000094E09F938F930E94B1928DB79EB782963C
:105610000FB6F8949EBF0FBE8DBF8091A1288F93C7
:105620008091A0288F9380919F288F9380919E28AE
:105630008F9386EB94E09F938F930E94B19261E0E9
:1056400070E080E090E00E94AB0B0F900F900F9005
:105650000F900F900F9061E070E081E090E00C946B
:10566000AB0BF894E0E0F0E081E280935700849186
:10567000E2E0F0E041E2409357004491E4E0F0E0E2
:1056800091E290935700E49190E0A0E0B0E0DC015B
:105690009927882750E060E070E0762F652F542F1F
:1056A0004427840F951FA61FB71F8E0F911DA11DA4
:1056B000B11D8093C81B9093C91BA093CA1BB093C4
:1056C000CB1B78940895CF93DF93CDB7DEB7619766
:1056D0000FB6F894DEBF0FBECDBF48E250E06EE1DA
:1056E00070E087E29BE10E9405942091271B309196
:1056F000281B4091291B50912A1B60912B1B7091F4
:105700002C1B80912D1B90912E1BAFEF0E94208EA1
:1057100009F05DC08DE48093271B80E88093281BEF
:1057200084E08093291B10922A1B10922B1B10924D
:105730002C1B10922D1B10922E1B8CE390E090934B
:10574000301B80932F1B1092311B1092321B109232
:10575000331B1092341B1092351B1092361B109283
:10576000371B1092381B10923A1B1092391B109263
:105770003B1B10923C1B10923D1B10923E1B109243
:105780003F1B1092401B1092411B1092421B109223
:10579000441B1092431B1092451B1092461B109203
:1057A000471B1092481B1092491B10924A1B1092E3
:1057B0004B1B10924C1B10924E1B10924D1B48E23B
:1057C00050E06EE170E087E29BE10E94239444E0A8
:1057D00050E06AE170E0CE010B960E9405948B8543
:1057E0009C85AD85BE858F3F2FEF9207A207B2073C
:1057F000A9F48AE090E4A0E0B0E08093580290938E
:105800005902A0935A02B0935B0244E050E06AE16F
:1058100070E088E592E00E94239408C080935802CB
:1058200090935902A0935A02B0935B0242E050E079
:1058300066E570E0CE010F960E9405948F859889E9
:105840008F3F2FEF920769F41092C6091092C50995
:1058500042E050E066E570E085EC99E00E94239418
:1058600004C09093C6098093C50949E050E06AE0FE
:1058700070E082EA98E20E9405940E94E30C44E002
:1058800050E06AE470E0CE010B960E9405948B858F
:105890009C85AD85BE8544E050E06AE470E08F3FB2
:1058A0009F4FAF4FBF4F29F488E792E00E942394A7
:1058B00004C088E792E00E94059444E050E066E46A
:1058C00070E0CE010B960E9405948B859C85AD857A
:1058D000BE8544E050E066E470E08F3F9F4FAF4FDD
:1058E000BF4F29F484E792E00E94239404C084E728
:1058F00092E00E94059444E050E06EE470E0CE0136
:105900000B960E9405948B859C85AD85BE8544E0F1
:1059100050E06EE470E08F3F9F4FAF4FBF4F29F4D0
:105920008CE792E00E94239404C08CE792E00E94EE
:10593000059441E050E069E170E0CE0141960E949B
:105940000594898941E050E069E170E08F3F29F4D6
:1059500081EC99E00E94239404C081EC99E00E94BC
:10596000059441E050E068E170E0CE0141960E946C
:105970000594898941E050E068E170E08F3F29F4A7
:1059800087E592E00E94239404C087E592E00E949C
:10599000059441E050E067E170E0CE0141960E943D
:1059A0000594898941E050E067E170E08F3F29F478
:1059B00086E592E00E94239404C086E592E00E946E
:1059C00005944AE050E060E070E0CE0101960E944C
:1059D000059489814AE050E060E070E08F3F29F44F
:1059E0008EE09BE10E94239404C08EE09BE10E9424
:1059F000059444E050E062E570E0CE010B960E9411
:105A000005948B859C85AD85BE8544E050E062E5BC
:105A100070E08F3F9F4FAF4FBF4F29F480E892E077
:105A20000E94239404C080E892E00E94059444E020
:105A300050E063E170E0CE010B960E9405948B85E7
:105A40009C85AD85BE8544E050E063E170E08F3F0A
:105A50009F4FAF4FBF4F29F482E592E00E942394FD
:105A600004C082E592E00E94059461960FB6F89416
:105A7000DEBF0FBECDBFDF91CF910895CF92DF92F1
:105A8000EF92FF92609171027091720280E090E05B
:105A90000E94E69165E975E00E94FA91892B09F070
:105AA0001FC18DE48093271B80E88093281B84E02E
:105AB0008093291B10922A1B10922B1B10922C1BD7
:105AC00010922D1B10922E1B8CE390E09093301BB4
:105AD00080932F1B1092311B1092321B1092331B9C
:105AE0001092341B1092351B1092361B1092371BEC
:105AF0001092381B10923A1B1092391B10923B1BCC
:105B000010923C1B10923D1B10923E1B10923F1BAB
:105B10001092401B1092411B1092421B1092441B8A
:105B20001092431B1092451B1092461B1092471B6C
:105B30001092481B1092491B10924A1B10924B1B4B
:105B400010924C1B10924E1B10924D1B48E250E0DD
:105B50006EE170E087E29BE10E9423948AE090E48A
:105B6000A0E0B0E08093580290935902A0935A02AB
:105B7000B0935B0244E050E06AE170E088E592E0B7
:105B80000E9423941092C6091092C50942E050E089
:105B900066E570E085EC99E00E94239442E2C42E11
:105BA000DD24DA944CECE42E4BE3F42EC092780220
:105BB000D0927902E0927A02F0927B0244E050E0C7
:105BC0006AE470E088E792E00E942394C092740235
:105BD000D0927502E0927602F092770244E050E0B3
:105BE00066E470E084E792E00E94239487ED94E3FA
:105BF000AFEEBCE380937C0290937D02A0937E0283
:105C0000B0937F0244E050E06EE470E08CE792E0F5
:105C10000E9423948AE999E9A9E1B0E48093800283
:105C200090938102A0938202B093830244E050E0FB
:105C300062E570E080E892E00E9423941092C1092E
:105C400080E00E942D6A41E050E069E170E081EC63
:105C500099E00E9423948AE1809357020E94D468BD
:105C600041E050E068E170E087E592E00E94239413
:105C70008FE08093560241E050E067E170E086E5F6
:105C800092E00E9423948AE0EEE0FBE1DF011D92A6
:105C90008A95E9F74AE050E060E070E0CF010E94A9
:105CA000239480EA96E8A1E0B0E0809352029093BA
:105CB0005302A0935402B093550244E050E063E1D4
:105CC00070E082E592E00E94239481E00E944922E4
:105CD00080E090E0FF90EF90DF90CF900C94F70C75
:105CE000FF90EF90DF90CF9008952F923F924F92C8
:105CF0005F926F927F928F929F92AF92BF92CF925C
:105D0000DF92EF92FF920F931F93CF93DF93CDB764
:105D1000DEB72B970FB6F894DEBF0FBECDBF9B87C3
:105D20008A874A01FC0180819181892B11F00C94B2
:105D300011416091710270917202CA010E94E69154
:105D400060E470E0C4010E941992009759F46091D8
:105D50006D3170916E318AE090E00E946D9281E029
:105D60000C9416418130910561F4F401B0801B2D33
:105D7000110F110B012F412E512E612E712EA12ECC
:105D8000BCC082309105B9F4F4018081992787FD68
:105D90009095982F88272181820F911D27FD9A9534
:105DA000B82E192F092F000F000B402E502E602EF9
:105DB000702EA02EA2C083309105B1F5F401208190
:105DC000922F990F990B392F492F592F692F792F1E
:105DD000892F00E10E94C28D19012A013B01B82FD1
:105DE000A92F2181922F990F990B392F492F592FC4
:105DF000692F792F892F08E00E94C28D59016A010D
:105E00007B018C019101A201B3018B2F9A2F0E947B
:105E1000F98DA2801A2D110F110BB12EC12ED12E8A
:105E2000E12EF12E012F55C004970CF45DC0F40152
:105E30002081922F990F990B392F492F592F692FB4
:105E4000792F892F08E10E94C28D19012A013B0197
:105E5000B82FA92F2181922F990F990B392F492FF4
:105E6000592F692F792F892F00E10E94C28D590186
:105E70006A017B018C019101A201B3018B2F9A2F42
:105E80000E94F98DA3801A2D110F110BB12EC12E76
:105E9000D12EE12EF12E012F0E94F98D19012A0138
:105EA0003B01B82FA92F2281922F990F990B392FDF
:105EB000492F592F692F792F892F08E00E94C28D11
:105EC00059016A017B018C019101A201B3018B2F61
:105ED0009A2F0E94F98DB22E132F042F452E562E85
:105EE000672E782EA92E09C07AE0B72E10E000E0C8
:105EF000412C512C612C712CA12C0E94A20B2B2D1A
:105F0000312F402F542D652D762D872D9A2D273634
:105F1000FFE63F07FCE64F07510561057105810566
:105F2000910511F40C941E3B2736EFE63E07ECE694
:105F30004E075105610571058105910511F008F0C5
:105F400096C12936F2E73F07410551056105710504
:105F50008105910511F40C943B3E2936E2E73E079A
:105F600041055105610571058105910511F008F0A4
:105F7000A6C02536F4E63F074105510561057105C8
:105F80008105910509F457C62536E4E63E0741052B
:105F90005105610571058105910509F0B8F5A6E780
:105FA0000E94208E11F40C9492380E94208E09F0E9
:105FB00068F4A8E60E94208E09F483C6A5E70E9433
:105FC000208E11F40C947C380C940F412B2D312F22
:105FD000402F542D652D762D872D9A2D2A33F6E2EC
:105FE0003F0741055105610571058105910509F4DA
:105FF0001FC32436314641055105610571058105F0
:10600000910511F40C94B43E0C940F412B2D312FBB
:10601000402F542D652D762D872D9A2D2737FFE69D
:106020003F0741055105610571058105910511F491
:106030000C945F3C2737EFE63E07410551056105AB
:1060400071058105910509F0C8F42436F9E63F078A
:1060500041055105610571058105910511F40C9407
:10606000553825363E4641055105610571058105C6
:10607000910511F40C94933C0C940F412B2D312F6E
:10608000402F542D652D762D872D9A2D2333F1E742
:106090003F0741055105610571058105910511F421
:1060A0000C94B43E25363247410551056105710512
:1060B0008105910511F40C945D3D0C940F412B2D3D
:1060C000312F402F542D652D762D872D9A2D283771
:1060D000F4E63F07F1E64F075105610571058105BB
:1060E000910509F4B5C22837E4E63E07E1E64E071C
:1060F0005105610571058105910511F008F050C049
:106100002837F4E73F074105510561057105810511
:10611000910509F48DC22837E4E73E074105510592
:10612000610571058105910509F0C8F42337F2E78F
:106130003F0741055105610571058105910511F480
:106140000C948C3E23373347410551056105710599
:106150008105910511F40C94A03E0C940F412B2D58
:10616000312F402F542D652D762D872D9A2D2133DB
:10617000F4E63F07F1E64F0751056105710581051A
:10618000910509F469C2233634464146510561053B
:1061900071058105910511F40C94B43E0C940F41E6
:1061A0002B2D312F402F542D652D762D872D9A2D97
:1061B0002336FDE63F07F8E64F07510561057105F7
:1061C0008105910509F440C32336EDE63E07E8E674
:1061D0004E075105610571058105910509F0C8F467
:1061E0002236F5E63F07F4E64F07510561057105D4
:1061F0008105910509F41FC52237324745465105EF
:10620000610571058105910511F40C94B83B0C945E
:106210000F412B2D312F402F542D652D762D872D9D
:106220009A2D2336F2E33F07F9E64F075105610542
:1062300071058105910509F42FC22436E3E63E0776
:10624000ECE64E075105610571058105910511F4D4
:106250000C941B3B2D3635474846510561057105A9
:106260008105910511F00C940F410C94CA3E2B2D21
:10627000312F402F542D652D762D872D9A2D2136C7
:10628000EDE63E07E5E74E07E8E65E0761057105C6
:106290008105910511F40C947D3C2136FDE63F0704
:1062A000F5E74F07F8E65F07610571058105910580
:1062B00011F008F0DAC02437E8E73E07E4E74E07BC
:1062C0005105610571058105910509F497C72437CA
:1062D000F8E73F07F4E74F075105610571058105B0
:1062E000910511F008F055C02133E1E33E07E1E7E5
:1062F0004E075105610571058105910511F40C9456
:10630000F93B2133F1E33F07F1E74F075105610501
:1063100071058105910509F0D0F42537E3E63E07C4
:10632000EDE64E075105610571058105910511F4F2
:106330000C94F93B20333143414751056105710508
:106340008105910511F40C94B83B0C940F412B2D51
:10635000312F402F542D652D762D872D9A2D2037E6
:10636000E5E63E07E2E74E07510561057105810547
:10637000910511F40C945D3D2C363447444751058A
:10638000610571058105910511F40C9438400C9458
:106390000F412B2D312F402F542D652D762D872D1C
:1063A0009A2D2936ECE63E07E1E64E07E3E65E0766
:1063B000610571058105910509F47BC22936FCE66A
:1063C0003F07F1E64F07F3E65F07610571058105B9
:1063D000910509F0E0F42437E4E63E07E7E74E07CD
:1063E0005105610571058105910511F40C948640F4
:1063F00024373F464F465246610571058105910598
:1064000011F00C940F410C9400000C9411412B2DB1
:10641000312F402F542D652D762D872D9A2D263323
:10642000E9E63E07E5E74E07E5E65E07610571052B
:106430008105910509F449C42037FCE63F07F5E6DC
:106440004F07F8E65F07610571058105910509F4BD
:1064500038C42E36314648465346610571058105DC
:10646000910509F49FC60C940F412B2D312F402F1D
:10647000542D652D762D872D9A2D2437F3E73F0770
:10648000F5E64F07F2E75F076105710581059105A4
:1064900011F40C940D3D2437E3E73E07E5E64E0783
:1064A000E2E75E07610571058105910511F008F0CD
:1064B00055C02337F2E73F07F7E74F07F0E75F07DD
:1064C000610571058105910511F40C94103D233788
:1064D000E2E73E07E7E74E07E0E75E076105710583
:1064E0008105910509F0C8F42237F7E73F07F0E787
:1064F0004F075F07610571058105910509F4A8C182
:10650000233735464247504761057105810591059E
:1065100011F40C947A3F0C940F412B2D312F402F06
:10652000542D652D762D872D9A2D2436FDE63F07B7
:10653000F3E64F07F2E75F076105710581059105F5
:1065400009F4CEC421363C464546524761057105E3
:106550008105910509F4D6C30C940F412B2D312FE1
:10656000402F542D652D762D872D9A2D2437F2E757
:106570003F07F1E64F07F5E75F0761057105810504
:10658000910509F408C52437E2E73E07E1E64E0726
:10659000E5E75E07610571058105910509F0C8F41D
:1065A0002437F3E73F07F5E64F07F4E75F07610598
:1065B00071058105910509F44CC6273730474847D6
:1065C0005447610571058105910509F4C1C50C9415
:1065D0000F412B2D312F402F542D652D762D872DDA
:1065E0009A2D2F36FCE63F07FFE54F07F6E75F07DA
:1065F000610571058105910509F41DC42C36E1E69C
:106600003E07E4E74E07E8E75E076105710581058F
:10661000910511F40C940240223737464047554704
:10662000610571058105910511F00C940F41E0C7DA
:1066300083E080939028109292281092912840E94C
:1066400058E262E184E392E00E9437540C941141D5
:106650000E94AF150C94114121E042E161E080ED10
:106660000E94716121E042E161E080ED0E94716170
:1066700021E042E161E080ED0E94716121E042E1B0
:1066800061E080ED0E94716121E042E161E080ED16
:106690000E9471610C9411416091710270917202BB
:1066A00080E090E00E94E6916CE975E00E94FA912A
:1066B000892B09F0C5C0609171027091720280E06F
:1066C00090E00E94E6915C01009709F497C060EEAB
:1066D00073E00E94FA91892BE1F488EE93E0A0E048
:1066E000B0E08093520290935302A0935402B0936F
:1066F000550268EE73E080E090E00E94985F44E00D
:1067000050E063E170E082E592E00E9423940C94F3
:10671000114162EA75E0C5010E94FA91892BE1F40A
:1067200080E197E2A0E0B0E08093520290935302A0
:10673000A0935402B093550260E177E280E090E0CC
:106740000E94985F44E050E063E170E082E592E0EF
:106750000E9423940C94114165EA75E0C5010E94E2
:10676000FA91892BE1F480EA96E8A1E0B0E0809309
:10677000520290935302A0935402B093550260EAE0
:1067800076E881E090E00E94985F44E050E063E1A9
:1067900070E082E592E00E9423940C94114169EA32
:1067A00075E0C5010E94FA91892BE1F480E89AE135
:1067B000A6E0B0E08093520290935302A09354025B
:1067C000B093550260E87AE186E090E00E94985F1D
:1067D00044E050E063E170E082E592E00E9423949F
:1067E0000C94114187EF92E09F938F930E94B19296
:1067F0000E94A20B0F900F900C94114160915202D5
:1068000070915302809154029091550228EE33E02A
:1068100040E050E00E94198C5F934F933F932F9379
:1068200083EF92E09F938F930E94B1920E94A20BFC
:106830000F900F900F900F900F900F900C941141AC
:106840000E9421100C9411410E9427160C941141B2
:10685000609171027091720280E090E00E94E69176
:106860008C016EE875E00E94FA91892B19F47798F3
:106870000C94114161E975E0C8010E94FA91892BDD
:1068800019F4779A0C941141779903C08EE895E03A
:1068900002C081E995E09F938F9380EA94E09F93F3
:1068A0008F930E94B1920F900F900F900F900C94C5
:1068B0001141609171027091720280E090E00E943B
:1068C000E6918C0168E575E00E94FA91892B09F048
:1068D00077C0609171027091720280E090E00E9436
:1068E000E6918C01009711F40C9411416DEA75E06A
:1068F0000E94FA91892BB1F482E29FEFACECBBE3EA
:106900008093780290937902A0937A02B0937B02ED
:1069100044E050E06AE470E088E792E00E9423944B
:106920000C94114163EB75E0C8010E94FA91892B28
:10693000B1F482E29FEFACECBAE3809378029093DB
:106940007902A0937A02B0937B0244E050E06AE4BB
:1069500070E088E792E00E9423940C941141C801F2
:106960000E94D0902B013C0120E030E0A9010E9460
:106970006B888823D9F081E00E94430A9B01AC0117
:10698000C301B2010E946F8860937802709379020C
:1069900080937A0290937B0244E050E06AE470E0D6
:1069A00088E792E00E9423940C94114186EE92E0D5
:1069B0009F938F930E94B1920F900F900C9411416E
:1069C0006BE575E0C8010E94FA91892B09F077C048
:1069D000609171027091720280E090E00E94E691F5
:1069E0008C01009711F40C9411416DEA75E00E943E
:1069F000FA91892BB1F482E29FEFACECBBE3809378
:106A0000740290937502A0937602B093770244E0EB
:106A100050E066E470E084E792E00E9423940C94D6
:106A2000114163EB75E0C8010E94FA91892BB1F422
:106A300082E29FEFACECBAE380937402909375020C
:106A4000A0937602B093770244E050E066E470E0F1
:106A500084E792E00E9423940C941141C8010E94A3
:106A6000D0902B013C0120E030E0A9010E946B880E
:106A70008823D9F082E00E94430A9B01AC01C30144
:106A8000B2010E946F8860937402709375028093C4
:106A900076029093770244E050E066E470E084E789
:106AA00092E00E9423940C94114189ED92E09F930F
:106AB0008F930E94B1920F900F900C94114163E557
:106AC00075E0C8010E94FA91892B09F073C06091AA
:106AD00071027091720280E090E00E94E6918C0158
:106AE000009711F40C9411416DEA75E00E94FA913F
:106AF000892BB1F487ED94E3AFEEBCE380937C0285
:106B000090937D02A0937E02B0937F0244E050E018
:106B10006EE470E08CE792E00E9423940C941141A3
:106B200063EB75E0C8010E94FA91892B51F48AEC5D
:106B300092E09F938F930E94B1920F900F900C94CC
:106B40001141C8010E94D0902B013C0120E030E0AF
:106B5000A9010E946B88882319F180E00E94430AF2
:106B60004B015C0121EE3AE744E95EE3C301B20167
:106B70000E94A487A50194010E946F8860937C0203
:106B800070937D0280937E0290937F0244E050E0F8
:106B90006EE470E08CE792E00E9423940C94114123
:106BA0008DEB92E09F938F930E94B1920F900F9084
:106BB0000C9411410E94920A9F938F937F936F933D
:106BC00086EB92E09F938F930E94B19282E00E94A5
:106BD000430A2091740230917502409176025091DF
:106BE00077020E94F08A162F072FF82EE92E81E0F7
:106BF0000E94430AEF92FF920F931F932091780215
:106C00003091790240917A0250917B020E94F08A81
:106C10009F938F937F936F938AEA92E09F938F93D2
:106C20000E94B1920E94A20B0FB6F894DEBF0FBE75
:106C3000CDBF0C941141609171027091720280E09D
:106C400090E00E94E6910097C1F00E946723209196
:106C5000C5093091C6098217930709F19093C609B7
:106C60008093C50942E050E066E570E085EC99E06C
:106C70000E94239489E994E002C082E994E09F9302
:106C80008F930E94B1926091C5097091C60980E00E
:106C900090E00E9479220E94A20B0F900F9087E84B
:106CA00094E09F938F930E94B1926FEF7FEF80E00B
:106CB00090E00E9479220E94A20B0F900F900C94FA
:106CC00011410E947A1F0C941141F4018481843394
:106CD00029F440E061E080E00E94CB1180917302D2
:106CE000882311F40C9411411F928F9384E894E04F
:106CF0009F938F930E94B1920F900F900F900F90DF
:106D00000C941141F4018481893709F080C06091AD
:106D100071027091720280E090E00E94E6918C0115
:106D20006EE875E00E94FA91892B51F48091580227
:106D300090915902A0915A02B0915B02906410C0E8
:106D400061E975E0C8010E94FA91892BD1F4809124
:106D5000580290915902A0915A02B0915B029F7B18
:106D60008093580290935902A0935A02B0935B0209
:106D700044E050E06AE170E088E592E00E942394EC
:106D800046C068EB75E0C8010E94FA91892B21F595
:106D90008091261B8F938091251B8F938091241BBC
:106DA0008F938091231B8F938091221B8F938091CF
:106DB000211B8F938091201B8F9380911F1B8F939A
:106DC0008FE792E09F938F930E94B1920FB6F89451
:106DD000DEBF0FBECDBF1BC08091580290915902FB
:106DE000A0915A02B0915B0296FF03C08EE895E035
:106DF00002C081E995E09F938F938BE792E09F9388
:106E00008F930E94B1920F900F900F900F908091EE
:106E10007302882311F40C9411411F928F9381E81F
:106E200094E09F938F930E94B1920F900F900F90D8
:106E30000F900C941141F40184818737E9F560913A
:106E400071027091720280E090E00E94E6910097DA
:106E5000D9F00E94D0902B013C0120E030E0A90144
:106E60000E946B88882381F04092800250928102B8
:106E7000609282027092830244E050E062E570E02A
:106E800080E892E00E942394809183028F93809106
:106E900082028F93809181028F93809180028F93E1
:106EA0008DE692E09F938F930E94B1920F900F9086
:106EB0000F900F900F900F9080917302882311F420
:106EC0000C9411411F928F938EE794E09F938F93C0
:106ED0000E94B1920F900F900F900F900C9411415F
:106EE000609171027091720280E090E00E94E691E0
:106EF0008C016EE875E00E94FA9140905802509023
:106F0000590260905A0270905B02892B19F46894C0
:106F100057F809C061E975E0C8010E94FA91892B10
:106F200099F4E89457F840925802509259026092AE
:106F30005A0270925B0244E050E06AE170E088E53A
:106F400092E00E94239413C057FE03C08EE895E0A0
:106F500002C081E995E09F938F9389E692E09F9329
:106F60008F930E94B1920F900F900F900F9080918D
:106F70007302882311F40C9411411F928F938BE7B5
:106F800094E09F938F930E94B1920F900F900F9077
:106F90000F900C941141609171027091720280E027
:106FA00090E00E94E6915C016EEB75E00E94FA9120
:106FB000892B11F489E108C062EC75E0C5010E94DB
:106FC000FA91892B49F480E18093C4001092C500A6
:106FD00082E08093C00055C066EC75E0C5010E9458
:106FE000FA91892B11F488E0EFCF6BEC75E0C501C5
:106FF0000E94FA91892B39F060ED75E0C5010E947D
:10700000FA91892B11F483E0DFCF8091C40089319C
:1070100041F484E692E09F938F930E94B1920F9087
:107020000F908091C400803141F48FE592E09F93EE
:107030008F930E94B1920F900F908091C40088307E
:1070400041F489E592E09F938F930E94B1920F9053
:107050000F908091C400833041F483E592E09F93C8
:107060008F930E94B1920F900F908091C40088304E
:1070700041F48DE492E09F938F930E94B1920F9020
:107080000F9080917302882311F40C9411411F9288
:107090008F9388E794E09F938F930E94B1920F9013
:1070A0000F900F900F900C941141609171027091AC
:1070B000720280E090E00E94E6916DEA75E00E9425
:1070C000FA91892B11F481E001C080E00E944922ED
:1070D00080917302882311F40C9411411F928F93B5
:1070E00085E794E09F938F930E94B1920F900F9049
:1070F0000F900F900C9411410E946F2080917302A9
:10710000882311F40C9411411F928F9382E794E02D
:107110009F938F930E94B1920F900F900F900F90BA
:107120000C9411410E946B2080917302882311F40A
:107130000C9411411F928F938FE694E09F938F934D
:107140000E94B1920F900F900F900F900C941141EC
:10715000609171027091720280E090E00E94E6916D
:107160000E94D490803170F48093C1090E942D6AEE
:1071700041E050E069E170E081EC99E00E942394E5
:107180000C9411418091C1091F928F9383E492E086
:107190009F938F930E94B1920F900F900F900F903A
:1071A0000C941141609171027091720280E090E044
:1071B0000E94E6910E94D49095EF980F903170F460
:1071C000809357020E94D46841E050E068E170E08B
:1071D00087E592E00E9423940C941141809157021C
:1071E0001F928F938AE392E09F938F930E94B192B4
:1071F0000F900F900F900F900C94114160917102BD
:107200007091720280E090E00E94E691009789F010
:107210004AE050E0BC018EE09BE10E940A924AE005
:1072200050E060E070E08EE09BE10E9423940C94BB
:1072300011418EE09BE19F938F9385ED95E09F93A5
:107240008F930E949F920F900F900F900F900C942D
:107250001141609171027091720280E090E00E9491
:10726000E6915C0160EE73E00E94FA91892BD9F4FB
:10727000219A8091580290915902A0915A02B0919E
:107280005B0280618093580290935902A0935A0246
:10729000B0935B0244E050E06AE170E088E592E080
:1072A0000E942394BEC76CE575E0C5010E94FA9167
:1072B000892BD9F4229A8091580290915902A09179
:1072C0005A02B0915B0280628093580290935902F7
:1072D000A0935A02B0935B0244E050E06AE170E090
:1072E00088E592E00E9423949CC762EC73E0C5019C
:1072F0000E94FA91892BD9F4239A80915802909197
:107300005902A0915A02B0915B02806480935802A6
:1073100090935902A0935A02B0935B0244E050E06C
:107320006AE170E088E592E00E9423947AC76FEFEB
:1073300074E0C5010E94FA91892BD9F4239A8091B7
:10734000580290915902A0915A02B0915B02806854
:107350008093580290935902A0935A02B0935B0213
:1073600044E050E06AE170E088E592E00E942394F6
:1073700058C76CE679E0C5010E94FA91892B71F536
:1073800081E08093342487E29BE1909336248093BC
:10739000352410923824109237248091580290910D
:1073A0005902A0915A02B0915B02916080935802F9
:1073B00090935902A0935A02B0935B0244E050E0CC
:1073C0006AE170E088E592E00E94239444E354E28D
:1073D00062E184E392E00E94375423C769EE73E0D0
:1073E000C5010E94FA91892B11F5E7E5FBE11192A5
:1073F00011922BE1E737F207D1F780915802909173
:107400005902A0915A02B0915B0292608093580297
:1074100090935902A0935A02B0935B0244E050E06B
:107420006AE170E088E592E00E942394FAC661E97F
:1074300075E0C5010E94FA9140915802509159029D
:1074400060915A0270915B02892BC1F44F705C7F8E
:10745000409358025093590260935A0270935B0212
:107460002B9A44E050E06AE170E088E592E00E94E7
:107470002394809199280E94E968D3C644FF03C0F1
:107480008EE895E002C081E995E09F938F938FE2AB
:1074900092E09F938F930E94B192809158020F9037
:1074A0000F900F900F9085FF03C08EE895E002C00B
:1074B00081E995E09F938F9384E292E09F938F936D
:1074C0000E94B192809158020F900F900F900F90F0
:1074D00086FF03C08EE895E002C081E995E09F93A6
:1074E0008F9389E192E09F938F930E94B192809154
:1074F00058020F900F900F900F9087FF03C08EE8F7
:1075000095E002C081E995E09F938F938EE092E031
:107510009F938F930E94B19280915802909159024B
:10752000A0915A02B0915B020F900F900F900F90B4
:1075300090FF03C08EE895E002C081E995E09F933B
:107540008F9383E092E09F938F930E94B1928091FA
:10755000580290915902A0915A02B0915B020F908B
:107560000F900F900F9091FF03C08EE895E002C03E
:1075700081E995E09F938F9388EF91E09F938F939C
:107580000E94B1928091580290915902A0915A02A2
:10759000B0915B020F900F900F900F9091FF41C63A
:1075A0008DED95E00E94D59257E5A52E5BE1B52EB5
:1075B0000BE010E065EE862E65E0962EF5018081E9
:1075C0009181F2E0AF0EB11C9F938F931F930F93A5
:1075D0009F928F920E949F920F5F1F4F0F900F906C
:1075E0000F900F900F900F900B31110539F719C6BE
:1075F0008BE694E09F938F930E94B19280917302E7
:107600000F900F90882361F01F928F9388E694E08B
:107610009F938F930E94B1920F900F900F900F90B5
:1076200088E10FB6F89480936000109260000FBE5E
:107630000C94007CF6C50E942261F3C56091710232
:107640007091720280E090E00E94E6918C016EE8F9
:1076500075E00E94FA91892BE9F40E94D36780912A
:10766000580290915902A0915A02B0915B028D7F0D
:1076700081608093580290935902A0935A02B0936C
:107680005B0244E050E06AE170E088E592E00E942D
:107690002394C7C561E975E0C8010E94FA91892B5E
:1076A000E1F40E948B678091580290915902A09159
:1076B0005A02B0915B028C7F8093580290935902DA
:1076C000A0935A02B0935B0244E050E06AE170E09C
:1076D00088E592E00E942394A4C560EF75E0C8019C
:1076E0000E94FA91892BE9F40E948B6780915802DD
:1076F00090915902A0915A02B0915B028E7F8260F4
:107700008093580290935902A0935A02B0935B025F
:1077100044E050E06AE170E088E592E00E94239442
:1077200080C58091580281FF0FC080EF95E09F9344
:107730008F9384EF91E09F938F930E94B1920F906B
:107740000F900F900F906DC580FF03C08EE895E0FD
:1077500002C081E995E09F938F9380EF91E09F9322
:107760008F930E94B1920F900F900F900F9059C578
:10777000809132248F93809131248F938091302493
:107780008F9380912F248F9380912E248F938091BB
:107790002D248F9380912C248F9380912B248F9371
:1077A00080912A248F93809129248F93809128247B
:1077B0008F93809127248F9385E494E09F938F93F8
:1077C0000E94B192809173020FB6F894DEBF0FBE93
:1077D000CDBF882309F425C51F928F9382E494E0DE
:1077E0009F938F930E94B1920F900F900F900F90E4
:1077F00018C5F89481E090E029E0FC01209357003F
:10780000C895E02C80E090E0FC0120935700C895DB
:10781000F02C7894F89483E090E0FC0120935700DA
:10782000C895002D82E090E0FC0120935700C89598
:10783000102D78948091CB1B8F938091CA1B8F93CE
:107840008091C91B8F938091C81B8F9328E334E0EC
:107850003F932F930E94B1921F92EF921F92FF923B
:107860001F920F931F921F9381E194E09F938F9338
:107870000E94B1920E940921809166001F928F930D
:1078800085E094E09F938F930E94B1920E94A20B97
:10789000809173020FB6F894DEBF0FBECDBF882370
:1078A00009F4BFC41F928F9382E094E09F938F935B
:1078B0000E94B1920F900F900F900F90B2C460E0B1
:1078C00070E080E090E00E94AB0B60E070E081E04F
:1078D00090E00E94AB0B80917302882309F4A1C44D
:1078E0001F928F938FEF93E09F938F930E94B1929B
:1078F0000F900F900F900F9094C40E943D1F0E9414
:10790000A20B80917302882309F48BC41F928F937A
:107910008CEF93E09F938F930E94B1920F900F9002
:107920000F900F907EC4609171027091720280E09E
:1079300090E00E94E69165EF75E00E94FA91892B34
:1079400031F5F8948CEF99E00E9424555C01009782
:1079500069F0C5010F960E942858B50184E092E0B5
:107960000E94DE54C5010E94CC55F0CF8CEF99E007
:107970000E94B155892B29F08CEF99E00E945D554A
:10798000F5CF8CEF99E00E942055789434C08CEFAD
:1079900099E00E9424555C010BEF15E0A114B1049D
:1079A00051F1F50186811F928F9380851F928F93ED
:1079B00085811F928F9381851F928F9387811F925C
:1079C0008F9384811F928F9383811F928F938281E3
:1079D0001F928F9382851F928F931F930F930E9404
:1079E0009F92C5010E94CC555C010FB6F894DEBF92
:1079F0000FBECDBFD3CF80917302882309F411C489
:107A00001F928F9389EF93E09F938F930E94B1927F
:107A10000F900F900F900F9004C40E943E2D01C450
:107A2000609171027091720280E090E00E94E69194
:107A30008C016AE376E00E94FA91892BD1F480915F
:107A4000580290915902A0915A02B0915B02977F1F
:107A50008093580290935902A0935A02B0935B020C
:107A600044E050E06AE170E088E592E00E942394EF
:107A7000D8C363EB75E0C8010E94FA91892BD1F459
:107A80008091580290915902A0915A02B0915B02E4
:107A900098608093580290935902A0935A02B09331
:107AA0005B0244E050E06AE170E088E592E00E9409
:107AB0002394B7C30E944509B4C3609171027091C9
:107AC000720280E090E00E94E691FC012081233266
:107AD000B1F44AE050E060E070E001960E94888EC8
:107AE0001B01609171027091720280E090E00E942F
:107AF000E691F4E02F1631040CF094C002C0212C62
:107B0000312C009709F48EC01982BE016F5F7F4F40
:107B10000E94662729013A014B01B82FA92F8AE05C
:107B2000829DF001839DF00D1124E95DF44E2081CA
:107B30002A8331813B8382818C8393819D8324813D
:107B40002E8335813F83868188879781998792012B
:107B5000A301B4018B2F9A2FAA80BB80CC80DD803B
:107B6000EE80FF80088519850E94178E09F45DC09C
:107B70008981882351F18CF02A81422A3B81532A42
:107B80008C81682A9D81792A2E81822A3F81932ABD
:107B90008885B82B9985A92B18C04094509460947F
:107BA000709480949094B095A0952A8142223B8154
:107BB00053228C8168229D8179222E8182223F81ED
:107BC00093228885B8239985A923408251826282B5
:107BD000738284829582B683A78348E250E06EE187
:107BE00070E087E29BE10E94239481EF93E09F93F2
:107BF0008F930E94B1928AE0829DF001839DF00DE7
:107C00001124E95DF44E20813181428153816481E8
:107C10007581868197810E9402240E94A20B0F9099
:107C20000F9003C082E00E94082985EE93E09F93A5
:107C30008F930E94B1922FEF3FEF4FEF5FEF6FEF07
:107C40007FEF8FEF9FEF0E9402240E94A20B809192
:107C500073020F900F90882309F4E3C21F928F9351
:107C600082EE93E09F938F930E94B1920F900F90BA
:107C70000F900F90D6C2609171027091720280E0F5
:107C800090E00E94E691FC0120812332A1F44AE0B9
:107C900050E060E070E001960E94888E8B01609158
:107CA00071027091720280E090E00E94E6910430CF
:107CB0001105ECF402C000E010E00097C1F04AE0CA
:107CC00050E060E070E00E94BC8F2AE0209FF0014D
:107CD000219FF00D1124E95DF44E7187608748E221
:107CE00050E06EE170E087E29BE10E94239481E026
:107CF0000E94082980917302882309F492C21F927E
:107D00008F938FED93E09F938F930E94B1920F908A
:107D10000F900F900F9085C20E946158809173025E
:107D2000882309F47EC21F928F938CED93E09F937A
:107D30008F930E94B1920F900F900F900F9071C28D
:107D40000E947D2980917302882309F46AC21F92E0
:107D50008F9389ED93E09F938F930E94B1920F9040
:107D60000F900F900F905DC280E090E00E9425215F
:107D700080917302882309F454C21F928F9386ED79
:107D800093E09F938F930E94B1920F900F900F906A
:107D90000F9047C280911D2081FF2DC00E94C51EFB
:107DA000892B49F58091141C8F938091131C8F931C
:107DB0008091121C8F938091111C8F938BEC93E018
:107DC0009F938F930E94B1928091B1288F9380915D
:107DD000B0288F938091AF288F938091AE288F9396
:107DE0008EEB93E09F938F930E94B1920FB6F8941D
:107DF000DEBF0FBECDBF0E94A20B80911D209091CF
:107E00001E2090FF63C081E090E00E943C1E3B0179
:107E10004C0180E090E00E943C1E1B012C010E945E
:107E20009A1D9F928F927F926F928DEA93E09F931B
:107E30008F930E94B1925F924F923F922F928DE961
:107E400093E09F938F930E94B192222D332D442D66
:107E5000552D662D772D882D992D0E943D1C9F93C1
:107E60008F937F936F9382E993E09F938F930E9408
:107E7000B192222D332D442D552D662D772D882D31
:107E8000992D0E949E1C9F938F937F936F9384E8FC
:107E900093E09F938F930E94B192222D332D442D16
:107EA000552D662D772D882D992D0E94FF1C9F93AF
:107EB0008F937F936F9381E793E09F938F930E94BB
:107EC000B1920FB6F894DEBF0FBECDBF0E94A20BD9
:107ED00080917302882309F4A4C11F928F938EE6C8
:107EE00093E09F938F930E94B1920F900F900F9009
:107EF0000F9097C180911D2082FF2BC021E048E0A8
:107F000061E083E00E94401380910F1C8F93809169
:107F10000E1C8F9380910D1C8F9380910C1C8F935E
:107F200080910B1C8F9380910A1C8F938091091C68
:107F30008F938091081C8F9387E593E09F938F9395
:107F40000E94B1920E94A20B0FB6F894DEBF0FBE42
:107F5000CDBF80911D2090911E2091FF41C00E94B5
:107F60008A17B62EA72E982E892E20E030E048ECF6
:107F700052E4D501F4016B2F7A2F8F2F9E2F0E9490
:107F8000F08A20E836EE45EC57E40E946F8821E045
:107F90003EED42E45EE30E94538B9B01AC0160E046
:107FA00070E080E89FE30E94A4872BE43AE34DEB66
:107FB00057E30E946F889F938F937F936F938F9265
:107FC0009F92AF92BF928EE393E09F938F930E9414
:107FD000B1920E94A20B0FB6F894DEBF0FBECDBFC8
:107FE00080917302882309F41CC11F928F938BE345
:107FF00093E09F938F930E94B1920F900F900F90F8
:108000000F900FC1609171027091720280E090E058
:108010000E94E6916FE376E00E94FA91892BB1F419
:10802000609171027091720280E090E00E94E6918E
:10803000009709F4F6C00E94D490803108F0F1C096
:1080400090915201982B90935201EBC08091520174
:108050008F701F928F9383EE91E09F938F930E9476
:10806000B1920E94A20B0F900F900F900F90D9C069
:10807000609171027091720280E090E00E94E6913E
:10808000009711F14AE050E060E070E00E94888EB5
:10809000603198F4609356021F926F938EE293E0E2
:1080A0009F938F930E94B19241E050E067E170E0AE
:1080B00086E592E00E94239411C0809156021F929F
:1080C0008F9385E293E006C0809156021F928F93B2
:1080D0008CE193E09F938F930E94B1920F900F9049
:1080E0000F900F900E94A20B80917302882309F4D5
:1080F00098C01F928F9389E193E09F938F930E9482
:10810000B1920F900F900F900F908BC06091710201
:108110007091720280E090E00E94E6918C016EE81E
:1081200075E00E94FA91892BE1F40E943C668091EF
:10813000580290915902A0915A02B0915B0290614D
:108140008093580290935902A0935A02B0935B0215
:1081500044E050E06AE170E088E592E00E942394F8
:1081600060C061E975E0C8010E94FA91892B81F530
:10817000F8940E944A6688E10FB6F89480936000F4
:10818000109260000FBE84B7877F84BF809160002B
:10819000886180936000109260007894809158020A
:1081A00090915902A0915A02B0915B029F7E8093F8
:1081B000580290935902A0935A02B0935B0244E094
:1081C00050E06AE170E088E592E00E94239429C0C3
:1081D00064E476E0C8010E94FA91409158025091FF
:1081E000590260915A0270915B02892B21F454FF6D
:1081F00018C0F894FFCF54FF03C08EE895E002C08A
:1082000081E995E09F938F938FED91E09F938F93FA
:108210000E94B1920F900F900F900F9002C00E9499
:10822000611FEA85FB851182108283E02B960FB6D1
:10823000F894DEBF0FBECDBFDF91CF911F910F919C
:10824000FF90EF90DF90CF90BF90AF909F908F9076
:108250007F906F905F904F903F902F9008950F9375
:108260001F93CF93DF93EC018A0188819981009756
:1082700011F18B36904121F01982188283E020C0E1
:108280006231E9F4A80162E170E08DEE99E00E94AC
:10829000752E84E080939028109292281092912855
:1082A000109394280093932840E958E262E184E314
:1082B00092E00E9437548BE690E19983888381E0B5
:1082C000DF91CF911F910F9108950E9430666C9AB3
:1082D0006B9A6A9A6F9A729A749A739A779A80983C
:1082E00080B3897F80BB8398849887E080937E00E9
:1082F000549A0E94312B0E94632B81E00E94B7099F
:1083000080E090E00E94F70C60915202709153025D
:1083100080915402909155020E94985F0E94A60A93
:1083200060931F247093202480932124909322240F
:108330008091580286FD239A0895CF93DF93EC0134
:1083400088819981009741F08635904109F48CC06D
:108350001982188283E093C00E946541809158027F
:1083600080FD05C081FF01C01D9B0E948B6780912D
:1083700070008C7F809370008091B6008062809343
:10838000B6001092B20082E08093B1008091B600F6
:108390008770E1F78091700081608093700063E6E0
:1083A00079E080E090E00E941A660E946B2080E0F5
:1083B0000E94492280EE9EE09F938F930E94B1928B
:1083C0000E94211080911D200F900F9086FD0E9429
:1083D000CE6080911D2090911E2090FD0E94561D20
:1083E00080911D2087FF06C021E04CE061E080ED18
:1083F0000E9471618091C1090E942D6A809157028B
:108400000E94D4680E94D1688093EC098091570241
:108410000E94D4688091C1091F928F938091EC09CA
:108420001F928F9389E496E09F938F930E949F926F
:108430001092EE091092ED090F900F900F900F908F
:108440000F900F9088E492E09093AC288093AB2833
:1084500083E290E09093FF118093FE1186E590E116
:108460009983888381E00BC06332E1F748E454E2EA
:1084700060E070E08DEE99E00E94752EE3CFDF9111
:10848000CF9108958436910514F19F938F938BE5D6
:1084900096E09F938F930E949F92809127249091C2
:1084A0002824A0912924B0912A240196A11DB11D50
:1084B0008093272490932824A0932924B0932A24DE
:1084C0000F900F900F900F9081E090E0089580E062
:1084D00090E008952F923F924F925F926F927F9219
:1084E0008F929F92AF92BF92CF92DF92EF92FF92C4
:1084F0000F931F93CF93DF93CDB7DEB7C859D10940
:108500000FB6F894DEBF0FBECDBFCF56DF4F9983B5
:108510008883C159D0408A01633871F481EF99E0B2
:10852000C856DF4F6883C859D0400E947A52C85657
:10853000DF4F6881C859D040CF56DF4FA881B9813D
:10854000C159D0402D913C912330B0E13B0709F453
:10855000C9C340F42115310581F021343E4009F4AE
:1085600007C4FBC3253140E1340709F4D7C32C31DC
:10857000304111F40C94824FF0C34AEE52E061E8AE
:1085800070E081EF99E00E94605281E49EE0A1C317
:10859000E3E0F0E0EC0FFD1FE20FF31F1082C901D2
:1085A0000E944242892B89F720E030E040E050E011
:1085B000C357DF4F6881CD58D040627070E080E0D3
:1085C00090E0A0E00E94208E09F084C6C557DF4FDE
:1085D0002881CB58D040287030E040E050E060E087
:1085E00070E080E090E0A0E00E94208EA1F127E002
:1085F0004AE250E06BE270E089E290E00E94B25CF7
:1086000082EA98E20E94205FBC01882777FD80956E
:10861000982F0E940E8920E030E048EC52E40E943E
:108620006F889F938F937F936F938FE896E09F93CC
:108630008F931F9287E78F93CE018E0D9F1D039618
:108640009F938F930E940293E80EF91E0FB6F89441
:10865000DEBF0FBECDBFC557DF4F2881CB58D040FE
:10866000207130E040E050E060E070E080E090E0B9
:10867000A0E00E94208EF1F126E04AE250E06BE299
:1086800070E089E290E00E94B25C81E090E00E949C
:10869000300B8093C00980E89BE10E94205FBC0101
:1086A000882777FD8095982F0E940E8920E030E082
:1086B00048EC52E40E946F889F938F937F936F934F
:1086C00089E996E09F938F931F9287E78F93C70165
:1086D0000296E1E0F0E0EC0FFD1F8E0F9F1F9F93CD
:1086E0008F930E940293E80EF91E0FB6F894DEBF36
:1086F0000FBECDBF272D30E040E050E060E070E0DD
:1087000080E090E0A0E00E94208E01F10E94EC0A3F
:108710009F938F937F936F9384EA96E09F938F93B9
:108720001F9287E78F93C701029641E050E04C0FFC
:108730005D1F840F951F9F938F930E940293E80EF5
:10874000F91E0FB6F894DEBF0FBECDBFC557DF4F81
:108750002881CB58D040207430E040E050E060E009
:1087600070E080E090E0A0E00E94208E31F18091E6
:1087700022248F93809121248F93809120248F93A2
:1087800080911F248F9382EB96E09F938F931F928B
:1087900087E78F93C7010296A1E0B0E0AC0FBD1F41
:1087A0008A0F9B1F9F938F930E940293E80EF91EDE
:1087B0000FB6F894DEBF0FBECDBFC557DF4F28817F
:1087C000CB58D040207830E040E050E060E070E0EE
:1087D00080E090E0A0E00E94208E41F1F89480912A
:1087E000882890918928A0918A28B0918B28789424
:1087F000BF93AF939F938F9380EC96E09F938F935B
:108800001F9287E78F93C701029621E030E02C0F7B
:108810003D1F820F931F9F938F930E940293E80E38
:10882000F91E0FB6F894DEBF0FBECDBF20E0C457CF
:10883000DF4F3881CC58D040317040E050E060E0EC
:1088400070E080E090E0A0E00E94208E09F054C526
:1088500020E0C457DF4F3881CC58D040327040E020
:1088600050E060E070E080E090E0A0E00E94208EA8
:1088700009F0B5C520E0C457DF4F3881CC58D0404F
:10888000347040E050E060E070E080E090E0A0E014
:108890000E94208E09F0D4C520E0C457DF4F3881F4
:1088A000CC58D040387040E050E060E070E080E0AC
:1088B00090E0A0E00E94208E09F0F1C520E0C457AE
:1088C000DF4F3881CC58D040307140E050E060E05C
:1088D00070E080E090E0A0E00E94208E09F052C697
:1088E00020E0C457DF4F3881CC58D040307240E090
:1088F00050E060E070E080E090E0A0E00E94208E18
:1089000009F070C620E030E040E050E0C357DF4F90
:108910006881CD58D040647070E080E090E0A0E0C5
:108920000E94208E09F08CC620E0C057DF4F3881AE
:10893000C059D04040E050E060E070E080E090E05E
:10894000A0E00E94208E09F0E8C620E0CA56DF4F62
:108950003881C659D04040E050E060E070E080E0EF
:1089600090E0A0E00E94208E09F005C720E030E0F2
:10897000402F417050E060E070E080E090E0A0E0C7
:108980000E94208E09F025C720E030E0402F427081
:1089900050E060E070E080E090E0A0E00E94208E77
:1089A00009F04AC720E030E0C657DF4F4881CA5877
:1089B000D04050E060E070E080E090E0A0E00E94F5
:1089C000208E09F06CC720E030E0402F487050E066
:1089D00060E070E080E090E0A0E00E94208E09F06E
:1089E00088C720E030E0402F407150E060E070E048
:1089F00080E090E0A0E00E94208E09F0AAC720E06D
:108A000030E0402F407250E060E070E080E090E0A5
:108A1000A0E00E94208E09F0CCC720E030E0402F7B
:108A2000407450E060E070E080E090E0A0E00E94E0
:108A3000208E09F0EFC7F02FF078BF2E20E030E055
:108A40004F2F50E060E070E080E090E0A0E00E94F6
:108A5000208E11F00C943B4D212F2170C22E20E06E
:108A600030E040E05C2D60E070E080E090E0A0E06D
:108A70000E94208E11F00C94484D20E030E04B2DE8
:108A800050E060E070E080E090E0A0E00E94208E86
:108A900011F00C94564D20E030E040E05C2D60E099
:108AA00070E080E090E0A0E00E94208E11F00C9435
:108AB0008B4D20E030E040E0512F527060E070E0DC
:108AC00080E090E0A0E00E94208E11F00C94C04D58
:108AD00020E030E040E0512F547060E070E080E032
:108AE00090E0A0E00E94208E11F00C94F34D20E065
:108AF00030E040E0512F507160E070E080E090E0A5
:108B0000A0E00E94208E11F00C94264E20E030E070
:108B100040E0512F507260E070E080E090E0A0E013
:108B20000E94208E11F00C94654E20E030E040E071
:108B3000512F507460E070E080E090E0A0E00E946F
:108B4000208E11F00C94A44E20E030E040E0512F34
:108B5000587060E070E080E090E0A0E00E94208E1D
:108B600011F00C94E34E20E030E040E05D2D60E039
:108B700070E080E090E0A0E00E94208E11F00C9464
:108B8000144F779A8091C5099091C60992FD749A05
:108B9000C557DF4F2881CB58D040C457DF4F3881AD
:108BA000CC58D040A801C357DF4F6881CD58D04082
:108BB000CD56DF4F7881C359D040CC56DF4F8881E6
:108BC000C459D040CB56DF4F9881C559D040A0E062
:108BD0008E010D5F1F4F0E94208E11F00C94504F9C
:108BE00080915602806189838091E5098A83F8012A
:108BF000EE0DFF1D10828091C5099091C609870175
:108C00000D5F1F4F80FF0CC01F930F9387E598E007
:108C10009F938F930E949F920F900F900F900F90B1
:108C2000B801CE0101960E94A95B8091580282FF93
:108C30000AC028E834E2A801BE016F5F7F4F81E6D9
:108C400092E00E943E608091C5099091C60982FD24
:108C500073980E94D36781EF99E00E947C528091C3
:108C6000580290915902A0915A02B0915B0290FF74
:108C700040C03FEFE31AF30A0E94D168D82E89E181
:108C80000E94E968409158025091590260915A023D
:108C900070915B0250FF29C073988091E5098F5F46
:108CA0008093E5098A83B7016F5F7F4FCE010196FC
:108CB0000E94A95B81EF99E00E947C5240E050E065
:108CC00065E880910212909103120E94375483E06C
:108CD00090E1CF56DF4FA881B981C159D0408D9323
:108CE0009C9338C0E12CF12CCDCF8D2D0E94E968EA
:108CF000739A8091C2099091C309892B11F00E9447
:108D00008B678091E5098F5F8093E5098091C509A4
:108D10009091C60982FF39CC739A37CC8DED99E0DA
:108D20000E94DD56892BB1F00E94D36780915802D2
:108D300087FD2B9860E470E08DED99E00E94B656B7
:108D40008CE190E1CF56DF4FE881F981C159D040E5
:108D50009183808381E00C94954FCF56DF4FA8819B
:108D6000B981C159D0401D921C9283E00C94954F5B
:108D7000623181F7C0905802D0905902E0905A02B7
:108D8000F0905B02D1FC01CCF8018081813091F53B
:108D90000180F281E02D2081C557DF4F2883CB5819
:108DA000D0403181C457DF4F3883CC58D040028146
:108DB00013814481C357DF4F4883CD58D04055813C
:108DC000CD56DF4F5883C359D0408681CC56DF4FF4
:108DD0008883C459D0409781CB56DF4F9883C559BB
:108DE000D04020843184C257DF4F19821882CE5878
:108DF000D0406AC08230E9F4A381B481C257DF4F0A
:108E0000B983A883CE58D040212C312CB1E0C5576E
:108E1000DF4FB883CB58D040C457DF4F1882CC58AF
:108E2000D04000E010E8C357DF4F1882CD58D04043
:108E30003CC08330F9F0843009F0A7CB212C312CD1
:108E4000C257DF4F19821882CE58D040E5E0C5578F
:108E5000DF4FE883CB58D040C457DF4F1882CC583F
:108E6000D04000E010E0F2E0C357DF4FF883CD5868
:108E7000D0401BC0212C312CC257DF4F19821882E1
:108E8000CE58D04025E0C557DF4F2883CB58D0407F
:108E9000C457DF4F1882CC58D04000E010E031E0DA
:108EA000C357DF4F3883CD58D040CD56DF4F18829F
:108EB000C359D040CC56DF4F1882C459D040CB564E
:108EC000DF4F1882C559D04080901F2490902024F5
:108ED000A0902124B09022244090800250908102E2
:108EE00060908202709083022DEC3CEC4CE45EE3D7
:108EF000C301B2010E94A5879B01AC01C501B40169
:108F00000E94318A87FD0BC0E894E0F8C0925802B5
:108F1000D0925902E0925A02F0925B024AC0A30139
:108F20009201C501B4010E946B8887FF42C0809105
:108F30002B2490912C24A0912D24B0912E240196C5
:108F4000A11DB11D80932B2490932C24A0932D243C
:108F5000B0932E24E0FC19CB6894E0F8C09258023C
:108F6000D0925902E0925A02F0925B0245E4C55752
:108F7000DF4F4883CB58D04050E2C457DF4F58836F
:108F8000CC58D04000E010E084E0C357DF4F888326
:108F9000CD58D040CD56DF4F1882C359D040CC5663
:108FA000DF4F1882C459D040CB56DF4F1882C559C5
:108FB000D040902F9470C657DF4F9883CA58D04046
:108FC00020E030E0492F50E060E070E080E090E089
:108FD000A0E00E94208E09F08C9AC557DF4FA8812F
:108FE000CB58D040A0727A2E2A2F30E040E050E0DB
:108FF00060E070E080E090E0A0E00E94208E11F040
:109000000E94EC0AC457DF4FB881CC58D040B074EE
:10901000C057DF4FB883C059D04020E03B2F40E01D
:1090200050E060E070E080E090E0A0E00E94208EE0
:1090300011F00E94C51EC457DF4FE881CC58D040C4
:10904000E078CA56DF4FE883C659D04020E03E2F73
:1090500040E050E060E070E080E090E0A0E00E943E
:10906000208E51F00E94920A609395287093962862
:109070008093972890939828C557DF4F2881CB5825
:10908000D040217030E040E050E060E070E080E0EF
:1090900090E0A0E00E94208EF1F08EE09BE19F9393
:1090A0008F938FE696E09F938F931F9287E78F931E
:1090B000CE0103969F938F930E9402936C010E94AE
:1090C00042420FB6F894DEBF0FBECDBF892B09F028
:1090D0005CCA760102C0E12CF12CC557DF4F288114
:1090E000CB58D040227030E040E050E060E070E0CB
:1090F00080E090E0A0E00E94208ED1F1C7010296AE
:1091000067E776E041E050E04C0F5D1F840F951F4C
:109110000E94039253E0E50EF11C22EAA22E28E2FF
:10912000B22E32EFC32E33E0D32E47E7942ED50173
:109130008D915D011F928F93DF92CF921F929F922C
:10914000C7010296E1E0F0E0EC0FFD1F8E0F9F1FBC
:109150009F938F930E940293E80EF91E0FB6F89426
:10916000DEBF0FBECDBF3AEAA31638E2B306F9F66A
:10917000C557DF4F2881CB58D040247030E040E005
:1091800050E060E070E080E090E0A0E00E94208E7F
:1091900009F447C0C70102966BE776E041E050E072
:1091A0004C0F5D1F840F951F0E94039254E0E50E43
:1091B000F11C4E018AE7880E911C80E1D4011D92BA
:1091C0008A95E9F728E0A40168E980EB0E94841100
:1091D0005401B8E0AB0EB11C82EFC82E83E0D82E4C
:1091E00097E7692EF40181914F011F928F93DF92CF
:1091F000CF921F926F92C701029621E030E02C0FB0
:109200003D1F820F931F9F938F930E940293E80E3E
:10921000F91E0FB6F894DEBF0FBECDBF8A149B04B3
:1092200009F7512F5078D52E20E030E040E060E083
:1092300070E080E090E0A0E00E94208EE1F4809158
:10924000C2099091C3099F938F9380E896E09F9302
:109250008F931F9287E78F93CE018E0D9F1D0396EC
:109260009F938F930E940293E80EF91E0FB6F89415
:10927000DEBF0FBECDBF20E030E040E050E0C3577E
:10928000DF4F6881CD58D040617070E080E090E0A1
:10929000A0E00E94208E09F487C9E3E0F0E0EC0F23
:1092A000FD1FEE0DFF1D80E28083EBE4F4E2808180
:1092B00097012F5F3F4F7901882309F469C98081A5
:1092C000A1E0B0E0AC0FBD1FAE0DBF1D12968C9398
:1092D0003196EDCFCE018E0D9F1D67E876E00396A7
:1092E0000E94039297E0E90EF11CC7010E944242DE
:1092F000892B09F04AC96AC92114310409F4A8CAA2
:10930000F894409088285090892860908A2870901E
:109310008B2878948091781B9091791BA0917A1B6F
:10932000B0917B1BA3019201281B390B4A0B5B0BED
:10933000CA01B9010E940C894B015C01B10180E0B6
:1093400090E00E940C899B01AC01C501B4010E9410
:109350006F88B82EC92E9F938F937F936F938BEC5A
:1093600096E09F938F931F9287E78F939E012E0D18
:109370003F1D2D5F3F4F3F932F93C856DF4F6883AC
:10938000C859D040C956DF4F7883C759D0400E9492
:109390000293E80EF91EC856DF4F6881C859D040C5
:1093A000C956DF4F7881C759D040862F972FAB2DF4
:1093B000BC2D80939A2890939B28A0939C28B093CF
:1093C0009D284092781B5092791B60927A1B709274
:1093D0007B1B0FB6F894DEBF0FBECDBF39CA211478
:1093E000310409F447CAF89480914F1B9091501BA7
:1093F000A091511BB091521B78949F938F938091B1
:109400005F028F9380915E028F9388ED96E09F9329
:109410008F931F9287E78F93C7010296A1E0B0E078
:10942000AC0FBD1F8A0F9B1F9F938F930E940293C7
:10943000E80EF91E0FB6F894DEBF0FBECDBF1ACAF4
:10944000F89480918C2890918D28A0918E28B091CD
:109450008F287894BF93AF939F938F9388EE96E075
:109460009F938F931F9287E78F93C701029621E006
:1094700030E02C0F3D1F820F931F9F938F930E940C
:109480000293E80EF91EC7010E9442420FB6F894FB
:10949000DEBF0FBECDBF892B09F077C8FDC92114EF
:1094A000310409F40BCAF89440908C2850908D2810
:1094B00060908E2870908F28789480917C1B90917A
:1094C0007D1BA0917E1BB0917F1BA3019201281BE5
:1094D000390B4A0B5B0BCA01B9010E940C894B0185
:1094E0005C01B10180E090E00E940C899B01AC011D
:1094F000C501B4010E946F88B82EC92E9F938F9327
:109500007F936F9383EF96E09F938F931F9287E7EC
:109510008F939E012E0D3F1D2D5F3F4F3F932F9345
:10952000C856DF4F6883C859D040C956DF4F78838B
:10953000C759D0400E940293E80EF91EC856DF4F6B
:109540006881C859D040C956DF4F7881C759D0408B
:10955000862F972FAB2DBC2D80939E2890939F280C
:10956000A093A028B093A12840927C1B50927D1B11
:1095700060927E1B70927F1B0FB6F894DEBF0FBE09
:10958000CDBF9CC9232809F4ABC9F8948091531B23
:109590009091541BA091551BB091561B78949F93AA
:1095A0008F9380915D028F9380915C028F9380E016
:1095B00097E09F938F931F9287E78F93C70102963F
:1095C000A1E0B0E0AC0FBD1F8A0F9B1F9F938F934C
:1095D0000E940293E80EF91E0FB6F894DEBF0FBE8C
:1095E000CDBF7EC98091232490912424A09125246D
:1095F000B0912624BF93AF939F938F9380E197E020
:109600009F938F931F9287E78F93C701029621E064
:1096100030E02C0F3D1F820F931F9F938F930E946A
:109620000293E80EF91EC7010E9442420FB6F89459
:10963000DEBF0FBECDBF892B11F00C94C54262C9AD
:1096400080912E248F9380912D248F9380912C24B0
:109650008F9380912B248F9380912A248F938091D4
:1096600029248F93809128248F93809127248F938E
:109670008BE197E09F938F931F92B7E7CB2ECF920A
:10968000C7010296A1E0B0E0AC0FBD1F8A0F9B1F7F
:109690009F938F930E940293E80EF91EC7010E94C8
:1096A00042420FB6F894DEBF0FBECDBF892B11F03A
:1096B0000C94C54280911D2090911E2090FF34C9CA
:1096C000809132248F93809131248F938091302424
:1096D0008F9380912F248F938FE397E09F938F93A5
:1096E0001F92CF92C701029621E030E02C0F3D1F60
:1096F000820F931F9F938F930E940293E80EF91E8F
:10970000C7010E9442420FB6F894DEBF0FBECDBF24
:10971000892B11F00C94C54207C98091141C8F93BA
:109720008091131C8F938091121C8F938091111C38
:109730008F9381E597E09F938F931F9287E78F9395
:10974000C7010296A1E0B0E0AC0FBD1F8A0F9B1FBE
:109750009F938F930E940293E80EF91EC7010E9407
:1097600042420FB6F894DEBF0FBECDBF892B11F079
:109770000C94C542EAC8809198288F9380919728CD
:109780008F93809196288F93809195288F938CE565
:1097900097E09F938F931F9287E78F93C70102965D
:1097A00021E030E02C0F3D1F820F931F9F938F937A
:1097B0000E940293E80EF91EC7010E9442420FB6B2
:1097C000F894DEBF0FBECDBF892B11F00C94C542BB
:1097D000CDC881E00E94430A20917802309179023D
:1097E00040917A0250917B020E94F08A9F938F935E
:1097F0007F936F9389E697E09F938F931F9287E7FC
:109800008F93C7010296A1E0B0E0AC0FBD1F8A0F95
:109810009B1F9F938F930E940293E80EF91EC7012E
:109820000E9442420FB6F894DEBF0FBECDBF892B17
:1098300011F00C94C542A8C882E00E94430A20910E
:1098400074023091750240917602509177020E9425
:10985000F08A9F938F937F936F9386E797E09F9310
:109860008F931F9287E78F93C701029621E030E024
:109870002C0F3D1F820F931F9F938F930E94029383
:10988000E80EF91EC7010E9442420FB6F894DEBFEF
:109890000FBECDBF892B11F00C94C54283C883E065
:1098A0000E94430A9F938F937F936F9383E897E07F
:1098B0009F938F931F9287E78F93C7010296A1E032
:1098C000B0E0AC0FBD1F8A0F9B1F9F938F930E9428
:1098D0000293E80EF91E8C98C7010E9442420FB60F
:1098E000F894DEBF0FBECDBF892B11F00C94C5429A
:1098F0006AC880911D2087FF74C821E042E161E0C1
:1099000080ED0E9471619F938F937F936F9380E9A5
:1099100097E09F938F931F9287E78F93C7010296DB
:1099200021E030E02C0F3D1F820F931F9F938F93F8
:109930000E940293E80EF91EC7010E9442420FB630
:10994000F894DEBF0FBECDBF892B11F00C94C54239
:1099500048C880911D2087FF52C821E042E162E0A3
:1099600080ED0E9471619F938F937F936F938EE937
:1099700097E09F938F931F9287E78F93C70102967B
:10998000A1E0B0E0AC0FBD1F8A0F9B1F9F938F9388
:109990000E940293E80EF91EC7010E9442420FB6D0
:1099A000F894DEBF0FBECDBF892B11F00C94C542D9
:1099B00026C880911D2087FF30C821E042E163E086
:1099C00080ED0E9471619F938F937F936F938CEAD8
:1099D00097E09F938F931F9287E78F93C70102961B
:1099E00021E030E02C0F3D1F820F931F9F938F9338
:1099F0000E940293E80EF91EC7010E9442420FB670
:109A0000F894DEBF0FBECDBF892B11F00C94C54278
:109A10000C940D4580911D2087FF0DC821E042E187
:109A200064E080ED0E9471619F938F937F936F93A9
:109A30008AEB97E09F938F931F9287E78F93C701DD
:109A40000296A1E0B0E0AC0FBD1F8A0F9B1F9F9351
:109A50008F930E940293E80EF91EC7010E944242B2
:109A60000FB6F894DEBF0FBECDBF892B11F00C945A
:109A7000C5420C941B4580911D2082FD02C00C94B0
:109A80002C4546E061E083E00E9440130C942C4595
:109A900080911D2082FD02C00C943D4521E046E0EE
:109AA00061E083E00E9440130C943D4580911D20AD
:109AB00082FD02C00C944B4580910B1C8F938091CA
:109AC0000A1C8F938091091C8F938091081C8F939F
:109AD00088EC97E09F938F931F9287E78F93C7013E
:109AE000029641E050E04C0F5D1F840F951F9F933D
:109AF0008F930E940293E80EF91EC7010E94424212
:109B00000FB6F894DEBF0FBECDBF892B11F00C94B9
:109B1000C5420C944B4580911D2082FD02C00C94DF
:109B2000594580910F1C8F9380910E1C8F938091CB
:109B30000D1C8F9380910C1C8F9380ED97E09F9369
:109B40008F931F9287E78F93C7010296E1E0F0E0C1
:109B5000EC0FFD1F8E0F9F1F9F938F930E94029308
:109B6000E80EF91EC7010E9442420FB6F894DEBF0C
:109B70000FBECDBF892B11F00C94C5420C945945F2
:109B800080911D2090911E2090FD02C00C9468458C
:109B900080E090E00E943C1E9F938F937F936F9391
:109BA0008BED97E09F938F931F9287E78F93C70169
:109BB000029641E050E04C0F5D1F840F951F9F936C
:109BC0008F930E940293E80EF91EC7010E94424241
:109BD0000FB6F894DEBF0FBECDBF892B11F00C94E9
:109BE000C5420C94684580911D2090911E2090FDE7
:109BF00002C00C94774581E090E00E943C1E9F9348
:109C00008F937F936F938BEE97E09F938F931F9229
:109C100087E78F93C7010296E1E0F0E0EC0FFD1FAC
:109C20008E0F9F1F9F938F930E940293E80EF91E41
:109C3000C7010E9442420FB6F894DEBF0FBECDBFEF
:109C4000892B11F00C94C5420C94774580911D200E
:109C500090911E2090FD02C00C94864581E090E01A
:109C60000E943C1E4B015C0180E090E00E943C1E83
:109C70009B01AC01C501B4010E943D1C9F938F93D1
:109C80007F936F938CEF97E09F938F931F9287E75B
:109C90008F93C701029641E050E04C0F5D1F840F87
:109CA000951F9F938F930E940293E80EF91EC701A0
:109CB0000E9442420FB6F894DEBF0FBECDBF892B83
:109CC00011F00C94C5420C94864580911D20909112
:109CD0001E2090FD02C00C94954581E090E00E940A
:109CE0003C1E4B015C0180E090E00E943C1E9B0109
:109CF000AC01C501B4010E949E1C9F938F937F937A
:109D00006F9387E098E09F938F931F9287E78F93DD
:109D1000C7010296E1E0F0E0EC0FFD1F8E0F9F1FE0
:109D20009F938F930E940293E80EF91EC7010E9431
:109D300042420FB6F894DEBF0FBECDBF892B11F0A3
:109D40000C94C5420C94954580911D2090911E2045
:109D500090FD02C00C94A44581E090E00E943C1E5E
:109D60004B015C0180E090E00E943C1E9B01AC0135
:109D7000C501B4010E94FF1C9F938F937F936F9343
:109D800085E198E09F938F931F9287E78F93C70198
:109D9000029641E050E04C0F5D1F840F951F9F938A
:109DA0008F930E940293E80EF91EC7010E9442425F
:109DB0000FB6F894DEBF0FBECDBF892B11F00C9407
:109DC000C5420C94A44580911D2090911E2091FDC8
:109DD00002C00C94B3450E948A179F938F937F9380
:109DE0006F9388E298E09F938F931F9287E78F93FA
:109DF000C7010296E1E0F0E0EC0FFD1F8E0F9F1F00
:109E00009F938F930E940293E80EF91EC7010E9450
:109E100042420FB6F894DEBF0FBECDBF892B11F0C2
:109E20000C94C5420C94B345C257DF4FA881B98149
:109E3000CE58D04016968C9116971F928F931596F8
:109E40008C9115971F928F9313968C9113971F9255
:109E50008F9312968C911F928F9389E398E09F9332
:109E60008F931F9287E78F93C7010296E1E0F0E09E
:109E7000EC0FFD1F8E0F9F1F9F938F930E940293E5
:109E8000E80EF91EC7010E9442420FB6F894DEBFE9
:109E90000FBECDBF892B11F00C94C5420C94C14567
:109EA0008091C5099091C60982FD0CC0809158022D
:109EB00080FD08C081FD02C00C94F0451D9902C0D0
:109EC0000C94F0451F930F9380E598E09F938F9338
:109ED0000E949F92809173020F900F900F900F90AD
:109EE000882311F40C94F0451F928F938DED9EE022
:109EF0009F938F930E94B1920F900F900F900F90AD
:109F00000C94F0458DED99E00E94DD56892B11F4FB
:109F10000C94AA460E948B678091580287FD02C06C
:109F20000C94C5422B9A0C94C542C856DF4F0FB60D
:109F3000F894DEBF0FBECDBFDF91CF911F910F917F
:109F4000FF90EF90DF90CF90BF90AF909F908F9059
:109F50007F906F905F904F903F902F9008950C945A
:109F6000A3524F925F926F927F928F929F92AF9285
:109F7000BF92CF92DF92EF92FF920F931F93CF93F6
:109F8000DF93CDB7DEB760970FB6F894DEBF0FBE94
:109F9000CDBF6B010E94D168E82FF0E0EE0FFF1FEC
:109FA000EF5BF44E80819181019691838083809153
:109FB000C5099091C60981FD7498809058029090CF
:109FC0005902A0905A02B0905B020E94FD5A7C0197
:109FD000FC018081982F92959F70913099F48F7039
:109FE00051F48091251B9091261B01969093261B7E
:109FF0008093251B07C1B60182EB98E20E9419529B
:10A00000892B51F08091231B9091241B01969093F2
:10A01000241B8093231BF6C0D501C4011EE0B69516
:10A02000A795979587951A95D1F7F82FF1708F2EF0
:10A030008CEF99E00E9424558C01009709F448C0E8
:10A04000B601C80102960E941952892BE9F19801C4
:10A050004DE759E060E074E6C8010F960E94A457EE
:10A06000F7019181F8018481981321C082858F5F67
:10A0700082878091211B9091221B01969093221B35
:10A080008093211B84E00E941A5CF801208530E057
:10A090002817390708F0A9C184E00E941A5CF8016A
:10A0A0008087F70180818F70F8018187ABC0F8014C
:10A0B000128684E00E941A5CF8018087F701808193
:10A0C0008F70F801818792C1C8010E94CC55B4CF2E
:10A0D00084E092E00E94B9548C01009709F492C088
:10A0E000B601C80102960E941052F7018181815089
:10A0F000F801848380E091E0A0E0B0E0838794875A
:10A10000A587B687128684E00E941A5CF8018087D2
:10A11000F70180818F70F8018187B8018CEF99E099
:10A120000E94845598014DE759E060E074E6C8014B
:10A130000F960E94A45799249394F7018181F80106
:10A140008483F70180818F70F801878384E00E9407
:10A150001A5CF801858383E00E941A5C5C01F801B7
:10A16000868387818F3009F0912CF7014180F801B7
:10A170008481481A512C612C712C76E0440C551CBA
:10A18000661C771C7A95D1F72385348545855685DD
:10A19000A0ECB0E00E94CE8BBB27A92F982F872F71
:10A1A000480E591E6A1E7B1E438654866586768637
:10A1B0008091C5099091C60981FD2EC080915802F9
:10A1C00080FD2AC081FD26C08091580290915902DD
:10A1D000A0915A02B0915B0297FDD2C0992091F0F4
:10A1E00082E0809334241092362410923524109308
:10A1F00038240093372444E354E262E184E392E09C
:10A200000E9437548091C5099091C60981FFF0C022
:10A21000749AEEC01D9BD8CFA4E6B0E0A3019201D2
:10A220000E94CE8B672F782F892F992724E630E064
:10A2300040E050E00E94198C7F936F93452C562C80
:10A24000672C77245F924F92BB24BF92AF92F801A4
:10A2500085811F928F93F70180818F701F928F935A
:10A2600081811F928F93F60181811F928F9380814C
:10A270001F928F93C70102969F938F9388E698E071
:10A280009F938F930E949F92809173020FB6F894D0
:10A29000DEBF0FBECDBF882361F01F928F938AED82
:10A2A0009EE09F938F930E94B1920F900F900F901A
:10A2B0000F908091580290915902A0915A02B0914A
:10A2C0005B0296FF2DC0882059F1F7012081322FC3
:10A2D0003F70832F90E00297D4F08FEF830F207FA1
:10A2E000822B808381EF99E00E94AF4F80911F1BEA
:10A2F0009091201B01969093201B80931F1B8091AF
:10A30000C5099091C60996FF0BC0739809C080914A
:10A31000251B9091261B01969093261B8093251B4D
:10A3200080911D2086FF50CF0E94C060C701059616
:10A330000E948C60F70181811F928F93F8018681C2
:10A340001F928F9385811F928F938CEA98E09F9341
:10A350008F931F9280E18F939E012F5F3F4F690182
:10A36000DF922F930E94029382E00E94A660C601B2
:10A370000E948C600FB6F894DEBF0FBECDBF24CF15
:10A380008EE09BE120910E1B222309F427CF9F939F
:10A390008F938FEB98E09F938F93FE0131966F011F
:10A3A000DF92EF930E943F935C01B601C7010296D2
:10A3B0000E9424920F900F900F900F900F900F908B
:10A3C000009709F40BCF95012F5F3F4F280F391FDE
:10A3D000A9012F5F3F4FFA0180818032C9F362E10A
:10A3E0008CE092E00E943754F9CE812C912CA5CEBE
:10A3F00060960FB6F894DEBF0FBECDBFDF91CF9150
:10A400001F910F91FF90EF90DF90CF90BF90AF9092
:10A410009F908F907F906F905F904F9008950895D8
:10A42000FB012081FC012083FB012181FC012183B0
:10A430000895FC019081DB018C91981309C081E0A3
:10A4400090E0318111962C91321721F080E008952F
:10A4500080E090E00895BC0182EB98E20C941052E9
:10A46000DC011996ED91FC911A970280F381E02DA1
:10A47000309709F0099408950F931F93CF93DF93BA
:10A4800000D0CDB7DEB78C0188E10E942D5CBC0105
:10A49000CE0101960E941052D8011996ED91FC91BF
:10A4A0001A970190F081E02DBE016F5F7F4FC801C8
:10A4B00009950F900F90DF91CF911F910F91089503
:10A4C000EF92FF920F931F93CF93DF93EC018B01D9
:10A4D0007A0142E053E00E948952FA86E98666E0FA
:10A4E00073E0C801DF91CF911F910F91FF90EF9022
:10A4F0000C94E2520C94A152CF93DF93EC0162EBE7
:10A5000078E288E10E94235CCE01DF91CF910C9428
:10A51000A352EF92FF920F931F93CF93DF93EC011F
:10A520008B017A010E94BE52F886EF826AE073E0E6
:10A53000C801DF91CF911F910F91FF90EF900C9484
:10A54000E2520C94C6520C944D6DDC011796ED91BD
:10A55000FC9118970190F081E02D0994DC01179689
:10A56000ED91FC9118970280F381E02D309709F06E
:10A570000994089580E092E10C942055FC017383C6
:10A580006283BC0180E092E10C948455BC0180E0C0
:10A5900092E10C946955CF93DF93EC0180E092E156
:10A5A0000E942455009749F0FC01228133812C1729
:10A5B0003D0729F00E94CC55F5CF80E090E0DF9177
:10A5C000CF9108950F931F93CF93DF938B010E9438
:10A5D000CB52EC01009731F01D830C83C8010E941F
:10A5E0007E6F8E83DF91CF911F910F9108951F93FE
:10A5F000CF93DF93EC01162FEC81FD813097D1F0E2
:10A60000909303128093021282E08887CE0106960F
:10A610000995992787FD90950297029710F01338B6
:10A6200039F4BE01CE01DF91CF911F910C942453D8
:10A6300081E08887DF91CF911F910895FC012085EB
:10A6400020FD0C94F7520895CF92DF92EF92FF9283
:10A650000F931F93CF93DF93EC016B01E0900212F5
:10A66000F09003120091041210910512F801EC17FA
:10A67000FD0739F0309709F44AC00190F081E02DD0
:10A68000F6CF209709F443C08885882309F11886FE
:10A690000115110561F0C017D10729F0AE0167E877
:10A6A000C8010E941E53F80100811181F1CFEC8195
:10A6B000FD81309769F0CC15DD0551F0D093031280
:10A6C000C093021240E050E063E8CE01069609957F
:10A6D000E0910412F0910512CE17DF0769F488812A
:10A6E000998190930512809304120DC0808191810D
:10A6F0008C179D0721F0FC013097C1F704C08881B9
:10A70000998191838083F0920312E0920212DF918B
:10A71000CF911F910F91FF90EF90DF90CF90089510
:10A720001F93CF93DF9310920E12C0910412D09119
:10A73000051211E0209779F08985882341F0188768
:10A74000198640E050E062E8CE010E94F75209907D
:10A75000D881C02DEFCFDF91CF911F9108958091C7
:10A76000B11291E0980F9093B11208956091021286
:10A77000709103120C9424538AE88093B1121092C2
:10A78000AF121092B0121092051210920412109291
:10A79000031210920212089580910E1281110E94EC
:10A7A00090537091B012772309F451C0E091AF1229
:10A7B0002E2F30E085E0E89FF0011124E15FFD4E8F
:10A7C000608160930D124181528150930C1240932D
:10A7D0000B128381948190930A12809309122F5F48
:10A7E0003F4F2F7133272093AF1271507093B012E7
:10A7F000009731F580910412909105129093081200
:10A80000809307128091071290910812892BF9F01A
:10A8100080910E1281110E94905340910B12509121
:10A820000C1260910D1280910712909108120E94F3
:10A830001E53E0910712F091081280819181DECFC2
:10A84000613819F421E0FC0120870E941E53809199
:10A850000E122091B01290E0820F911D0895809108
:10A860000E122091B01290E0820F911D0895209158
:10A87000B0122032B9F0E091AF12E20FEF71E09325
:10A88000061235E0E39FF0011124E15FFD4E608385
:10A8900052834183948383832F5F2093B01280E09F
:10A8A00090E0089581E090E00895CF93DF93C09108
:10A8B0000212D09103120E941E53D0930312C09330
:10A8C0000212DF91CF910895AB01309104122091D3
:10A8D0000512E32FF22FE817F907B1F0309721F0B6
:10A8E0000190F081E02DF7CF009771F0FC013083EB
:10A8F0002183909305128093041221E02087178210
:10A90000168261E80C9455540895009749F0FC01B3
:10A9100020852150223020F421E0218720930E123F
:10A92000089521E030E0FC018085811102C020E023
:10A9300030E0C9010895CF93DF93EC014A815B8138
:10A9400060E070E08C819D810E94F3912A813B81BF
:10A9500088819981289FA001299F500D389F500D13
:10A96000112460E070E08E819F81DF91CF910C9483
:10A97000F391FC018281938120E030E028173907B0
:10A98000D1F0A481B581A20FB31F4C91411110C029
:10A9900081E08C9380819181289FA001299F500D97
:10A9A000389F500D112486819781840F951F08953B
:10A9B0002F5F3F4FE3CF80E090E00895FC012681B8
:10A9C00037814281538180E090E084179507C9F078
:10A9D0002617370781F4A481B581A80FB91F2C91E0
:10A9E000121614F421502C930480F581E02DE80F09
:10A9F000F91F80810895A081B1812A0F3B1F019624
:10AA0000E4CF8FEF0895FC0186819781681779075D
:10AA1000A0F0A081B18142815381A49F9001A59FA4
:10AA2000300DB49F300D1124280F391F81E090E0C4
:10AA30006217730720F080E0089580E090E00895A9
:10AA4000FC01118210820895FC018081918108959A
:10AA5000FB0120813181FC01318320830895DC01D9
:10AA6000ED91FC91309731F080819181009729F030
:10AA7000FC01FACF80E090E00895CF010895DC0159
:10AA8000ED91FC9111973097A9F020813181232B12
:10AA900021F41D921C92CF010895A081B1818D9166
:10AAA0009C911197892B11F0FD01F7CF1182108233
:10AAB000CD01089580E090E00895DC01ED91FC91D6
:10AAC0001197309721F0208131812D933C93CF0154
:10AAD0000895DC01ED91FC913097A9F0A0E0B0E081
:10AAE00020813181E617F70741F4109709F4DC0162
:10AAF0002D933C931182108208952115310519F090
:10AB0000DF01F901EDCF08950F931F93CF93DF93EA
:10AB10008C01EB010E94695519821882C8010E94BC
:10AB20002F55009711F4F80101C0FC01D183C083B7
:10AB3000DF91CF911F910F9108950F931F93CF93A2
:10AB4000DF93EC018B010E94695588819981F8019E
:10AB50009183808319830883DF91CF911F910F9197
:10AB60000895DC01ED91FC9180E090E0309729F0B0
:10AB700001960190F081E02DF9CF0895FB01309707
:10AB800019F4BA010C949D5580819181DA018D935D
:10AB90009C93518340830895009721F0FC018081AC
:10ABA0009181089580E090E008958091B412909191
:10ABB000B512892B29F41092B3121092B212089593
:10ABC0000E94D864E091B412F091B51222813381D1
:10ABD00040815181240F351F281B390B0480F581DA
:10ABE000E02D309769F04281538160817181460F79
:10ABF000571F481B590B4217530780F79A01EECF96
:10AC0000280F391F3093B3122093B212089586E8AB
:10AC100092E00C948554EF92FF920F931F93CF9381
:10AC2000DF938C01FC0180819181009799F08A3536
:10AC30009105D9F0F8011182108283E068C0868105
:10AC400097818417950709F049C00480F581E02DAC
:10AC50003097A9F71092B5121092B4128AE590E0DD
:10AC6000F8019183808381E052C0673891F16238A6
:10AC7000A9F7C091B412D091B512E12CF12C209714
:10AC800069F3CE010E944F73892BF1F0AE0168E8A1
:10AC90008E819F810E943754892BA1F41F821E82CE
:10ACA0008C819D81E114F10421F0F7019583848367
:10ACB00004C09093B5128093B4121D821C820E942E
:10ACC000D555D7CF0E9407567E010C80DD81C02D5F
:10ACD000D6CFE091B412F091B512BACFF093B5127D
:10ACE000E093B412A481B581109709F4B7CF1696FA
:10ACF0008D919C9117978417950711F0FD01F2CF64
:10AD000014968D919C91159795838483EBCFDF9159
:10AD1000CF911F910F91FF90EF900895CF93DF9304
:10AD2000EC010E9407568E819F813091B4122091D0
:10AD3000B512892B59F0E32FF22F309739F0EC1729
:10AD4000FD0781F00480F581E02DF7CF809102129C
:10AD5000909103129F838E833C832D83D093B512F1
:10AD6000C093B412DF91CF910C94D555CF93DF935C
:10AD7000EC010E942F73CE01DF91CF910C948E567F
:10AD8000CF93DF93EC010E943B73CE01DF91CF9113
:10AD90000C948E56CF93DF93EC010E944573CE0145
:10ADA000DF91CF910C948E56FC0120813181260FCA
:10ADB000371F318320830C94D55521E030E0FC010E
:10ADC00086819781892B11F020E030E0C901089538
:10ADD000FC012281338180819181820F931F08952C
:10ADE000FC0180819181089581E090E02091B4126E
:10ADF0003091B512232B11F480E090E008958091FA
:10AE0000B4129091B512892B29F08091B2129091D1
:10AE1000B312089580E090E00895CF93DF93EC01A2
:10AE2000E091B412F091B5128E179F0769F48C81EE
:10AE30009D819093B5128093B4120DC08481958149
:10AE40008C179D0721F0FC013097C1F706C08C815B
:10AE50009D81958384830E94D5551D821C821F820B
:10AE60001E82DF91CF910895EF92FF920F931F936F
:10AE7000CF93DF938C017A01FC018081918100974F
:10AE800041F08B34910501F1F8011182108283E0C9
:10AE900048C087EB92E10E942455EC01209751F0C5
:10AEA0006C817D81CE0102960E94B6560990D881B0
:10AEB000C02DF4CF81E08093B6128BE490E0F801CE
:10AEC0009183808381E02DC06838E1F787EB92E1C0
:10AED0000E942455EC01209781F3CE010296E816DA
:10AEE000F906D9F4BE0187EB92E10E946955E09022
:10AEF0000212F09003128A859B859093031280932F
:10AF00000212EC85FD85309719F08E859F85099595
:10AF1000F0920312E0920212D0CF0990D881C02D96
:10AF2000DACFDF91CF911F910F91FF90EF900895AD
:10AF30001092B61287EB92E10E94205560E070E01B
:10AF400080E992E00C9464540F931F93CF93DF93A6
:10AF5000EC0100910212109103121B870A875D8792
:10AF60004C873F872E878091B612882379F080E93D
:10AF700092E09093031280930212CE0102960E94F7
:10AF8000B656109303120093021202C07D836C83A5
:10AF9000BE0187EB92E10E946955BE0187EB92E109
:10AFA000DF91CF911F910F910C9484550F931F93B4
:10AFB000CF93DF93EC018091B612882391F000913A
:10AFC00002121091031280E992E090930312809391
:10AFD0000212CE0102960E94C056109303120093F3
:10AFE0000212BE0187EB92E10E946955BE0187EB18
:10AFF00092E1DF91CF911F910F910C9484550F93A3
:10B000001F93CF93DF93EC018091B612882391F0C8
:10B01000009102121091031280E992E090930312C2
:10B0200080930212CE0102960E94CA561093031218
:10B0300000930212BE0187EB92E10E946955BE01A6
:10B0400087EB92E1DF91CF911F910F910C94845582
:10B05000CF93DF93EC018091B612882329F0CE01C3
:10B0600002960E940D5704C01F821E821986188600
:10B07000BE0187EB92E1DF91CF910C946955CF939C
:10B08000DF93EC018091B612882331F0CE01029655
:10B09000DF91CF910C94DD5687EB92E10E9424550D
:10B0A000009739F08C179D0739F0FC018081918160
:10B0B000F7CF81E090E002C080E090E0DF91CF9197
:10B0C00008952F923F924F925F926F927F928F924C
:10B0D0009F92AF92BF92CF92DF92EF92FF920F9327
:10B0E0001F93CF93DF93CDB7DEB7E8970FB6F894F1
:10B0F000DEBF0FBECDBFE9EEFAE220813181428191
:10B100005381E5EEFAE25080418032802380E1EE07
:10B11000FAE28081898391819A83A281AB836380E3
:10B12000EDEDFAE2B081BC8381818D8392819E83B3
:10B13000A381AF83E9EDFAE2B081B8878181898785
:10B1400092819A87A381AB87E5EDFAE2B081BC8753
:10B1500081818D8792819E87A381AF87E1EDFAE29D
:10B16000B081B88B8181898B92819A8BA381AB8BC3
:10B17000EDECFAE2B081BC8B81818D8B92819E8B4C
:10B18000A381AF8BE9ECFAE2B081B88F8181898F1E
:10B1900092819A8FA381AB8FE5ECFAE2B081BC8FEC
:10B1A00081818D8F92819E8FA381AF8FE1ECFAE236
:10B1B000B081B8A3818189A392819AA3A381ABA313
:10B1C000EDEBFAE2B081BCA381818DA392819EA3B5
:10B1D000A381AFA3E9EBFAE2B081B8A7818189A787
:10B1E00092819AA7A381ABA7E5EBFAE2B081BCA755
:10B1F00081818DA792819EA7A381AFA7E1EBFAE29F
:10B20000B081B8AB818189AB92819AAB7380EDEA52
:10B21000FAE2B080A18092808380E9EAFAE2F080CD
:10B22000E180D280C380E5EAFAE2A081AFABB181D0
:10B23000B8AF128103812BAB3CAB4DAB5EAB0E9430
:10B2400006655EA95F934DA94F933CA93F932BA937
:10B250002F932F923F924F925F926F922B812F9359
:10B260002A812F9329812F932F812F932E812F9322
:10B270002D812F932C812F932B852F932A852F930C
:10B2800029852F9328852F932F852F932E852F93F4
:10B290002D852F932C852F932B892F932A892F93DC
:10B2A00029892F9328892F932F892F932E892F93C4
:10B2B0002D892F932C892F932B8D2F932A8D2F93AC
:10B2C000298D2F93288D2F932F8D2F932E8D2F9394
:10B2D0002D8D2F932C8D2F932BA12F932AA12F935C
:10B2E00029A12F9328A12F932FA12F932EA12F9324
:10B2F0002DA12F932CA12F932BA52F932AA52F930C
:10B3000029A52F9328A52F932FA52F932EA52F93F3
:10B310002DA52F932CA52F937F922AA92F9329A98E
:10B320002F9328A92F938F929F92AF92BF92CF9283
:10B33000DF92EF92FF920F931F9328AD2F932FA9C7
:10B340002F939F938F937F936F93A3EBB8E28C918E
:10B350001F928F93E2EBF8E280811F928F9385E535
:10B360009FE09F938F930E94B192E9E1FBE22081DD
:10B37000318142815381E5E1FBE25080418032809E
:10B380002380E9E0FBE29080818072806380E5E0C9
:10B39000FBE28081898391819A83A281AB83B3810F
:10B3A000BC83E1E0FBE280818D8391819E83A28159
:10B3B000AF83B381B887EDEFFAE28081898791810D
:10B3C0009A87A281AB87B381BC87E9EFFAE28081DB
:10B3D0008D8791819E87A281AF87B381B88BE5EF7E
:10B3E000FAE28081898B91819A8BB280A380E1EF10
:10B3F000FAE2F080E180D280C380EDEEFAE2A08133
:10B40000AB8BB181BC8B128103810FB6F894DEBF88
:10B410000FBECDBF2BAB3CAB4DAB5EAB0E94066508
:10B420005EA95F934DA94F933CA93F932BA92F93FE
:10B430002F923F924F925F926F927F928F929F9244
:10B440002C812F932B812F932A812F9329812F9346
:10B4500028852F932F812F932E812F932D812F932A
:10B460002C852F932B852F932A852F9329852F9316
:10B4700028892F932F852F932E852F932D852F93FA
:10B48000AF92BF922A892F9329892F93CF92DF926F
:10B49000EF92FF920F931F932C892F932B892F9359
:10B4A0009F938F937F936F93A3EBB8E28C911F923E
:10B4B0008F93E2EBF8E280811F928F9386EE9EE0FD
:10B4C0009F938F930E94B1920FB6F894DEBF0FBE88
:10B4D000CDBFE8960FB6F894DEBF0FBECDBFDF91AB
:10B4E000CF911F910F91FF90EF90DF90CF90BF9081
:10B4F000AF909F908F907F906F905F904F903F9014
:10B500002F90089580E380936D130895CF93DF9378
:10B5100060916D1370E0C0E3D0E0C61BD70B65549B
:10B520007D4EAE010E94EA91CE01DF91CF91089548
:10B53000CF92DF92EF92FF920F931F93CF93DF93FF
:10B540007C01C0907013D090711360916D1370E006
:10B55000E601E096C61BD70BC138D105D8F400E34D
:10B5600010E0061B170B65547D4EA8010E94EA915E
:10B570006091B9127091BA1280916E1390916F130D
:10B58000680F791FA601C701800F911F0E94EA91E1
:10B59000CE0102C080E090E0DF91CF911F910F912A
:10B5A000FF90EF90DF90CF90089590916D13980FDA
:10B5B00090936D1308954091701350917113481733
:10B5C000590798F020916E1330916F13280F391F8F
:10B5D00030936F1320936E13481B590B50937113C4
:10B5E0004093701381E090E0089580E090E008952A
:10B5F0009093711380937013089580916E139091BE
:10B600006F1385519D4E089580916D1390E0855480
:10B610009D4E089581E090E02091B9123091BA12C8
:10B620002B5E324111F480E090E008950E940A5BA5
:10B63000892B61F06091B9127091BA124091701328
:10B64000509171138BEE92E10C94EA9120916E135C
:10B6500030916F1321153105B9F0809170139091DD
:10B660007113C096EBEEF2E1AF014B5B524148170C
:10B67000590734F4DF01A20FB31F4C914193F4CF6B
:10B6800010926F1310926E1308958091B9129091D9
:10B69000BA1208958091701390917113089590914A
:10B6A0006D1380E3891B089520E380916D13281B9F
:10B6B0008091701390917113820F911D08951F93C3
:10B6C000CF93DF93EC0110916D13812F90E08C17D5
:10B6D0009D076CF00E94545B8C0F9D1F8138910573
:10B6E00030F41C1B10936D1381E090E002C080E0E9
:10B6F00090E0DF91CF911F910895CF93DF93ECEB12
:10B70000F8E21192119288E2EC3EF807D1F7C4EB0F
:10B71000D8E260E073E0CE010E941052229688E2E7
:10B72000CC3BD807B1F7DF91CF91089510926F13FA
:10B7300010926E13109271131092701380E3809325
:10B740006D138BEE92E19093BA128093B9120C9420
:10B750007D5BEF92FF920F931F93CF93DF9300D007
:10B76000CDB7DEB78C0169837A830E94965B6981CD
:10B77000E62E7A81F72E81E8E816F10418F080E8C9
:10B78000E82EF12CA701B8018091B9129091BA125C
:10B790000E94EA91F0927113E0927013C7010F902A
:10B7A0000F90DF91CF911F910F91FF90EF9008952F
:10B7B0000F931F93CF93DF938C01EB010E94965B55
:10B7C0001093BA120093B912D0937113C0937013EF
:10B7D000DF91CF911F910F91089520E3ECEBF8E2F8
:10B7E000DC0101900D922A95E1F788E0E4EBF8E2A4
:10B7F000DB0101900D928A95E1F7089520E3FC01A9
:10B80000ACEBB8E201900D922A95E1F788E0FB01DC
:10B81000A4EBB8E201900D928A95E1F70895E82F24
:10B82000F0E0EE0FFF1FE454F74D7183608381E079
:10B8300090E00895E82FF0E0EE0FFF1FE454F74D7D
:10B8400080819181089590E0880F991F8C57974DC2
:10B850000E94105281E090E0089590E0880F991FB7
:10B860008C57974D08958115910511F00197F1F7C7
:10B870000895E091EF28F091F02890818091EE28D2
:10B8800089230895E091EC28F091ED288081909132
:10B89000EE28892B8083E091F128F091F2288081B5
:10B8A0009091EE28892B80830895E091EC28F09107
:10B8B000ED2890818091EE28809589238083E09106
:10B8C000F128F091F22890818091EE2880958923CB
:10B8D000808308951F93CF93DF93E091EC28F0913C
:10B8E000ED2890818091EE28809589238083E091D6
:10B8F000F128F091F22880819091EE28892B8083A5
:10B900008FEB93E00E94335C1FB7F894E091F1282D
:10B91000F091F22890818091EE2880958923808390
:10B9200083E890E00E94335CE091EF28F091F028EA
:10B93000D081C091EE281FBF78948BE393E00E94E2
:10B94000335CE091EF28F091F02890818091EE280F
:10B95000982319F08D2F8C2301C081E0DF91CF91C6
:10B960001F9108955093F2284093F1287093ED2889
:10B970006093EC289093F0288093EF2881E001C039
:10B98000880F2A95EAF78093EE280C946A5CCF938F
:10B99000DF93C82FDFB7F894E091F128F091F228F7
:10B9A00080819091EE28892B808383E090E00E9433
:10B9B000335CCC2351F0E091F128F091F2288081A2
:10B9C0009091EE2890959823908387E190E00E94D3
:10B9D000335CE091EF28F091F02880819091EE287F
:10B9E000892309F4C0E089E590E00E94335CE0918E
:10B9F000F128F091F22880819091EE28909598237B
:10BA00009083DFBF8BE390E00E94335C8C2FDF914B
:10BA1000CF910895CF93DF93C82FD8E08C2F8170FA
:10BA20000E94C75CC6958111C068D150B9F78C2FB0
:10BA3000DF91CF9108958FEF0C940A5DDF92EF9222
:10BA4000FF920F931F93CF93DF93E82EEB010E9499
:10BA50006A5C81112FC080EF0E940A5DF12C10E416
:10BA600088EFD82ED10E81E00E94C75C082F81E0BC
:10BA70000E94C75C882319F0002361F01DC00111EA
:10BA800009C01E1528F0888180FF04C0E11611F05E
:10BA9000F12E01E0802F0E94C75C988196950111DC
:10BAA0009068988311501D11DECF21961111D8CFC7
:10BAB0008F2D03C08FEF01C08EEFDF91CF911F91CB
:10BAC0000F91FF90EF90DF900895FF920F931F93D7
:10BAD000CF93DF93F82EEB010E946A5C209769F008
:10BAE00085E50E940A5D8E01085F1F4F89910E94C3
:10BAF0000A5DC017D107D1F703C08CEC0E940A5D24
:10BB00008F2DDF91CF911F910F91FF900C940A5DC3
:10BB10000F931F93CF93DF93DB01EC9111969C91D0
:10BB20001197F0E0F92B803181F4BF016E7FE3E0E3
:10BB3000660F771FEA95E1F716969C911697ECE051
:10BB4000F0E0E91BF109E60FF71FF7FF07C091E0EE
:10BB5000EA019883F195E195F10902C0EA011882A2
:10BB6000883279F414968C91982F9076903649F01B
:10BB700086FF02C0EE7F05C085FF02C0EC7F01C0DA
:10BB8000E87FCF0144E0969587954A95E1F7D90182
:10BB90008C93EF70E801E88380E0DF91CF911F91F3
:10BBA0000F9108950F931F93CF93DF93EC018B01B7
:10BBB000B80188810E941E5D888381508D3F30F4DA
:10BBC000F8018081883211F0803191F7DF91CF91B7
:10BBD0001F910F910895CF93DF93EC010E946A5C4F
:10BBE000BE0184EB0E94655D81E00E94C75CC82FA6
:10BBF0000E946A5C81E0C11101C080E0DF91CF91B9
:10BC000008951F93CF93DF9300D0CDB7DEB7182FE1
:10BC100069837A830E946A5C0E94395C69817A81B7
:10BC2000882341F084E40E94655D113029F00E9470
:10BC3000425C02C082E001C080E00F900F90DF9173
:10BC4000CF911F9108954F925F926F927F928F9242
:10BC50009F92AF92BF92CF92DF92EF92FF920F939B
:10BC60001F93CF93DF93CDB7DEB729970FB6F89424
:10BC7000DEBF0FBECDBF6C015B014A0189010E948E
:10BC80006A5CB6018EEB0E94655DCE0101967C0177
:10BC90003E019AE0690E711C27010E941B5DF701AD
:10BCA00081937F01E615F705C1F769E070E0C201F5
:10BCB0000E94C077811109C09401A501B201F6016B
:10BCC00080810E94885D80E001C083E029960FB6E4
:10BCD000F894DEBF0FBECDBFDF91CF911F910F91C2
:10BCE000FF90EF90DF90CF90BF90AF909F908F909C
:10BCF0007F906F905F904F9008955F926F927F92C8
:10BD00008F929F92AF92BF92CF92DF92EF92FF926B
:10BD10000F931F93CF93DF93CDB7DEB729970FB65D
:10BD2000F894DEBF0FBECDBF582E6B015A018901BA
:10BD300060E070E08EEB0E94655DCE0101967C01B3
:10BD40004E019AE0890E911C37010E941B5DF7019C
:10BD500081937F01E815F905C1F769E070E0C3013F
:10BD60000E94C077811108C09501A601B301852DFD
:10BD70000E94885D80E001C083E029960FB6F894A8
:10BD8000DEBF0FBECDBFDF91CF911F910F91FF900E
:10BD9000EF90DF90CF90BF90AF909F908F907F906B
:10BDA0006F905F9008950F931F93CF93DF93CDB75C
:10BDB000DEB728970FB6F894DEBF0FBECDBF182FA1
:10BDC000062F98E0ECE0F3E0DE01119601900D9271
:10BDD0009A95E1F7242F332727FD309541E752E06C
:10BDE000249FC001259F900D349F900D112464E67F
:10BDF00070E00E94058CCB0144E6049F800D911DEC
:10BE00001124FE013196AE01475F5F4F619170E0F2
:10BE10002617370711F4019603C0E417F507B1F7A9
:10BE2000112319F091958195910928960FB6F894F0
:10BE3000DEBF0FBECDBFDF91CF911F910F9108954F
:10BE4000EF92FF920F931F93CF93DF93CDB7DEB79F
:10BE50002B970FB6F894DEBF0FBECDBFF82EE92E9C
:10BE6000682F792F88E08F0D0E94015E882319F0DA
:10BE700084E391E243C066E471E48FE090E00E94C5
:10BE80008B5F8E01075F1F4F9801AE01465F5F4FCA
:10BE9000BE01655F7F4F8F2D9E2D0E94235E811115
:10BEA000E7CF88E0ECE0F3E0DE01119601900D921F
:10BEB0008A95E1F7498521E732E0429FC001439F1F
:10BEC000900D112464E670E00E94058C8A8594E64A
:10BED000899F600D711D1124FE01319681914813D7
:10BEE00003C06F5F7F4F03C0E017F107B9F78B8581
:10BEF000882319F0719561957109CB012B960FB6C6
:10BF0000F894DEBF0FBECDBFDF91CF911F910F918F
:10BF1000FF90EF900895DC01CB0181159105A105FB
:10BF2000B10529F081509040A040B040D9F7089564
:10BF30009B01AC011092B90060E072E18AE790E0E9
:10BF40000E94198C20513109410951095695479594
:10BF5000379527952093B800089594EA9093BC00F4
:10BF600040EA56E861E070E09091BC0097FD0BC09C
:10BF7000415051096109710941155105610571056A
:10BF800099F781E008959091B900987F983011F069
:10BF90009031B9F78093BB0084E88093BC0080EABD
:10BFA00096E8A1E0B0E02091BC0027FD08C0019711
:10BFB000A109B1090097A105B105A9F7E2CF8091C8
:10BFC000B900887F883111F08034D9F680E0089577
:10BFD00024EA34E844E92093BC009091BC0097FF28
:10BFE000FCCF9091B900987F983011F0903199F77B
:10BFF0008093BB003093BC009091BC0097FFFCCFB6
:10C000009091B900987F903211F0983539F44093AF
:10C01000BC009091BC0094FDFCCFDDCF08950C9442
:10C02000AD5F84E98093BC008091BC0084FDFCCFAF
:10C0300008958093BB0084E88093BC008091BC008D
:10C0400087FFFCCF9091B900987F81E0983209F486
:10C0500080E0089584EC8093BC008091BC0087FF51
:10C06000FCCF8091BB00089584E88093BC00809150
:10C07000BC0087FFFCCF8091BB000895E0E1DC01AC
:10C08000FD91CD01F0933F01E150C9F780913C0152
:10C090008F7D80933C0180913C01877F80933C01A0
:10C0A000FB0180E1919190933E018150D9F78091FD
:10C0B0003C01806880933C0180913D0180FFFCCF72
:10C0C0004051510980913C01806280933C018091F4
:10C0D0003C01877F80933C01141615069CF4FB01FC
:10C0E00080E1919190933E018150D9F780913C017C
:10C0F000806880933C0180913D0180FFFCCF4051DE
:10C100005109EACFF90180E190913E01919381506C
:10C11000D9F781E090E008950F931F93CF93DF93B9
:10C12000EC018CE70E94E85F8CE70E9419608E01A9
:10C13000005F1F4F89910E941960C017D107D1F786
:10C14000DF91CF911F910F910C941160813019F400
:10C1500040E050E002C040EC50E060E070E08CE76E
:10C1600090E00C946D11813019F44EE050E002C063
:10C1700048E050E060E070E08CE790E00C946D11D6
:10C1800041E050E060E070E08CE790E00E946D11CB
:10C190006AE67AE080E090E00C948B5F48E350E040
:10C1A00060E070E08CE790E00E946D1149E350E0A0
:10C1B00060E070E08CE790E00E946D1144E150E097
:10C1C00060E070E08CE790E00E946D1148E750E07D
:10C1D00060E070E08CE790E00E946D114EE550E069
:10C1E00060E070E08CE790E00E946D114DE650E059
:10C1F00060E070E08CE790E00E946D116CE17AE104
:10C2000086E090E00E948B5F4CE050E060E070E0E0
:10C210008CE790E00E946D1141E050E060E070E03A
:10C220008CE790E00E946D1146E050E060E070E025
:10C230008CE790E00E946D116AE67AE080E090E081
:10C240000C948B5FCF93DF93CDB7DEB7A2970FB679
:10C25000F894DEBF0FBECDBF81E1E0E4F9E0DE017E
:10C26000529601900D928A95E1F781E1E1E5F9E0BE
:10C27000DE01119601900D928A95E1F70E94CE6041
:10C28000CE0142960E948C6082E00E94A6606AE61F
:10C290007AE080E090E00E948B5FCE0101960E94E0
:10C2A0008C6060E17EEA88E290E00E948B5F80E033
:10C2B0000E94B36060E17EEA88E290E00E948B5FBA
:10C2C0004EE050E060E070E08CE790E00E946D117D
:10C2D000A2960FB6F894DEBF0FBECDBFDF91CF910F
:10C2E0000895CF92DF92EF92FF920F931F93CF9317
:10C2F000DF9300D01F92CDB7DEB7F82E042F122F98
:10C30000213031F0223031F0243031F0283031F05A
:10C3100090E005C091E003C092E001C093E00C30D2
:10C3200059F00E3011F4946007C0003111F4986098
:10C3300003C0023109F49C60613059F0623011F49D
:10C34000906207C0633011F4906403C0643009F454
:10C3500090669068692F70E023E030E0AE014F5F97
:10C360005F4F8F2D90E00E94841169E07AE180E0B8
:10C3700090E00E948B5F8F2D8160F82E0E94AD5F50
:10C380000E942A6089830E942A608A83023119F4FC
:10C390000E942A608B830E942A6087FDF1CF0E9451
:10C3A00034600E94116069E07AE180E090E00E94D0
:10C3B0008B5F8F2D0E94AD5F0E942A6089830E944F
:10C3C0002A608A83023119F40E9434608B830E94B0
:10C3D00034600E94116039812A81023149F5832F2E
:10C3E00090E0A0E0B0E04B817727662731FF0EC0D8
:10C3F00030E0322F2227620F731F811D911D640FC1
:10C40000711D811D911D8C6F9F6F0BC030E0322F0D
:10C410002227620F731F811D911D640F711D811DE5
:10C42000911D0E940E8920E83FEF4FEF57E420C096
:10C43000632F70E0762F6627620F711D882777FDC6
:10C440008095982F0E940E890C3029F420E030EE60
:10C450004FEF54E40DC00E3029F420E038EF4FEFD9
:10C4600055E406C0003131F420E03EEF4FEF56E4D2
:10C470000E946F882FE632E143E050E40E94F08A88
:10C480006B017C01612F70E080E090E00E940E89DA
:10C490009B01AC01C701B6010E946F880F900F90FD
:10C4A0000F90DF91CF911F910F91FF90EF90DF9050
:10C4B000CF900895E6E4F1E0808120819081308181
:10C4C000829586958695837022952F70822B832B7B
:10C4D00092959F70892B08950F931F93CF93DF93AD
:10C4E00000D0CDB7DEB746E06CE080E00E949C65EE
:10C4F00089E18093C4001092C50082E08093C0005F
:10C5000080E00E9427660E94C86484B784B784B71D
:10C5100084B784B7E3E7F1E322E432E43183208394
:10C520003A968DB79EB70A97E817F907B8F382E6EF
:10C5300099E09F938F9382EA90E19F938F930E945B
:10C54000B1920E9403740E94BC5360E070E086E8E0
:10C5500092E00E9464540E949857E0911403F09175
:10C56000150309950E945A6290E00E943F74CE0123
:10C5700001960E94FD630F900F900F900F908823FB
:10C5800041F082E890E19F938F930E94B1920F90C7
:10C590000F90CE0101960E942B520E940B648C01D9
:10C5A0000E940764AE014F5F5F4FB8010E94F368BD
:10C5B0000E9477630E94D4680E940F640E942D6AD3
:10C5C00085E790E19F938F930E94B1928A811F9299
:10C5D0008F9301E710E11F930F930E94B19289811D
:10C5E0001F928F931F930F930E94B1928FE690E159
:10C5F0009F938F930E94B1920E944374E0915103E4
:10C60000F09152030995E0914303F0914403099599
:10C61000E0912A03F0912B0309950E94346A182FA8
:10C620000E94D1681F921F931F928F938091500395
:10C630008F9380914F038F93809142038F938091CA
:10C6400041038F9384E590E19F938F930E94B19271
:10C65000E0915B03F0915C030FB6F894DEBF0FBE70
:10C66000CDBF309791F00995BC0180E890E00E9421
:10C67000F18B7F936F9381E490E19F938F930E945E
:10C68000B1920F900F900F900F908FE390E19F93D6
:10C690008F930E94B19260E070E08CED92E00E9476
:10C6A000645480EF92E00E94137387E390E19F93BC
:10C6B0008F930E94B1920F900F900F900F900F9058
:10C6C0000F90DF91CF911F910F9108957F936F93FA
:10C6D0009F938F9381E390E19F938F930E94B192F8
:10C6E0000F900F900F900F900F900F9008951F9341
:10C6F000CF93DF93CDB7DEB7A0970FB6F894DEBF28
:10C700000FBECDBF8DE590E00E941D94182F282FFD
:10C7100035EF380F303108F0982F9095291709F42C
:10C7200061C08DEB90E19F938F930E94B192E2E004
:10C73000F1E10F900F90DE01119684918D93319667
:10C7400081E1EA30F807C9F7F89448E050E069E77A
:10C7500070E0CE0101960E942394E4EFF0E1DE0147
:10C76000119684918D93319681E1E230F807C9F7F3
:10C770004EE050E06BE670E0CE0101960E942394FB
:10C78000EAEEF0E1DE01119684918D93319680E11D
:10C79000E43FF807C9F74AE050E061E670E0CE01F7
:10C7A00001960E9423946DEC7BEA8BE590E00E9459
:10C7B0003B9460E070E089E590E00E943B9460E08B
:10C7C00088E590E00E942D9460E070E08FE590E0B5
:10C7D0000E943B941AE16AE175EE8DE590E00E94BB
:10C7E0003B947894812FA0960FB6F894DEBF0FBECD
:10C7F000CDBFDF91CF911F910895F89442E050E0B2
:10C8000069E770E00E940594789480E008958BE5D4
:10C8100090E00C941D9489E590E00C941D9488E5BB
:10C8200090E00C9415944091012950910229609157
:10C8300003297091042990E0A0E0B0E0480F591F4F
:10C840006A1F7B1F4093012950930229609303299B
:10C85000709304294091FD285091FE286091FF2893
:10C8600070910029480F591F6A1F7B1F4093FD28B4
:10C870005093FE286093FF28709300292091A12AED
:10C880002223A1F04091F9285091FA286091FB28C9
:10C890007091FC28480F591F6A1F7B1F4093F9288D
:10C8A0005093FA286093FB287093FC2808951F92F8
:10C8B0000F920FB60F9211240BB60F922F933F9346
:10C8C0004F935F936F937F938F939F93AF93BF9398
:10C8D000EF93FF9380917413909175130196909349
:10C8E000751380937413809173138F5F8093731308
:10C8F0008038A9F410927313809101299091022934
:10C90000A0910329B09104290196A11DB11D809326
:10C91000012990930229A0930329B09304298091BF
:10C92000A12A8823E1F0809172138F5F80937213A4
:10C930008038A9F4109272138091F9289091FA2806
:10C94000A091FB28B091FC280196A11DB11D8093F8
:10C95000F9289093FA28A093FB28B093FC280E9412
:10C96000F456892B11F00E940756FF91EF91BF9169
:10C97000AF919F918F917F916F915F914F913F9177
:10C980002F910F900BBE0F900FBE0F901F90189518
:10C99000F8941092B60016BC83EF87BD82E084BD88
:10C9A00094E095BD95B395BB80936E0078940895FF
:10C9B00080917413909175132091741330917513B5
:10C9C00082179307A9F70895009751F022E330E00A
:10C9D00000002150310921153105D1F70197F4CF1D
:10C9E00008950F931F93CF93DF93EC010E94D864B7
:10C9F0008C010E94D864801B910B8C179D07C8F393
:10CA0000DF91CF911F910F91089508950F931F9378
:10CA10006091012970910229809103299091042944
:10CA200000910129109102292091032930910429B4
:10CA3000601771078207930759F71F910F910895A7
:10CA40001F920F920FB60F9211241092B2020F9004
:10CA50000FBE0F901F9018951F920F920FB60F9256
:10CA600011240BB60F922F933F934F935F936F93C5
:10CA70007F938F939F93AF93BF93EF93FF93E09137
:10CA8000A802F091A9028081E091B302F091B40272
:10CA9000309709F00995FF91EF91BF91AF919F9168
:10CAA0008F917F916F915F914F913F912F910F9057
:10CAB0000BBE0F900FBE0F901F9018951F920F92F4
:10CAC0000FB60F9211241092BF020F900FBE0F905D
:10CAD0001F9018951F920F920FB60F9211240BB64C
:10CAE0000F922F933F934F935F936F937F938F9307
:10CAF0009F93AF93BF93EF93FF93E091B502F091B3
:10CB0000B6028081E091C002F091C102309709F035
:10CB10000995FF91EF91BF91AF919F918F917F9177
:10CB20006F915F914F913F912F910F900BBE0F909E
:10CB30000FBE0F901F9018959DE0899FF001112462
:10CB4000E855FD4FA281B3811C92A481B5816C93FD
:10CB5000A681B78188ED8C93A085B1854C93128610
:10CB60001486138608959DE0899FF0011124E855ED
:10CB7000FD4F81E08287A081B1816C933A968081DC
:10CB80008111FDCF08951F93CF93DF93182FEB01F1
:10CB9000FE016491662329F0812F0E94B3652196DE
:10CBA000F7CFDF91CF911F9108951F93CF93DF931C
:10CBB000182FEB018881882369F08A3021F46DE019
:10CBC000812F0E94B36569916D30A1F3812F0E947E
:10CBD000B365F0CFDF91CF911F910895CF93DF938D
:10CBE000CDB7DEB79E01285F3F4F4E815F8160E485
:10CBF00070E086E793E10E946E9366E773E18D81B2
:10CC00000E94D565DF91CF910895CF93C82F8A30C8
:10CC100031F46DE08091B6130E94B36502C08D308F
:10CC200029F06C2F8091B6130E94B36580E090E0EC
:10CC3000CF9108959DE0899FF0011124E855FD4FA3
:10CC4000748763870895682F80E00C94B3658093A0
:10CC5000B6138AE992E090936E3180936D31089516
:10CC600084B7877F84BF88E10FB6F8948093600013
:10CC7000109260000FBE08952FE088E190E00FB69B
:10CC8000F894A895809360000FBE209360000895EB
:10CC9000A895089588E10FB6F894809360001092EB
:10CCA00060000FBE0895F89428E088E190E00FB688
:10CCB000F894A895809360000FBE20936000FFCF8A
:10CCC00080910C2980910C2990E0089540E06FE15B
:10CCD00081E491E00C94C96BE9E3F1E0808180810B
:10CCE0008D7F80838DE090E00197F1F723E040E0B5
:10CCF0006FE182E491E00E94D36B83E090E00197C2
:10CD0000F1F708959091390191FD0AC0282F8031E3
:10CD100008F02FE040E06FE085E491E00C94D36BE5
:10CD200008958091390181FD0EC040E06FE181E4FA
:10CD300091E00E94C96B282F2F7E81E090E0213086
:10CD400021F080E0089580E090E00895809139011D
:10CD500081FD10C040E06FE181E491E00E94C96B69
:10CD60008F3131F0982F9F7E915081E0923018F4EE
:10CD700080E0089581E008950E94A6668823E1F38B
:10CD80000895CF93DF93C82F0E94BC660E94666609
:10CD9000D82FC81789F1C83019F40E946C6625C0D5
:10CDA000C93121F4863189F429E005C0C63169F41E
:10CDB000893159F426E040E06FE182E491E00E947D
:10CDC000D36BE3E0F0E03197F1F72C2F40E06FE117
:10CDD00082E491E00E94D36BD83019F4E9E6F1E0E7
:10CDE00002C0E3E0F0E03197F1F70E9466668C172D
:10CDF00019F083E490E002C080E490E0DF91CF91ED
:10CE000008950E94BC661092A12A0E946C668091CF
:10CE100039018260809339018091242B8823D9F1D4
:10CE200080919400909195004091352B5091362B34
:10CE300084179507A0F48091012B9091022BA0916B
:10CE4000032BB091042B8C57914EAF4FBF4F809363
:10CE5000012B9093022BA093032BB093042B2091D2
:10CE6000940030919500241B350B8091012B9091FB
:10CE7000022BA091032BB091042B820F931FA11DB5
:10CE8000B11D8093012B9093022BA093032BB093A1
:10CE9000042B1092242B8091262B8823D9F180918A
:10CEA0009400909195004091392B50913A2B841722
:10CEB0009507A0F48091092B90910A2BA0910B2B40
:10CEC000B0910C2B8C57914EAF4FBF4F8093092BD5
:10CED00090930A2BA0930B2BB0930C2B20919400D2
:10CEE00030919500241B350B8091092B90910A2BD2
:10CEF000A0910B2BB0910C2B820F931FA11DB11D84
:10CF00008093092B90930A2BA0930B2BB0930C2B9F
:10CF10001092262B08958091A12A882381F0809178
:10CF20003A14811104C00E94A666811106C081E0F6
:10CF30008093381481E090E008950E94016780E0BA
:10CF400090E00895809194009091950090933A2BF1
:10CF50008093392B21E02093262B8091390181FD8C
:10CF600008C08091390181FD1AC086E10E94C16626
:10CF700016C02093A02A80919400909195009093E0
:10CF8000362B8093352B2093242B809139018D7F74
:10CF9000809339018091A02A8111FCCFE2CF81E0FA
:10CFA0008093A12A08958091A12A81110AC08091BD
:10CFB0003A14882321F081E08093391402C00E9442
:10CFC000A26781E090E008951F93CF93DF931F92B3
:10CFD000CDB7DEB78FB7898380913A14811126C00F
:10CFE000F8948091A12A882351F08091390181FD24
:10CFF0001BC00E94A6668823B9F080E003C00E948F
:10D00000D36781E02091470191E02E3008F090E055
:10D01000192F119581110E948B67107429F0898155
:10D020008FBF81E090E004C089818FBF80E090E0F5
:10D030000F90DF91CF911F9108958091391488232B
:10D0400021F00E94A267109239148091381488232D
:10D0500021F00E9401671092381410923A1408953A
:10D060000F931F93AB0121E020933A140091E52A1E
:10D070001091E62A2091E72A3091E82A0F5F1F4F8E
:10D080002F4F3F4F0093E52A1093E62A2093E72A7B
:10D090003093E82A22E0260F27FF0CC080919E2AB9
:10D0A00090919F2A019690939F2A80939E2A0FEF3A
:10D0B0001FEF07C0BC0187EB93E10E94EA9100E0FB
:10D0C00010E00E941D68C8011F910F910895809380
:10D0D0003C1408950E946666823011F0823111F48A
:10D0E00080E0089581E0089508958FEF80934E01C8
:10D0F00022E044E060EF8CE691E00E94D36B25E0F3
:10D1000041E06EE08CE290E00E94D36B80E8809377
:10D110006F018091460180936D0121E045E060E25E
:10D1200084E491E00C94D36B8DEF93E00197F1F7D9
:10D130000E94BF6B10921529109297291092192AFC
:10D140001092142910921329E9E3F1E080818E7F77
:10D15000808380818D7F80838DE090E00197F1F75F
:10D16000E9E3F1E080818160808323E040E06FE1CA
:10D1700082E491E00E94D36B8DEF93E00197F1F789
:10D1800080915D0180915E010E94756860E070E0B1
:10D1900082EC92E00E9464540E94A26781E090E0D9
:10D1A000089580913B140895CF93DF931F92CDB7DC
:10D1B000DEB789830E94BC66898180933B14282F47
:10D1C00040E06FE188E491E00F90DF91CF910C9403
:10D1D000D36B0E94D4688091390181FD03C086E041
:10D1E0000C94C1660895FA018093620190936301E3
:10D1F00060936001709361013097C1F080818093EA
:10D200006B01818180936A018281809369018381AE
:10D210008093680184818093670185818093660192
:10D22000868180936501878180936401089582ECF3
:10D2300092E00E94855481E080930C2980910D2911
:10D2400090910E29019690930E2980930D2981E0EB
:10D2500090E008958091142992E8899FF0011124AB
:10D26000EB5EF64D10828F5F833018F480931429A3
:10D2700002C010921429E091142982E8E89FF0017D
:10D280001124EB5EF64D808181110C941769109288
:10D290000C2908951F93CF93DF932091142912E84E
:10D2A000129F90011124D901AB5EB64D4C914111F2
:10D2B00003C00E942A6993C05091390151FD8FC06B
:10D2C0005091A12A552309F48AC047FF16C00E9435
:10D2D0002A698091D52A9091D62AA091D72AB09117
:10D2E000D82A0196A11DB11D8093D52A9093D62AE4
:10D2F000A093D72AB093D82A72C04330B0F40E94CA
:10D300002A698091D12A9091D22AA091D32AB091F2
:10D31000D42A0196A11DB11D8093D12A9093D22ABF
:10D32000A093D32AB093D42A5AC050E0EA0122979E
:10D330006C177D07B0F40E942A698091CD2A9091E4
:10D34000CE2AA091CF2AB091D02A0196A11DB11D5D
:10D350008093CD2A9093CE2AA093CF2AB093D02A3F
:10D360003EC0B9016A5E764D0E94EA91E0911429AF
:10D370001E9FF0011124EB56F64D80818093052904
:10D380000E942A69809147018093062990910B2978
:10D39000992311F0891710F480930B2960910629C5
:10D3A00070E084E00E940F5C6091052970E083E0EA
:10D3B0000E940F5C4091E92A5091EA2A6091EB2A81
:10D3C0007091EC2A4F5F5F4F6F4F7F4F4093E92A78
:10D3D0005093EA2A6093EB2A7093EC2A02C0C0E0D3
:10D3E000D0E0CE01DF91CF911F910895CF93DF93CD
:10D3F000EC01888199810097E9F08730954021F010
:10D400001982188283E026C06238C1F410920C2978
:10D410000E94965B0E94FD5A60E870E00E944A6993
:10D42000181619066CF40E94F85AE0915503F09111
:10D430005603099587E095E09983888381E00AC0C7
:10D440008091092990910A29019690930A29809345
:10D450000929F0CFDF91CF91089591E090933A148C
:10D460000E9482660C941D688091390181FD06C07E
:10D4700040E06FE085E491E00C94C96B80E1089591
:10D480000F931F93CF93DF93182F21E020933A142B
:10D490000091A12A8091390181FF16C080919400EA
:10D4A000909195009093362B8093352B2093242BCD
:10D4B0002093A02A809139018D7F8093390180913A
:10D4C000A02A8111FCCF00E00E94BC668091A12AB5
:10D4D000882309F43FC08091262B8823D9F18091BD
:10D4E000940090919500E091392BF0913A2B8E1792
:10D4F0009F07A0F44091092B50910A2B60910B2BB0
:10D5000070910C2B4C57514E6F4F7F4F4093092B0E
:10D5100050930A2B60930B2B70930C2B209194004B
:10D52000309195002E1B3F0B4091092B50910A2BF7
:10D5300060910B2B70910C2B420F531F611D711DBD
:10D540004093092B50930A2B60930B2B70930C2B59
:10D550001092262B8091390181FD03C089E10E9440
:10D56000C16686E00E941A5C892B51F00E94346AE1
:10D57000C82F86E00E941A5C81500E94826602C019
:10D58000C0E0D0E020919400309195003093382B8A
:10D590002093372B81E08093252BF89480913901DB
:10D5A000826080933901809139018D7F80933901A8
:10D5B00062E0610F87EB93E10E94046C7894209104
:10D5C0009B2A30919C2A2F5F3F4F30939C2A2093B7
:10D5D0009B2A0E94BC6645E060EE82E491E00E94D6
:10D5E000C96B182F86E00E941A5C892B19F08C2FCA
:10D5F0000E948266002319F00E94A26702C00E9466
:10D6000001678091252B8823D9F180919400909116
:10D610009500E091372BF091382B8E179F07A0F4DF
:10D620004091052B5091062B6091072B7091082B90
:10D630004C57514E6F4F7F4F4093052B5093062B05
:10D640006093072B7093082B2091940030919500E4
:10D650002E1B3F0B4091052B5091062B6091072B01
:10D660007091082B420F531F611D711D4093052BB4
:10D670005093062B6093072B7093082B1092252B49
:10D680008091A12A882361F0209194003091950027
:10D6900030933A2B2093392B81E08093262B07C0BF
:10D6A00023E040E06FE182E491E00E94D36B0E94AE
:10D6B0001D681130E9F01330A9F48091DD2A9091B2
:10D6C000DE2AA091DF2AB091E02A0196A11DB11DAA
:10D6D0008093DD2A9093DE2AA093DF2AB093E02A7C
:10D6E00012E009C0153031F0173029F411E003C001
:10D6F00010E001C013E0812F90E0DF91CF911F91E6
:10D700000F910895CF93DF93EB010E94306800974B
:10D7100029F4CE010E94406A009751F020919E2A80
:10D7200030919F2A2F5F3F4F30939F2A20939E2A4C
:10D73000DF91CF910895CF93DF938091A12A81113A
:10D7400004C00E94D367D1E001C0D0E00E946666A9
:10D75000863111F0813119F4C091470109C040E0D0
:10D760006FE186E491E00E94C96BC82FCC0FC80F0F
:10D77000D1110E948B678C2FDF91CF910895109269
:10D780003E1410923D14EFE6F0E0808180628083C9
:10D790000895FC018081862390E002C095958795CD
:10D7A0004A95E2F70895F894FC015081362F3095A0
:10D7B0005323042E01C0220F0A94EAF72623522B8A
:10D7C00050837894089540917B01FC014193A0E837
:10D7D000B1E050E8540F9D012F5F3F4F6C91619372
:10D7E000521711F0D901F7CF4150E42FF0E0E05883
:10D7F000FE4F2181FC01E058FF4F2083FC01EF57D1
:10D80000FF4F21E02083089560938001E1E8F1E07B
:10D8100061589F012F5F3F4FDC014D91CD01408347
:10D82000621711F0F901F5CF08951F920F920FB60C
:10D830000F9211240BB60F922F933F934F935F9348
:10D840006F937F938F939F93AF93BF93EF93FF93C8
:10D8500080914701809306298091132922E8829FB5
:10D86000C00111248B5E964D0E94E36B80911329B9
:10D870008F5F833018F48093132902C0109213290C
:10D880000E941769FF91EF91BF91AF919F918F9186
:10D890007F916F915F914F913F912F910F900BBEB0
:10D8A0000F900FBE0F901F9018951F920F920FB6FA
:10D8B0000F9211240F900FBE0F901F9018951F927A
:10D8C0000F920FB60F9211240F900FBE0F901F9062
:10D8D00018951F920F920FB60F9211240F900FBE42
:10D8E0000F901F9018951F920F920FB60F92112450
:10D8F0001092A02A0F900FBE0F901F9018951F92A4
:10D900000F920FB60F9211241092A02A0F900FBE03
:10D910000F901F9018951F920F920FB60F9211241F
:10D920008F9381E080930C298F910F900FBE0F9001
:10D930001F9018951F920F920FB60F9211241092FC
:10D94000A02A0F900FBE0F901F9018951F920F9254
:10D950000FB60F9211248F939F9380913D14909155
:10D960003E14019690933E1480933D149F918F91A5
:10D970000F900FBE0F901F901895CF92DF92EF92ED
:10D98000FF920F931F93CF93DF937C018B016A016A
:10D990008FE394E10E942455EC01009751F0EC8153
:10D9A000FD81309711F0C8010995CE010E94CC5538
:10D9B000F3CFA601B801C701DF91CF911F910F915D
:10D9C000FF90EF90DF90CF900C94AE520F931F9387
:10D9D000CF93DF9300D0CDB7DEB78091A92A909185
:10D9E000AA2AA091AB2AB091AC2A0196A11DB11D23
:10D9F0008093A92A9093AA2AA093AB2AB093AC2A29
:10DA00000E94506F8C018FE394E10E94245500978F
:10DA100079F0DC011296ED91FC911397309729F083
:10DA200089839A8309959A8189810E94CC55EFCF89
:10DA30000115110549F0C8010F900F90DF91CF91AA
:10DA40001F910F910C94A5520F900F90DF91CF91E1
:10DA50001F910F9108950E9443740E94965B0E944B
:10DA6000776D81E493E09093A42A8093A32A0E9487
:10DA70004E6F2FEF31E040E05EE160E074E082E065
:10DA800090E00C94176FBC018FE394E10C948455E3
:10DA9000BC018FE394E10C946955CF93DF93EC01C3
:10DAA0004091A52A5091A62A6091A72A7091A82A90
:10DAB0004F5F5F4F6F4F7F4F4093A52A5093A62A29
:10DAC0006093A72A7093A82A0E94636F009761F061
:10DAD0000E94165BE0914503F0914603BE018DEB79
:10DAE0009CE6099581E090E0DF91CF91089585E46F
:10DAF00094E10C9420550F93CF93DF93EC017B833B
:10DB00006A8318865F834E83BC0185E494E10E949A
:10DB10008455E0914114F0914214309749F04C81C2
:10DB20005D8101E020E030E068858A819B81099574
:10DB3000DF91CF910F910895BC0185E494E10C949D
:10DB400069550F93DC0118961C921897E0914114C7
:10DB5000F0914214309759F000E020E030E040E0CE
:10DB600050E060E012968D919C91139709950F916A
:10DB700008950F93DC01AB0114962D913C911597FC
:10DB800081E018968C93189715967C936E93149752
:10DB9000E0914114F0914214309739F000E061E0D7
:10DBA00012968D919C91139709950F9108950F935B
:10DBB000DC01E0914114F0914214309771F0149619
:10DBC0004D915C91159701E09A0118966C91189708
:10DBD00012968D919C91139709950F910895E0915C
:10DBE0004314F0914414309709F0099408959093E8
:10DBF00044148093431408959093421480934114E5
:10DC0000089585E494E10C942455EF92FF920F93CC
:10DC10001F93CF93DF938C01EB017A0185E494E1AC
:10DC20000E9424550097D9F0DC0112962D913C9169
:10DC300013972C173D0781F41696ED91FC911797D9
:10DC4000309769F09701AE01B801DF91CF911F9134
:10DC50000F91FF90EF9009940E94CC55E3CFDF9194
:10DC6000CF911F910F91FF90EF9008950895CF935A
:10DC7000DF93C8E7D4E16881798120E030E046E5B0
:10DC80005EE682E694E10E94A4570E944174688196
:10DC900079810E94F18B20E030E04AE65EE6BC012B
:10DCA00082E594E1DF91CF910C94A4578091781490
:10DCB000909179142091761430917714880F991FE0
:10DCC0002817390708F4C9019093791480937814C0
:10DCD0000C94376ECF93DF930E94965B0E94FD5A9F
:10DCE000EC01198218820E94016E28813981009707
:10DCF00019F1FC0140854423F9F0FC014281538174
:10DD0000F901EE0FFF1FEE0FFF1FEC0FFD1F5383F6
:10DD10004283FC01448155812F5F3F4FF901EE0F93
:10DD2000FF1FEE0FFF1FEC0FFD1F51834083398350
:10DD300028830E94CC55D9CFC901880F991F880F1D
:10DD4000991F02960E94F85A88819981892B31F097
:10DD500087E494E1DF91CF910C947C52DF91CF91D5
:10DD60000895AF92BF92CF92DF92EF92FF920F93FE
:10DD70001F93CF93DF9300D0CDB7DEB76B010E9426
:10DD8000FD5AFC01008111811A8309830C301105B1
:10DD900018F4E12CF12C0DC01F930F9380E899E04B
:10DDA0009F938F930E949F920F900F900F900F90D0
:10DDB00021C0E016F106F1F00E94FD5AF701EE0FC6
:10DDC000FF1FEE0FFF1FE80FF91FA280B3800E9414
:10DDD000FD5AFFEFEF1AFF0AF701EE0FFF1FEE0FDC
:10DDE000FF1FE80FF91F40815181B501C6010E9454
:10DDF000056EDFCF0F900F90DF91CF911F910F91A4
:10DE0000FF90EF90DF90CF90BF90AF9008950F9369
:10DE1000013059F480917214909173149093791495
:10DE2000809378140F910C94376E0F910895EF92B0
:10DE3000FF920F931F93CF93DF938B01EA01790138
:10DE40004EE253E0BC0187E494E10E9460521093DB
:10DE5000731400937214D0937514C0937414F092D9
:10DE60007714E092761487E09FE6DF91CF911F91BF
:10DE70000F91FF90EF900C94FC6D82E694E10E946C
:10DE8000285882E594E10E94285887E494E10C9494
:10DE90007A52809178149091791408950C94BA5222
:10DEA000CF93DF93E0913203F09133030995EC01B6
:10DEB000009729F06A817B8181E00E940F5CCE018E
:10DEC000DF91CF9108950F931F93CF93DF93EC01D0
:10DED000E0913403F091350309958C016A817B81CF
:10DEE00081E00E940F5C81E090E0012B11F480E062
:10DEF00090E0DF91CF911F910F910895E09136034B
:10DF0000F0913703099420E030E00296FC0132974B
:10DF10004081442331F0FC0131974081240F311DB1
:10DF2000F4CFC9010895FC01208130E0322F22276F
:10DF30008181282B02C0220F331F6A95E2F7832FBD
:10DF40009927FA01E85CFC4F208130E0822393237B
:10DF500028E030E0241B350B02C0969587952A9562
:10DF6000E2F708956F927F928F929F92AF92BF9245
:10DF7000CF92DF92EF92FF920F931F93CF93DF9395
:10DF80008C01EB016A0179012830310524F4A901E3
:10DF9000B601CE014AC0590123E0B594A7942A9551
:10DFA000E1F74115510521F04801612C712C03C0A6
:10DFB000D801FB0120C048E050E0B601CE01860D3B
:10DFC000971D0E94936FF40181934F01FFEF6F1A29
:10DFD0007F0A6A147B047CF3C501B7FE02C080E0AF
:10DFE00090E0A701477055274115510511F1080F21
:10DFF000191FB60118C0CF018C1B9D0B8A159B05FC
:10E000001CF481918D93F7CFC501B7FE02C080E06B
:10E0100090E0A701477055274115510551F0080FB1
:10E02000191F60E070E08C0F9D1F0E94936FF80134
:10E030008083DF91CF911F910F91FF90EF90DF9040
:10E04000CF90BF90AF909F908F907F906F900895EA
:10E050008F929F92AF92BF92CF92DF92EF92FF92F8
:10E060000F931F93CF93DF9300D0CDB7DEB70E94FD
:10E07000FD5A8C0182E090E00E94DB5A892B19F452
:10E0800080E090E05DC0F801818190E0982F8827C2
:10E090002081820F911D0E94CB527C01009781F359
:10E0A0000E94FD5A4C01F7012681822F86958695A4
:10E0B000869590E0422F477021E030E011F420E097
:10E0C00030E0820F931F0E94DB5A892BC9F2F701BF
:10E0D00004811581C12CD12CF8018081882379F12C
:10E0E000F801A180B12CB60133E0759567953A959A
:10E0F000E1F7A60147705527680D791D883168F052
:10E100009501CE0101960E94B26FBE016F5F7F4FF5
:10E11000F80180810E94235C0DC01A82198295014A
:10E12000CE0101960E94B26F69817A81F8018081E7
:10E130000E940F5CCA0CDB1C0E5F1F4FCDCFC701C6
:10E140000F900F90DF91CF911F910F91FF90EF9063
:10E15000DF90CF90BF90AF909F908F900895DC019B
:10E1600050E0E0E1F0E0E61BF70BE21BF30B02C02E
:10E17000440F551FEA95E2F78C91852B8C931196ED
:10E180008C911197842B11968C9308956F927F92A6
:10E190008F929F92AF92BF92CF92DF92EF92FF92B7
:10E1A0000F931F93CF93DF938C016B01EA017901E9
:10E1B000283031051CF44881C8015CC0390153E0A6
:10E1C000759467945A95E1F76115710521F04E0138
:10E1D000A12CB12C03C0D801FE0127C0F40141914C
:10E1E0004F0128E030E0B601C8018A0D9B1D0E9456
:10E1F000AF70FFEFAF1ABF0AA614B7047CF3C301D8
:10E2000077FE02C080E090E0970127703327211548
:10E21000310509F43FC0C80FD91F488150E0B6014D
:10E22000621B730B685F7F4F1CC0CF018C1B9D0B63
:10E23000861597051CF481918D93F7CFC30177FE66
:10E2400002C080E090E09701277033272115310547
:10E2500009F1C80FD91F488150E068E070E0621BE7
:10E26000730B02C0559547956A95E2F760E070E040
:10E27000800F911FDF91CF911F910F91FF90EF9031
:10E28000DF90CF90BF90AF909F908F907F906F90D6
:10E290000C94AF70DF91CF911F910F91FF90EF9091
:10E2A000DF90CF90BF90AF909F908F907F906F90B6
:10E2B00008956F927F928F929F92AF92BF92CF926A
:10E2C000DF92EF92FF920F931F93CF93DF9300D0D3
:10E2D000CDB7DEB78C01FC018681E82EE694E6948A
:10E2E000E694F12C282F277081E090E011F480E073
:10E2F00090E0E80EF91EC70102960E945F5B00974E
:10E3000009F445C00E94045BF8012281FC012083CE
:10E31000F8012381FC0121830E94045B02965C01C9
:10E32000A70160E070E00E94F391F801048115817B
:10E33000E12CF12CF8018081882339F1F8018180EA
:10E34000912C670163E0D594C7946A95E1F7370192
:10E35000F7E06F227724CA0CDB1C883128F00E947A
:10E360002D5C9401AC0108C00E941A5C9A838983D9
:10E370009401AE014F5F5F4FB301C6010E94C670AA
:10E38000E80CF91C0E5F1F4FD5CF81E090E00F9095
:10E390000F90DF91CF911F910F91FF90EF90DF9041
:10E3A000CF90BF90AF909F908F907F906F90089587
:10E3B000E0915303F09154030994E0912C03F09100
:10E3C0002D030994E0915703F09158030994E091CB
:10E3D0005903F0915A03099480E090E0089508955C
:10E3E000E0912403F0912503099480E090E00895E2
:10E3F0000F931F93CF93DF93CDB7DEB7E0970FB6A0
:10E40000F894DEBF0FBECDBF0E944A5B8C010E9414
:10E41000FD5AAE014F5F5F4F602F0E94C87988237D
:10E4200009F446C088A99801281B3109C9010E9436
:10E43000DB5A892BE9F12E8121110CC0BE016A5EE5
:10E440007F4F88E10E94235CE0914703F0914803ED
:10E4500009952EC08A859B858D3C3BEA930711F078
:10E46000019631F5223019F088E090E002C082E098
:10E4700090E001979C012F5F3F4F12161306F4F6B0
:10E48000E1E0F0E0EC0FFD1FE80FF91F23852F3FBF
:10E4900081F3BE01645F7F4F89E10E94235C89E1C3
:10E4A0000E942D5C62EB78E20E941952892B31F6B2
:10E4B000E0960FB6F894DEBF0FBECDBFDF91CF91CF
:10E4C0001F910F910895AF92BF92CF92DF92EF927A
:10E4D000FF920F931F93CF93DF93CDB7DEB7E097F3
:10E4E0000FB6F894DEBF0FBECDBF8C016B01CE011D
:10E4F00001967C0180E3F70111928A95E9F781E0AA
:10E5000089838CE00E941A5C8C831D821F8280911B
:10E510007C1491E0980F90937C14898783E0B82E47
:10E52000B8868DEC9BEA9B878A8789E10E942D5CE7
:10E5300060E073E00E941952892B31F082E08E83F3
:10E540008FEF8C878D8709C089E10E942D5CBC010B
:10E55000CE010C960E941052BE828DEC9BEA9D8BE0
:10E560008C8B62EB78E2CE0146960E9410520E949C
:10E57000FD5A9FA78EA70E944A5B88ABC7010E94E5
:10E58000C178B82E90E00E945F5B892B31F10E9428
:10E59000045BBC014B2DC7010E94DF78E0901A0399
:10E5A000F0901B030E94545B5C010E94045BB50168
:10E5B000F70109950115110581F0009739F00197D0
:10E5C00061F441E050E064E070E004C041E050E0FC
:10E5D00060E070E0C601F8010995E0960FB6F89486
:10E5E000DEBF0FBECDBFDF91CF911F910F91FF9086
:10E5F000EF90DF90CF90BF90AF9008950E9441744C
:10E6000080937C14E0912403F09125030994892BD5
:10E6100029F0E0912403F091250304C0E091260342
:10E62000F09127030994CF93DF93EC01899199919D
:10E63000009729F060E070E00E946454F7CFDF910A
:10E64000CF910895CF93DF93EC0189919991009731
:10E6500019F00E94B653F9CFDF91CF910895CF936F
:10E66000DF93EC017B836A830E94D864998388835B
:10E67000DF91CF910895FC018081918122813381C6
:10E68000820F931F918380830895CF93DF93EC01D2
:10E690000E94D86499838883DF91CF910895CF93A6
:10E6A000DF93EC010E94D86428813981821B930B8F
:10E6B0009C012F5F3F4F81E090E04A815B814217D0
:10E6C000530710F080E090E0DF91CF910895CF9351
:10E6D000DF93FC01C281D38180819181C80FD91F52
:10E6E0000E94D8649E01281B390BC901DF91CF918C
:10E6F0000895CF93DF93EBE2FBE2CDEEDAE2AFE1F8
:10E70000BBE21192119219921992199219921D92CB
:10E710008BE2E334F807A9F7DF91CF910895CF9307
:10E72000DF93FC01E15EF44D40819C01220F331F19
:10E73000220F331F442301F1A0919400B091950062
:10E74000FC01EE0FFF1FE55DF44D80819181AD016D
:10E75000481B590BCA01E901C351D54D4881598164
:10E760006A817B81480F591F611D711D4883598340
:10E770006A837B83B183A083F901E351F54D608106
:10E78000718182819381DF91CF91089560E070E083
:10E79000CB010895FC01EE0FFF1FEE0FFF1FE351A9
:10E7A000F54D40835183628373830895CF93DF9344
:10E7B0002FE13BE2CDEEDAE2EBE2FBE2D9018D9113
:10E7C0009D018823B9F0409194005091950080817B
:10E7D0009181BA01681B790B88819981AA81BB81DB
:10E7E000860F971FA11DB11D88839983AA83BB83C0
:10E7F0005183408324963296BBE22B323B07F1F6DD
:10E80000DF91CF9108950C9450780F931F93FC01E2
:10E81000CB0140917D1450917E1433832283158364
:10E82000048371836083F0937E14E0937D14452B01
:10E8300011F40E946A7880E090E01F910F91089592
:10E8400080917D1490917E140097C1F010927E14F7
:10E8500010927D14DC0114966D917C91159712969F
:10E86000ED91FC9113970995E0917D14F0917E1440
:10E87000309721F0808191810C946A7808950C94EE
:10E880007D8E0C94798E84ED92E00E949B548CECEA
:10E8900092E00C949B54CF93DF930E940A5B892BE8
:10E8A000A9F08CEC92E00E94B954EC01009721F1A0
:10E8B0000E944A5B998388830E94455B9B838A837D
:10E8C000CE0104960E94865A8CAB14C084ED92E06F
:10E8D0000E94B954EC01009779F002960E94985A70
:10E8E00099838883BE016E547F4FCE018E579F4F10
:10E8F0000E94ED5BCE0102C080E090E0DF91CF91FD
:10E900000895BC016E547F4F8E579F4F0C94ED5B62
:10E91000CF93DF93EC01BC0184ED92E00E9403559C
:10E92000BE01892B19F084ED92E009C08CEC92E0D5
:10E930000E940355892B39F0BE018CEC92E0DF91E7
:10E94000CF910C94DE54DF91CF9108950F931F93D4
:10E95000CF93DF93EC01BC0184ED92E00E9403555C
:10E96000892B91F0FE0161917191CF010E94A95B09
:10E97000BE016E547F4FCE018E579F4FDF91CF91D6
:10E980001F910F910C94FE5BBE018CEC92E00E94F3
:10E990000355892BD1F00E94965B688179818A8129
:10E9A0009B810E94A95B8CA990E00E945F5B0CA9EF
:10E9B00010E00E94045BBE016C5F7F4FA801DF91F5
:10E9C000CF911F910F910C94EA91DF91CF911F91FC
:10E9D0000F910895CF93DF93EC01BC0184ED92E099
:10E9E0000E940355892B19F0CE0102960CC0BE017E
:10E9F0008CEC92E00E940355892B19F08A819B814F
:10EA000002C080E090E0DF91CF910895FC01808109
:10EA100091810895860F911D860F911D8E579F4FEE
:10EA20000895860F911D860F911D8E579F4FFC01F3
:10EA300080819181089508958CED9AE10E94DD56C0
:10EA4000892B21F08CED9AE10C94CA560895E0913F
:10EA5000C81AF091C91A309709F0099480E0089516
:10EA6000EF92FF920F931F93CF93DF937C01EA0104
:10EA7000FC0180819181009741F08C30934071F1CD
:10EA8000F7011182108283E0F2C080E024E0829FCF
:10EA9000F0011124E653F54E118210828F5F84300D
:10EAA000A8F38093C71A8091021290910312909359
:10EAB000DB1A8093DA1A0E94AF538093432B60E4F1
:10EAC00070E08CED9AE10E94B6560E943E7B8CE08D
:10EAD00093E0F7019183808381E0C9C06230D9F46B
:10EAE0008091442B9091452B892B89F38091552B54
:10EAF000863029F480916D2B81FD0E941C7581E088
:10EB00000E947C7C8091442B9091452B892BF9F2BB
:10EB10000E944077DCCF633060F5611114C020970C
:10EB2000B1F2D0935230C093513083E00E947C7C8C
:10EB30008091442B9091452B892B11F00E942775D1
:10EB40000E941C75C4CF613011F6209709F4BFCF25
:10EB5000D0934E30C0934D3085E00E947C7C8091F4
:10EB6000442B9091452B892B09F4B1CF0E94277536
:10EB7000AECF6738E9F51092C61A0AEC1AE1809117
:10EB8000C61A8430B8F4F801828193818C179D07EE
:10EB900049F4808191810E94497CF80111821082A0
:10EBA000138212820C5F1F4F8091C61A8F5F809371
:10EBB000C61AE5CFECE6F0E3838194818C179D07BC
:10EBC00019F4148213821082B09620E3EC3EF2070F
:10EBD00099F7E9EEF0E3818592858C179D0711F492
:10EBE000158214823D9681E3EB36F807A1F76FCFCB
:10EBF000683809F06CCFCC5DDA4109F068CF8CED54
:10EC00009AE10E94DD56892B09F461CF1092C61A51
:10EC1000E091C61AE43008F05ACF20E2E29FF001FA
:10EC20001124ED5AFF4C818D8823D9F08CED9AE1A7
:10EC30000E94CA568091C61AE0E28E9FC00111243C
:10EC40008D5A9F4C909352308093513082E00E94B5
:10EC50007C7C8091442B9091452B892B11F00E9454
:10EC600027758091C61A8F5F8093C61AD1CFDF9126
:10EC7000CF911F910F91FF90EF9008959093C91A33
:10EC80008093C81A0895209102123091031260E017
:10EC9000EAECFAE1643098F4408151814817590751
:10ECA00059F4428153814217530731F46093C51AD6
:10ECB000118210820C94497C34966F5FEBCF609385
:10ECC000C51A089540E0EAECFAE14430A8F451E0B6
:10ECD000540F20813181232B61F44093C41A918316
:10ECE00080832091021230910312338322830C948B
:10ECF000637C3496452FE9CF4093C41A0895209140
:10ED0000021230910312FC01358F248F778F668FAA
:10ED100008952091021230910312FC01328721875D
:10ED2000748763870895CF93DF93EA010E94EC7B99
:10ED3000009749F02091021230910312FC013287B2
:10ED40002187D487C387DF91CF9108950F931F93B5
:10ED5000CF93DF9300D000D0CDB7DEB78C01AB01ED
:10ED60008FEF89838A838B838C83B801CE010196D0
:10ED70000E949376009719F0FC01158304830F908D
:10ED80000F900F900F90DF91CF911F910F910895E9
:10ED900040E050E062E08CED92E00E945554109209
:10EDA000452B1092442B0895AC0161E08CED92E06C
:10EDB0000C943754AC0160E08CED92E00C94375425
:10EDC0000F931F93CF93DF938A010E946A7BEC011C
:10EDD000009759F080910212909103129D8F8C8FB1
:10EDE0001F8F0E8FCE010E94DA76CE01DF91CF9178
:10EDF0001F910F910895CF93DF93A0915130B0915F
:10EE00005230109719F0ED016C9605C0C0914D304D
:10EE1000D0914E30299680914C3086FF22C01092BE
:10EE2000C31A40E0EAECFAE14430B8F420813181C1
:10EE300014968D919C9115972817390759F4828162
:10EE40009381009739F04093C31A998388831B827A
:10EE50001A8205C034964F5FE7CF4093C31A0E94D1
:10EE60001C7588819981009741F04A815B8160918E
:10EE7000432BDF91CF910C945554DF91CF9108959E
:10EE80000F931F93CF93DF938091552B863009F01A
:10EE900071C08091442B9091452B8115954009F0CC
:10EEA00069C0C4E9D2E0D093452BC093442B02E063
:10EEB00000934E2B14E910934F2B1092712B10924C
:10EEC000702B0E94387B809590959093712B809346
:10EED000702B1092572B1092562B0E94277B8095F7
:10EEE00090959093572B8093562B0E942775D09323
:10EEF000452BC093442B00934E2B10934F2BA09186
:10EF00004F30B0915030FD01E459FD4F8CE692E056
:10EF100001900D920197E1F76CE672E084E69BE2C6
:10EF20000E94E67A8091482B8093642B8091492B34
:10EF30008093652B80914A2B8093662B80914B2B7D
:10EF40008093672B1092712B1092702B0E94387B4C
:10EF5000809590959093712B8093702B1092572BE6
:10EF60001092562B0E94277B809590959093572B5B
:10EF70008093562BDF91CF911F910F910C942775A1
:10EF8000FC01680F791F80E048E1E617F70781F080
:10EF9000219198E0322F3827532F517030FD84276C
:10EFA0008695513009F480682695915099F7EDCFF8
:10EFB00008951F920F920FB60F9211240BB60F9265
:10EFC0002F933F934F935F936F937F938F939F9371
:10EFD000AF93BF93EF93FF9380919400909195002E
:10EFE0009093302B80932F2B81E08093212B809165
:10EFF0007100807D809371000E9420748091212B8C
:10F000008823D9F1809194009091950040912F2B05
:10F010005091302B84179507A0F48091F52A909198
:10F02000F62AA091F72AB091F82A8C57914EAF4F4B
:10F03000BF4F8093F52A9093F62AA093F72AB093B6
:10F04000F82A2091940030919500241B350B809173
:10F05000F52A9091F62AA091F72AB091F82A820F0A
:10F06000931FA11DB11D8093F52A9093F62AA093BA
:10F07000F72AB093F82A1092212BFF91EF91BF91BC
:10F08000AF919F918F917F916F915F914F913F9140
:10F090002F910F900BBE0F900FBE0F901F901895E1
:10F0A0009FB7F894E1E7F0E08081807D808388B3AA
:10F0B0008F6288BB10929000E1E9F0E0108210921C
:10F0C0009200109295001092940080818560808358
:10F0D0009FBF08952FB7F89490939900809398005C
:10F0E00088B38F6288BBE1E7F0E080818260808333
:10F0F0002FBF0895CF93DF93FC01DB0185E0EB0187
:10F1000019928A95E9F78581837011F082E08C93DA
:10F110008781837021F082E012968C93129785810B
:10F12000837081F08781837069F0238934898185B8
:10F1300092852817390731F481E0848312961C9256
:10F14000129701C0148285818370823021F0833050
:10F1500021F080E003C082E001C088E011968C932A
:10F16000119787818370823021F0833021F080E015
:10F1700003C082E001C088E013968C93DF91CF91A9
:10F180000895CF93DF9300D000D01F92CDB7DEB7A4
:10F19000BE016F5F7F4F0E947A7889819A81890FC3
:10F1A0008D5F9B81890F9C81890F9D81890F0F90B5
:10F1B0000F900F900F900F90DF91CF9108954F9285
:10F1C0005F926F927F928F929F92AF92BF92CF92F7
:10F1D000DF92EF92FF920F931F93CF93DF9300D0B4
:10F1E00000D000D0CDB7DEB78C017B01BE016F5FD0
:10F1F0007F4F4E830E947A78B981AA815B804C80D0
:10F200008B2F90E003962A2F30E0820F931F850DFD
:10F21000911D642D70E0860F971F5D81850F911DF4
:10F220004E8150E0481759070CF49AC0F8018181CB
:10F2300080FB662460F8712C43E0660C771C4A95CD
:10F24000E1F7828180FB882480F8912C54E0880CBF
:10F25000991C5A95E1F7862880818770882A8381D6
:10F2600080FBAA24A0F8B12C85E0AA0CBB1C8A95CF
:10F27000E1F78A28848180FBCC24C0F8D12C96E069
:10F28000CC0CDD1C9A95E1F78C28F7018082F801FF
:10F2900045814370F4E04F9FA0011124F80186815D
:10F2A0008370F0E18F9FC0011124482BF801878102
:10F2B000F0E48F9FC0011124482BF7014183F8012E
:10F2C0008085F7018283B23059F4F8018185F70116
:10F2D0008383F8018285F701848395E0C92E02C0FB
:10F2E00083E0C82EB0E080E090E0200F311FDB2EDD
:10F2F000DC0C0197BA1761F0A901480F591FFA01F8
:10F30000B384A7014D0D511DFA01B082BF5FEFCF4D
:10F310009D2DF2E05F120EC0D701AD0DB11DF801B9
:10F3200083898C9381E08D0DD701A80FB11D9E5F5D
:10F3300084898C9340E020E030E0060F171F842F73
:10F34000890F21503109441561F0D801A20FB31F74
:10F3500055965C91D701A80FB11D5C934F5FEFCF1D
:10F3600080E026960FB6F894DEBF0FBECDBFDF91CA
:10F37000CF911F910F91FF90EF90DF90CF90BF90B2
:10F38000AF909F908F907F906F905F904F90089577
:10F39000BF92CF92DF92EF92FF920F931F93CF9382
:10F3A000DF937C01D62EEA0182E0861708F0B2C016
:10F3B000F701808186FBBB24B0F89181292F269527
:10F3C00026952370C92EC294C694C69453E0C522D4
:10F3D000382F3770388383FB332730F9398384FB28
:10F3E000332730F93A8385FB882780F98B83BC82E9
:10F3F0002D83892F829583708E83CF828281888727
:10F40000222391F13381848190E0982F8827830F04
:10F41000911D9A87898787010B5F1F4F223079F4EE
:10F4200060E073E0CE010B960E941052F7018681D6
:10F430008B8785818C878701095F1F4F20C0233010
:10F44000F1F4F7013D9680E090E03E2F2F2F42919E
:10F45000DE01A80FB91F1B964C93019688309105C9
:10F46000B1F7032F122F0BC087010D5F1F4F60E014
:10F4700073E0CE010B960E9410521A861986CC209A
:10F48000B9F1B1100DC0F8012081818190E0982F71
:10F490008827820F911D9C8B8B8B0E5F1F4F04C0A2
:10F4A00089859A859C8B8B8BF2E0CF120EC060E031
:10F4B00073E0CE0145960E941052F80181818D8B38
:10F4C00080818E8B0E5F1F4F1BC0F3E0CF1218C0E0
:10F4D000085F1F4FF80180E090E02291DE01A80F45
:10F4E000B91F55962C93019688309105B1F708C045
:10F4F00060E073E0CE0145960E9410521C8A1B8A80
:10F50000C8018E199F092D2D281B2FA71EA70DA7F7
:10F51000D81608F480E0DF91CF911F910F91FF90F2
:10F52000EF90DF90CF90BF900895FB0141505109BB
:10F53000460F571FE417F50778F4208130E0322F8B
:10F5400022276181260F311D820F931F8217930797
:10F5500008F401963296EECFE417F50751F42081B6
:10F5600030E0322F2227820F931F8217930708F46F
:10F5700001960895CF93DF93C0914F2BD0E064970D
:10F5800020914E2B30E0322F2227C20FD31F48E0AC
:10F5900050E068E57BE29E01280F311DC9010E9401
:10F5A000957AAE0160E67BE20E94957A009721F0A1
:10F5B00098278927982702C08FEF9FEFDF91CF917F
:10F5C00008959093F51A8093F41A0895FC015381DD
:10F5D000560F50934B2B872F99274281480F40930A
:10F5E0004A2BA181A093492BE081E093482B242F43
:10F5F00030E02817390748F481E08A0F8093492BBF
:10F60000811103C0EF5FE093482B852F90E07727AF
:10F610008617970788F44F5F40934A2B41110CC01F
:10F620008091492B8F5F8093492B811105C0809178
:10F63000482B8F5F8093482B0895AB01BC0180E07D
:10F6400090E00E94957A982789279827089544E1A9
:10F6500050E06CE47BE280E090E00E94957A0097B5
:10F6600021F098278927982708958FEF9FEF089515
:10F6700086E00C94BA7A81E10C94BA7A80E0E82FA3
:10F68000F0E0EE0FFF1FED52FF4C118210828F5FF2
:10F690008430A8F380E090E2899FF0011124ED5AB4
:10F6A000FF4C118E8F5F8430B0F380E094E0909334
:10F6B000EF1A8093EE1A80E09DE0989FF0011124EC
:10F6C000E751FF4C158214828F5F8A30B0F380932C
:10F6D000ED1A0895CF932091EE1A3091EF1A2F5F13
:10F6E0003F4F21154DE7340710F020E030E1522F55
:10F6F000432FE3E5F0E3C0E0C43059F0A18DAA2325
:10F7000029F0A481B581A417B50749F3CF5FB0965E
:10F71000F3CF3093EF1A2093EE1A1092ED1A20E0F7
:10F72000E0E0F0E02430E8F430E2239FD00111243F
:10F73000AD5ABF4C59963C915997311104C0209352
:10F74000ED1AFD0110C0373041F4309739F05A9668
:10F750004C915A97328D341708F0DF012F5FFD016D
:10F76000E1CF2093ED1A3097A1F122E0218F209173
:10F77000F01A24872091F11A25872091F21A268702
:10F780002091F31A278728ED34E0338B228B358BB9
:10F79000248B21E030E0318B208B138E21E0228FEF
:10F7A00023E0208F168A20E1278B2091EE1A3091DA
:10F7B000EF1A322723273227358324837783668302
:10F7C000DC014D915D916D917C9140835183628309
:10F7D0007383CF01CF910895CF93DF932091EE1AD9
:10F7E0003091EF1A2F5F3F4F21154DE7340710F08E
:10F7F00020E030E1522F432FEDEEF0E3C0E0CA30BD
:10F8000041F0A081B181CF5F3D96A417B507B9F74C
:10F81000E9CF3093EF1A2093EE1A40E05DE04A30D2
:10F82000A0F4A1E0A40F549FF0011124E751FF4C74
:10F8300024813581232B39F44093ED1A309741F41C
:10F8400080E090E023C04A2FEACF4093ED1AF8CF32
:10F850002091EE1A3091EF1A322723273227358371
:10F86000248377836683009729F4108211821282A1
:10F87000138209C0EC0188819981AA81BB818083B0
:10F880009183A283B38380E48087CF01DF91CF91FE
:10F89000089540E04430A0F4E42FF0E051E0540F2C
:10F8A000EE0FFF1FED52FF4C2081318128173907E1
:10F8B00029F44093ED1A118210820895452FEACF62
:10F8C0004093ED1A089540E0443098F4E42FF0E0BE
:10F8D00051E0540FEE0FFF1FED52FF4C208131819C
:10F8E000232B29F44093ED1A918380830895452FAB
:10F8F000EBCF4093ED1A0895AF92BF92CF92DF9273
:10F90000EF92FF920F931F93CF93DF93C0915130EB
:10F91000D0915230843009F4DCC124E73BE23093CB
:10F92000503020934F303093472B2093462B833019
:10F9300059F4898D8F70833009F06BC0888999895B
:10F94000892B09F0DFC67FC0823009F080C080912A
:10F95000F31A8F5F8093F31A811113C08091F21A0A
:10F960008F5F8093F21A81110CC08091F11A8F5F22
:10F970008093F11A811105C08091F01A8F5F8093F6
:10F98000F01A1092452B1092442B1092E8301092EE
:10F99000E730298D822F8D7F853041F48A8D8F5FEE
:10F9A0008A8F843109F0AEC6198EACC6222309F4C1
:10F9B000A9C688899989892B09F441C08A8D9FEF4E
:10F9C000980F9A8F81119EC68B8D883031F09FEFF2
:10F9D000920F923048F4853039F4198E80E8809384
:10F9E0004C300E94FB7647C5853038F493E0082EF2
:10F9F00001C0990F0A94EAF701C090E39A8F8F5FD4
:10FA00008B8F822F8F708330A1F048F4813009F4FE
:10FA10004FC3823009F076C610926D2B4CC38630EE
:10FA200009F4C8C4883009F4C5C4843009F06AC632
:10FA3000C1C484E080934C300E94FB764EC52F7089
:10FA4000233009F05FC688E080934C3009C58530CB
:10FA500019F5E0914D30F0914E3084819581892BDC
:10FA600009F450C6109252301092513088E69BE251
:10FA70009093503080934F309093472B8093462B38
:10FA80001092E8301092E7301092452B1092442BE0
:10FA900088E080934C301BC180914C2B853409F059
:10FAA00031C600914E2B10E0102F002780914F2B74
:10FAB000080F111D8091442B9091452B80179107C1
:10FAC00008F420C61093452B0093442B8091522BB1
:10FAD0008F7309F017C68091532B811113C6809143
:10FAE000E3309091E430C0915D03D0915E038C17B8
:10FAF0009D0759F44091E5305091E63020915F0325
:10FB00003091600342175307A1F020915C2B309194
:10FB10005D2B2817390709F0F5C520915E2B309130
:10FB20005F2B8091E5309091E6302817390709F076
:10FB3000E9C50E94277B019609F0E4C58091552B09
:10FB4000863009F429C18131E9F1813009F0DAC543
:10FB50008091602B883009F0D5C51092602B809180
:10FB6000622B9091632B873F3FEF930710F009962C
:10FB700001C008969093632B8093622B8091582B41
:10FB80009091592BA0915A2BB0915B2B80935C2BB9
:10FB900090935D2BA0935E2BB0935F2B8091E3300D
:10FBA0009091E430A091E530B091E6308093582BED
:10FBB0009093592BA0935A2BB0935B2B80E48093A6
:10FBC000542B7DC50C5111091093452B0093442BE8
:10FBD00088E69BE29093503080934F308091662B63
:10FBE0009091672B892B29F00E943B7B019609F0AD
:10FBF00089C52091622B3091632B2115310509F4C1
:10FC000081C589EE90E390934E3080934D30A09063
:10FC1000602BB090612B40915F0350916003609125
:10FC2000610370916203A0916303B091640300913A
:10FC3000582B1091592BE0905A2BF0905B2BE091B0
:10FC40004D30F0914E3081E3EB36F80708F05AC59D
:10FC500084819581009721F12817390709F586815C
:10FC60009781009719F0A816B906D1F48081918187
:10FC70008C179D0729F4C280D380C416D506B1F035
:10FC80008617970729F4C280D380CA16DB0671F065
:10FC90000817190729F482819381E816F90631F0D3
:10FCA0003D96F0934E30E0934D30C9CF10925230D4
:10FCB0001092513082E080934C3088E69BE2909322
:10FCC000472B8093462B1092E8301092E7300E9429
:10FCD000FB768091E7309091E830009709F412C5E7
:10FCE0009C01245E3F4F3093452B2093442B30934F
:10FCF0004E2B20934F2BE0914D30F0914E302085CC
:10FD00002093542B21E12093552B0896982789277F
:10FD100098279093652B8093642B1092672B1092F9
:10FD2000662B848195819093612B8093602B8681D3
:10FD300097819093632B8093622B8091E330909115
:10FD4000E430A091E530B091E6308093582B909349
:10FD5000592BA0935A2BB0935B2B80819181A28168
:10FD6000B38180935C2B90935D2BA0935E2BB0931B
:10FD70005F2B84E79BE29093503080934F300E943A
:10FD80003B7B80959095009711F48FEF9FEF9093B8
:10FD9000672B8093662B93C40E94387B019609F0F1
:10FDA000B1C48091622B9091632B009709F4AAC48F
:10FDB0002091602B3091612B2115310509F4A2C4EB
:10FDC0004091582B5091592B60915A2B70915B2B7D
:10FDD000ECE6F0E3C3E5D0E3F080FF20A9F0AC81CE
:10FDE000BD818A179B0781F4AE81BF812A173B072B
:10FDF00059F4A881B9814A175B0731F4AA81BB8104
:10FE00006A177B0709F46FC1A096B096A0E3C33DC3
:10FE1000DA0711F720916D2B2F732230D9F49093CC
:10FE2000EB1A8093EA1A40E0443090F4E42FF0E0BB
:10FE3000EE0FFF1FED52FF4C208131814F5F821783
:10FE4000930791F71092ED1A20E0C0E0D0E07EC059
:10FE50004093ED1A80916D2B82FD54C484E1809310
:10FE60006D2B88E290E09093452B8093442B80E5A6
:10FE700080936C2B8091672B90916B2B9093672BC9
:10FE80003091662B90916A2B9093662B30936A2B5E
:10FE90002091652B9091692B9093652B2093692B72
:10FEA0009091642B9093ED1A4091682B4093642BB2
:10FEB0009093682B8F5F80936B2B81110FC081E033
:10FEC000830F80936A2B811109C081E0820F809398
:10FED000692B811103C09F5F9093682B8091602BE9
:10FEE0009091612B9093EB1A8093EA1A2091622BE8
:10FEF0003091632B3093612B2093602B9093632B75
:10FF00008093622B8091582B9091592BA0915A2B62
:10FF1000B0915B2B80935C2B90935D2BA0935E2B19
:10FF2000B0935F2B8091E3309091E430A091E53065
:10FF3000B091E6308093582B9093592BA0935A2B75
:10FF4000B0935B2BA1C3373089F02F5F2430C0F40E
:10FF500030E2239FC0011124FC01ED5AFF4C318D8A
:10FF60003111F1CF2093ED1AEF010CC0209721F051
:10FF7000428D3A8D341748F7EC01CD5ADF4CE5CF6E
:10FF80002093ED1A209709F4BDC3D0935230C0934B
:10FF9000513083E08A8F888F1E8A84E08F8B1B8E7E
:10FFA0008091622B9091632B9D838C838091602B39
:10FFB0009091612B9F838E838091582B9091592B28
:10FFC000A0915A2BB0915B2B88839983AA83BB8322
:10FFD00081E0898F8091F01A8C878091F11A8D874A
:10FFE0008091F21A8E878091F31A8F8781E090E0DA
:10FFF000998B888B8091672B8B878091662B8A8762
:020000021000EC
:100000008091652B89878091642B888781E090E0BF
:100010000E94E68380916C2B282F207F30E02135D1
:1000200031050CF445C082958F7090E00597880FDC
:10003000991F880F991F3091EC1A20E0E22FF0E011
:10004000E817F9078CF5E45BF44D30A5311105C0D4
:100050002093ED1A1092EC1A2BC0313011F42F5F5F
:10006000EDCF3230E1F441A54430C9F42093ED1ACC
:100070003093EC1A82A590E0982F882723A5822B35
:100080009093EB1A8093EA1A893DA4E09A0710F046
:1000900088ED94E09B8B8A8B9D8B8C8B09C041A54E
:1000A000442311F0240FCACF2093ED1A3093EC1A99
:1000B00080E180936D2B80916D2B826080936D2BFE
:1000C00082E08093742B84E08093752B8093762B51
:1000D00088ED8093772B8CE290E09093452B809372
:1000E000442B80E67EC2D0935230C09351301092A0
:1000F0004C3090916D2B92FF03C0198E80E21AC292
:1001000080916C2B82958F70880F880F8093ED1AE9
:10011000081B1109045111091093452B0093442B1E
:100120008F2D8F70823029F4892F8F73823139F4AB
:100130001FC0813021F4892F8F738230C9F0012BC9
:1001400019F4892F8370A1F02091642B88852813DE
:100150003EC22091652B8985281339C22091662BD8
:100160008A85281334C22091672B8B8528132FC2D0
:1001700094FF4AC0688979896115710509F444C002
:10018000CE010C960E94E67A3091682B8091482B24
:1001900038133AC02091692B8091492B281334C021
:1001A00090916A2B80914A2B98132EC080916B2BD3
:1001B00040914B2B841328C03C872D879E878F87C7
:1001C0008B8D81111AC02E89888D9A8D891B922F53
:1001D000969596959695891B280F2E8B87FD819570
:1001E0009F89392F36953695931B980F9F8B822FB9
:1001F000869586958695890F888F81E080934C300F
:10020000888D8A8F198A188A498D842F8F7090E083
:10021000FC013197E830F10508F074C2E057FF4F58
:100220000C94B58D80914C3080FF14C083E0898F91
:1002300080E480934C30198A188A8091442B9091E5
:10024000452B009709F408C122E420934C300E940A
:10025000E68302C180916D2B8F73823009F052C208
:1002600027CF80914C3080FF70C080916D2B8F73B1
:10027000823109F06AC080916C2B282F207F30E0FA
:10028000213531050CF445C082958F7090E00597BB
:10029000880F991F880F991F3091EC1A20E0E22FE8
:1002A000F0E0E817F9078CF5E45BF44D30A5311167
:1002B00005C02093ED1A1092EC1A2BC0313011F4C6
:1002C0002F5FEDCF3230E1F441A54430C9F42093E3
:1002D000ED1A3093EC1A82A590E0982F882723A579
:1002E000822B9093EB1A8093EA1A893D24E09207BF
:1002F00010F088ED94E09B8B8A8B9D8B8C8B09C0D2
:1003000041A5442311F0240FCACF2093ED1A309356
:10031000EC1A83E0898F8091642B88878091652B0C
:1003200089878091662B8A878091672B8B8781E0F4
:1003300090E00E94E68382E480934C30198A188A08
:100340001092452B1092442B87C080E280934C3052
:100350000E94FB76E0915130F0915230118E7ACDAF
:1003600080916D2B80FF28C044FD26C08889998923
:10037000892B09F0C7C18091442B9091452B0196A0
:100380000E94E68320914C30822F806180934C3014
:100390008091442B9091452B892B19F02261209359
:1003A0004C300E94FB7681E090E0998B888B88E04E
:1003B000898F1B8E81E10CC185FF1CC08091722B3F
:1003C00090E0982F88272091732B822B20914F301B
:1003D00030915030280F391F3093503020934F30D8
:1003E0002091442B3091452B281B390B3093452B02
:1003F0002093442B8091442B9091452B009749F0FA
:1004000044FD07C020914C30226020934C300E9464
:10041000E68380916E2B90E0982F882720916F2B98
:10042000820F911D9093EB1A8093EA1A2C893D89D3
:100430002817390710F0892B21F43093EB1A2093F9
:10044000EA1A8091EA1A9091EB1A9B8B8A8B809121
:100450004C30837009F456C11092E8301092E730A6
:100460000E94FB7680914C3085FF07C01092E830E7
:100470001092E730198E84E1ABC084FF0AC010925D
:10048000E8301092E73081E090E0998B888B84E02F
:100490008FCF2091E7303091E83021153105E1F020
:1004A00080FF02C0198A188A88899989009781F487
:1004B0008A899B898217930720F49093E830809370
:1004C000E7308091E7309091E830998B888B04C0B9
:1004D0009093E8308093E7301B8E8091462B90916B
:1004E000472B9093503080934F308091E73090911C
:1004F000E830892B59F088899989009739F08896D6
:100500009093452B8093442B88E10BC080914C3015
:1005100081FFF8C088E290E09093452B8093442BB4
:1005200080E180936D2B5CC080914C3080FFEAC0ED
:10053000198E80E180934C300E94FB76E3C080915D
:10054000442B9091452B009711F00E94E6839091E7
:100550006D2B80914C3090FF0BC080FF06C087E070
:10056000898F1A8E198A188A19C086E0898F16C059
:1005700080FF1EC085E0898F198A188AC3C08091C8
:10058000442B9091452B009711F00E94E6838091B7
:100590006D2B80FF0DC087E0898F1A8E81E090E07F
:1005A0000E94E68380E180934C300E94FB760FC06E
:1005B0008091442B9091452B892B49F4A3C08091C5
:1005C0004C3080FF9FC087E0898F1A8E9BC080E1EE
:1005D00080936D2B88E290E09093452B8093442B81
:1005E00080E580936C2B88858093682B8985809328
:1005F000692B8A8580936A2B8B8580936B2B8C85E6
:100600008093642B8D858093652B8E858093662BDC
:100610008F858093672B86E08093552B8C819D81FD
:100620009093612B8093602B8E819F819093632B9D
:100630008093622B8091E3309091E430A091E5307B
:10064000B091E6308093582B9093592BA0935A2B5E
:10065000B0935B2B88819981AA81BB8180935C2BAD
:1006600090935D2BA0935E2BB0935F2B898D84FFBD
:1006700005C010926F2B10926E2B06C084E0809301
:100680006E2B88ED80936F2B80E48093542B8091A8
:10069000442B9091452B90934E2B80934F2B10928F
:1006A000732B1092722B1092712B1092702B0E9450
:1006B000387B809590959093712B8093702B85E477
:1006C00080934C2B10924D2B1092532B1092522B47
:1006D0008091F41A9091F51A01969093F51A8093EF
:1006E000F41A9093502B8093512B1092572B109209
:1006F000562B0E94277B809590959093572B809343
:10070000562B04C01092452B1092442B10924C3063
:10071000DF91CF911F910F91FF90EF90DF90CF90DD
:10072000BF90AF90089598278927982708950E9431
:10073000BB8D0895FC018091462B9091472B2CE4B2
:1007400030E3281B390BAB01261737070CF4A9013E
:100750001416150654F45093E8304093E730E81728
:10076000F90719F0BF010C94EA91089580E880938D
:100770006100109261000E946C620E94CC530E9442
:1007800048668091F3289091F428009729F001970A
:100790009093F4288093F328C090F528D090F62801
:1007A000E090F728F090F8280E940665C616D70654
:1007B000E806F90611F30E9406656093F528709328
:1007C000F6288093F7289093F828D7CF20915130BE
:1007D00030915230BC01C90108960E94E67AE0913E
:1007E0005130F09152308091482B80878091492B75
:1007F000818780914A2B828780914B2B8387089534
:100800002F923F924F925F926F927F928F929F9220
:10081000AF92BF92CF92DF92EF92FF920F931F930E
:10082000CF93DF93CDB7DEB763970FB6F894DEBFF3
:100830000FBECDBF7C011B016A01FC01178216822D
:10084000838181FF66C3BE016F5F7F4F4B01F7015C
:100850009381F10193FD859193FF81911F0188237D
:1008600009F453C3853239F493FD859193FF819147
:100870001F01853239F4B70190E00E946D92560154
:100880006501E5CF10E0512C20E02032A0F48B323E
:1008900069F030F4803259F0833269F420612CC061
:1008A0008D3239F0803339F4216026C02260246013
:1008B00023C0286021C027FD27C030ED380F3A3013
:1008C00078F426FF06C0FAE01F9F300D1124132F85
:1008D00013C06AE0569E300D1124532E20620CC0C6
:1008E0008E3221F426FD11C3206406C08C3611F42B
:1008F000206802C0883641F4F10193FD859193FF91
:1009000081911F018111C1CF9BEB980F933018F497
:100910002061805E06C09BE9980F933008F0AAC161
:100920002F7E26FF16E02F73722E853621F4F22FCC
:10093000F0647F2E08C0863621F4622F6068762E20
:1009400002C01111115077FE07C01C3348F4442433
:100950004394410E27E00BC0183030F4212F06C01D
:1009600027E04CE3442E03C027E017E0412C56015A
:1009700074E0A70EB11CF6016081718182819381C0
:10098000042DA4010E94F2906C01098100FF02C0B5
:1009900003FF06C071FC07C072FC08C0612C08C0D0
:1009A0003DE2632E05C02BE2622E02C090E2692E6A
:1009B000802F8C7099F1662011F084E001C083E0F3
:1009C000851510F0512C0BC0581A73FC08C0B701E4
:1009D00080E290E00E946D925A94C9F7F3CF6620AE
:1009E00029F0B701862D90E00E946D9203FD03C0AF
:1009F0000EE011E102C00AE011E1F72DF0717F2E47
:100A0000F8018491882309F476C271108052B701ED
:100A100090E00E946D920F5F1F4FF2CF77FE0FC0E4
:100A20004C0C04FF04C08A81813309F44A941414E5
:100A300074F5F8E0F41578F588E0482E2CC076FCC3
:100A40002AC0812F90E08C159D059CF06CEFC61696
:100A50006FEFD60674F0772D7068772E0AC0E2E04B
:100A6000F0E0EC0FFD1FE10FF11D8081803319F4E0
:100A700011501111F4CF77FE0EC044244394410E5F
:100A8000812F90E0C816D9062CF41C1904C0442408
:100A9000439401C010E077FE07C01C141D043CF411
:100AA00096012F5F3F4F05C025E030E002C021E0F6
:100AB00030E0662011F02F5F3F4F112331F0412FBE
:100AC00050E04F5F5F4F240F351F452D50E0241736
:100AD000350714F4521A01C0512C872D897049F43E
:100AE000552039F0B70180E290E00E946D925A944F
:100AF000F7CF662029F0B701862D90E00E946D9215
:100B000073FC09C0552039F0B70180E390E00E94E2
:100B10006D925A94F7CF77FE5FC09C2D8D2DD7FE36
:100B200002C090E080E0692E782E40E050E0C601DF
:100B3000841991099D878C87960126193709280DFC
:100B4000391D812F90E0EE27FF27E81BF90BFF8767
:100B5000EE87FFEF6F167F0669F4B7018EE290E033
:100B60002B8B3A8B488B598B0E946D9259894889FF
:100B70003A892B89C614D70454F06C857D85661597
:100B800077052CF4F901E40FF51F818101C080E3A2
:100B900071E0671A71084F5F5F4FEE85FF856E1633
:100BA0007F066CF0B70190E02B8B3A8B488B598B0A
:100BB0000E946D922B893A8948895989CACF6C1451
:100BC0007D0439F49A81963318F4953311F404FFB7
:100BD00081E3B70190E04BC08A81813309F00F7E39
:100BE000B70190E00E946D92111105C074FE18C00B
:100BF00085E490E017C0B7018EE290E00E946D920C
:100C000082E066246394680EF401E80FF11D808190
:100C1000B70190E00E946D92115041F3862DF1CF03
:100C200085E690E0B7010E946D92D7FC05C0C11423
:100C3000D10439F404FF05C0D194C194D1088DE2E8
:100C400001C08BE2B70190E00E946D9280E36AE000
:100C5000C616D1042CF08F5FFAE0CF1AD108F7CF77
:100C6000B70190E00E946D92B701C601C0960E9444
:100C70006D9241C1833631F0833779F0833509F0C5
:100C800058C021C0560172E0A70EB11CF601808148
:100C9000898301E010E0640114C05601F2E0AF0E58
:100CA000B11CF601C080D18026FF03C0612F70E027
:100CB00002C06FEF7FEFC6012B8B0E9419928C014F
:100CC0002B892F7715C05601F2E0AF0EB11CF6014B
:100CD000C080D18026FF03C0612F70E002C06FEF9B
:100CE0007FEFC6012B8B0E94DB918C012B89206842
:100CF000722E23FD1AC0852D90E008171907A8F45D
:100D0000B70180E290E00E946D925A94F4CFF60110
:100D100077FC859177FE81916F01B70190E00E9489
:100D20006D9251105A94015011090115110579F76E
:100D3000E2C0843611F0893651F5560127FF09C00B
:100D4000F4E0AF0EB11CF601608171818281938164
:100D50000AC0F2E0AF0EB11CF601608171818827F4
:100D600077FD8095982F022F0F7697FF08C09095FA
:100D70008095709561957F4F8F4F9F4F00682AE057
:100D800030E0A4010E94A793C82EC8183EC0022FCD
:100D9000853721F40F7E2AE030E01DC0097F8F36B1
:100DA00091F018F4883559F0B0C0803719F08837C1
:100DB00011F0ABC0006104FF09C0046007C024FF4C
:100DC00008C0066006C028E030E005C020E130E041
:100DD00002C020E132E0560107FF09C0F4E0AF0E87
:100DE000B11CF601608171818281938108C0F2E0BB
:100DF000AF0EB11CF6016081718180E090E0A4012A
:100E00000E94A793C82EC8180F7706FF0BC0202F8B
:100E10002E7FC11650F404FF0AC002FD08C0202F27
:100E20002E7E05C0DC2C202F03C0DC2C01C0D12E6F
:100E300024FF0DC0FE01EC0DF11D8081803311F403
:100E4000297E09C022FF06C0D394D39404C0822F08
:100E5000867809F0D39423FD13C020FF06C01C2D13
:100E6000D51418F4150D1D19D52CD51468F4B70137
:100E700080E290E02B8B0E946D92D3942B89F5CF6A
:100E8000D51410F45D1801C0512C24FF12C0B70115
:100E900080E390E02B8B0E946D922B8922FF17C07C
:100EA00021FF03C088E590E002C088E790E0B70129
:100EB0000CC0822F867859F021FD02C080E201C06B
:100EC0008BE227FD8DE2B70190E00E946D92C11682
:100ED00038F4B70180E390E00E946D921150F7CF93
:100EE000CA94F401EC0DF11D8081B70190E00E94DD
:100EF0006D92C110F5CF552009F4C2CCB70180E244
:100F000090E00E946D925A94F6CFF7018681978106
:100F100002C08FEF9FEF63960FB6F894DEBF0FBE4F
:100F2000CDBFDF91CF911F910F91FF90EF90DF9098
:100F3000CF90BF90AF909F908F907F906F905F9079
:100F40004F903F902F9008955058BB27AA270ED05E
:100F50004EC23FD230F044D220F031F49F3F11F422
:100F60001EF4FFC10EF4E095E7FBF5C1E92F50D266
:100F700080F3BA17620773078407950718F071F4B6
:100F80009EF568C20EF4E0950B2EBA2FA02D0B0132
:100F9000B90190010C01CA01A0011124FF27591BBE
:100FA00099F0593F50F4503E68F11A16F040A22FC4
:100FB000232F342F4427585FF3CF46953795279535
:100FC000A795F0405395C9F77EF41F16BA0B620B34
:100FD000730B840BBAF09150A1F0FF0FBB1F661F7B
:100FE000771F881FC2F70EC0BA0F621F731F841FBE
:100FF00048F4879577956795B795F7959E3F08F0E4
:10100000B3CF9395880F08F09927EE0F97958795A2
:101010000895DFD158F080E891E009F49EEFE0D127
:1010200028F040E851E059F45EEF09C09AC112C2BD
:10103000E92FE078EDD168F3092E052AC1F32617D0
:1010400037074807590738F00E2E07F8E02569F0F2
:10105000E025E0640AC0EF6307F8009407FADB01BB
:10106000B9019D01DC01CA01AD01EF9347D0BFD1A9
:101070000AD05F91552331F02BED3FE049E450FD5C
:1010800049EC63CF0895DF93DD27B92FBF7740E8A0
:101090005FE31616170648075B0710F4D92FE5D152
:1010A0009F938F937F936F934AD3E0E3F1E06CD1EA
:1010B0009ED12F913F914F915F919ED2DD2349F0B8
:1010C0009058A2EA2AED3FE049EC5FE3D0785D2733
:1010D0004DDFDF918CC11BD108F481E008950CD065
:1010E00086C17ED140F075D130F021F45F3F19F018
:1010F00032C15111B0C135C18BD198F39923C9F3D5
:101100005523B1F3951B550BBB27AA27621773070D
:10111000840738F09F5F5F4F220F331F441FAA1FC1
:10112000A9F333D00E2E3AF0E0E830D09150504081
:10113000E695001CCAF729D0FE2F27D0660F771F2F
:10114000881FBB1F261737074807AB07B0E809F011
:10115000BB0B802DBF01FF2793585F4F2AF09E3FA6
:10116000510568F0F8C077C15F3FECF3983EDCF3BF
:10117000869577956795B795F7959F5FC9F7880F1F
:10118000911D9695879597F90895E1E0660F771F71
:10119000881FBB1F621773078407BA0720F0621B02
:1011A000730B840BBA0BEE1F88F7E095089519F4C2
:1011B0000EF0D1C04FC1D5C033D1C8F39638C0F7B7
:1011C00007F80F92E8942BE33AEA48EB5FE716D270
:1011D0000F920F920F924DB75EB70F92CED1EDE501
:1011E000F1E0D2D04F915F91EF91FF91E595EE1F25
:1011F000FF1F49F0FE57E0684427EE0F441FFA95A1
:10120000E1F74195550B3AD10F9007FE2EC1089595
:1012100097FB0EF4A9D03EC0E89409C097FB3EF4BA
:1012200090958095709561957F4F8F4F9F4F992333
:10123000A9F0F92F96E9BB279395F69587957795B1
:101240006795B795F111F8CFFAF4BB0F11F460FF71
:101250001BC06F5F7F4F8F4F9F4F16C0882311F0C9
:1012600096E911C0772321F09EE8872F762F05C0DD
:10127000662371F096E8862F70E060E02AF09A9578
:10128000660F771F881FDAF7880F9695879597F96D
:101290000895E894F92F96EBFF2381F012161306B8
:1012A0001406440B9395F695879577956795579512
:1012B0004040FF23B9F71BC099270895882351F4B4
:1012C0009850D2F7872B762F652F542F432F322F2C
:1012D00020E0B1F3121613061406440B88233AF0EB
:1012E0009A95440F551F661F771F881FCAF755230D
:1012F0004AF4440F551F11F460FF04C06F5F7F4F25
:101300008F4F9F4F880F9695879597F90895990F5E
:101310000008550FAA0BE0E8FEEF16161706E807BF
:10132000F907C0F012161306E407F50798F0621BE0
:10133000730B840B950B39F40A2661F0232B242BB5
:10134000252B21F408950A2609F4A140A6958FEFD4
:10135000811D811D089597F99F6780E870E060E026
:1013600008959FEF80EC0895909580957095609515
:1013700050954095309521953F4F4F4F5F4F6F4FA0
:101380007F4F8F4F9F4F0895DF93CF931F930F93FE
:10139000FF92EF92DF927B018C01689405C0DA2EF8
:1013A000EF012AD1FE01E894A5912591359145914F
:1013B0005591AEF3EF01DADDFE019701A801DA9451
:1013C00079F7DF90EF90FF900F911F91CF91DF9110
:1013D000089500240A94161617061806090608959B
:1013E00000240A9412161306140605060895092E01
:1013F0000394000C11F4882352F0BB0F40F4BF2B70
:1014000011F460FF04C06F5F7F4F8F4F9F4F0895AF
:1014100057FD9058440F551F59F05F3F71F04795A5
:10142000880F97FB991F61F09F3F79F0879508958A
:10143000121613061406551FF2CF4695F1DF08C0A9
:10144000161617061806991FF1CF869571056105C6
:1014500008940895E894BB2766277727CB0197F96E
:10146000089555DF08F48FEF08959B01AC0160E00B
:1014700070E080E89FE333CE6ECF64C1D1DFE8F344
:101480009923D9F3940F511DBBF39150504094F020
:1014900059F0882332F0660F771F881F9150504013
:1014A000C1F79E3F510544F7880F911D969587958A
:1014B00097F908955F3FACF0983E9CF0BB27869566
:1014C00077956795B79508F4B1609395C1F7BB0F11
:1014D00058F711F460FFE8CF6F5F7F4F8F4F9F4F3A
:1014E000E3CFB9CF0AD029ED3BE54EED5EE378C0FE
:1014F0000EF028C136CF68942ECF92DFC8F399231F
:10150000D1F3C6F3DF93CF931F930F93FF92C92FAD
:10151000DD2788232AF02197660F771F881FDAF7C7
:1015200020E030E040E85FEB9FE3883920F0803E28
:1015300030F021968F7709DDE5E8F1E003C005DDA5
:10154000E2EBF1E021DF8B01BE01EC01FB2E6F57D6
:1015500071097595771F880B990B60DE28E132E7DA
:1015600041E35FE349D0AF2D9801AE01FF900F91A9
:101570001F91CF91DF91FADC3ACFFA01DC01AA0F7B
:10158000BB1F9B01AC01BF5728F4222733274427F8
:1015900050781FC0B75188F4AB2F0024469537957B
:1015A0002795011CA395D2F3002069F0220F331F69
:1015B000441FB395DAF30DD0C7CC61307105A0E8B4
:1015C0008A07B94630F49B01AC0166277727882744
:1015D0009078309621F0208331834283538308959D
:1015E0000BD005CFF6DE28F0FBDE18F0952309F0CE
:1015F000B2CEB7CE11242FCF0BDFA0F3959FD1F33E
:10160000950F50E0551F629FF001729FBB27F00DB0
:10161000B11D639FAA27F00DB11DAA1F649F662705
:10162000B00DA11D661F829F2227B00DA11D621F54
:10163000739FB00DA11D621F839FA00D611D221F0E
:10164000749F3327A00D611D231F849F600D211DF2
:10165000822F762F6A2F11249F5750408AF0E1F095
:1016600088234AF0EE0FFF1FBB1F661F771F881FDE
:1016700091505040A9F79E3F510570F06CCEEBCED3
:101680005F3FECF3983EDCF3869577956795B795C9
:10169000F795E7959F5FC1F7FE2B880F911D9695F3
:1016A000879597F90895FA01EE0FFF1F30962105EF
:1016B000310599F16115710561F48038BFE39B072D
:1016C00049F168949038810561F08038BFEF9B073D
:1016D00041F0992342F5FF3FE1053105210511F164
:1016E000E8940894E795D901AA2329F4AB2FBE2FDB
:1016F000F85FD0F310C0FF5F70F4A695E0F7F739FC
:1017000050F019F0FF3A38F49F779F930CD00F9068
:1017100007FC905808953EF024CE60E070E080E829
:101720009FE308954FE79F775F934F933F932F93E6
:10173000E4DE2F913F914F915F9152DF3DCD9B01B0
:10174000AC014ECF9F3F31F0915020F487957795B3
:101750006795B795880F911D9695879597F9089588
:101760000E94B88B332312F48A1B9B0B0C94C98BF9
:10177000A29FB001B39FC001A39F700D811D1124D2
:10178000911DB29F700D811D1124911D08950E941D
:10179000B88BB7FF0895821B930B08950E94B88BF6
:1017A000A59F900DB49F900DA49F800D911D1124B5
:1017B0000895B7FF0C94CE8B0E94CE8B821B930BA7
:1017C0000895DB018F939F930E94CE8BBF91AF91C1
:1017D000A29F800D911DA39F900DB29F900D11248B
:1017E0000895AA1BBB1B51E107C0AA1FBB1FA61768
:1017F000B70710F0A61BB70B881F991F5A95A9F7BA
:1018000080959095BC01CD01089597FB072E16F4A5
:10181000009407D077FD09D00E94F18B07FC05D01A
:101820003EF4909581959F4F0895709561957F4FF7
:101830000895A1E21A2EAA1BBB1BFD010DC0AA1F11
:10184000BB1FEE1FFF1FA217B307E407F50720F029
:10185000A21BB30BE40BF50B661F771F881F991FA4
:101860001A9469F760957095809590959B01AC01ED
:10187000BD01CF010895052E97FB1EF400940E9430
:10188000668D57FD07D00E94198C07FC03D04EF4DB
:101890000C94668D50954095309521953F4F4F4F54
:1018A0005F4F0895689401C0E894F92FF12B12F06E
:1018B0000C94868CA0E0B0E0E0E6FCE80C94848D0B
:1018C000092E059422F40E946E8D112392F4F0E803
:1018D0000F26FFEFE094F09400951095B094C0941B
:1018E000D094A194BF0ACF0ADF0AEF0AFF0A0F0BB8
:1018F0001F0B0E94158D07FC0E946E8DCDB7DEB7C1
:10190000ECE00C94A08D689401C0E8948F929F92B3
:10191000CF93DF930E94158DDF91CF919F908F9091
:101920000895DF93CF931F930F939A9DF02D219FDE
:10193000F00D8B9DF00D8A9DE02DF10D039FF00DB4
:10194000029FE00DF11D4E9DE00DF11D5E9DF00D1D
:101950004F9DF00D7F936F93BF92AF925F934F9324
:10196000D5010E94B88B8B01AC01D7010E94B88BC6
:10197000EB01E80FF91FD6010E94E18C2F913F91F6
:10198000D6010E94B88BC60FD71FE81FF91FAF9171
:10199000BF910E94E18C2F913F910E94B88BC60F9E
:1019A000D71FE81FF91FD6010E94B88BE60FF71F5B
:1019B0009801BE01CF0111240F911F91CF91DF91AA
:1019C00008950E94B88B460F571FC81FD91F08F4EF
:1019D00031960895E894DF93CF93FC01DB010E94D8
:1019E000B88B7F936F93E9019A01AC01BF93AF93DA
:1019F0003F932F93DF010E94B88B26F46C1B7D0B65
:101A0000820B930B9E01EB01FC010E94E18CAF91D4
:101A1000BF912F913F910E94E18CBE01CF01F9014E
:101A20002F913F91CF91DF91089588249924F4015B
:101A3000E401B0E49F93AA279A158B049C04ED055A
:101A4000FE05CF05D007A10798F4AD2FDC2FCF2FCF
:101A5000FE2FE92D982C892E982F872F762F652F12
:101A6000542F432F322F2227B85031F7BF9127C070
:101A70001B2EBF91BB27220F331F441F551F661F0C
:101A8000771F881F991F881C991CEE1FFF1FCC1FF2
:101A9000DD1FAA1FBB1F8A149B04EC05FD05CE05A4
:101AA000DF05A007B10748F08A189B08EC09FD097B
:101AB000CE09DF09A00BB10B21601A94E1F62EF4D8
:101AC0009401AF01BE01CD01000C08959095809561
:101AD000709561957F4F8F4F9F4F089560957095DA
:101AE0008095909530954095509521953F4F4F4F5B
:101AF0005F4F6F4F7F4F8F4F9F4F08952F923F92B1
:101B00004F925F926F927F928F929F92AF92BF920D
:101B1000CF92DF92EF92FF920F931F93CF93DF93B9
:101B2000CDB7DEB7CA1BDB0B0FB6F894DEBF0FBE16
:101B3000CDBF09942A88398848885F846E847D8463
:101B40008C849B84AA84B984C884DF80EE80FD8065
:101B50000C811B81AA81B981CE0FD11D0FB6F894DB
:101B6000DEBF0FBECDBFED010895EE0FFF1F059044
:101B7000F491E02D0994692796276927782787270C
:101B8000782708950F93083090F0982F872F762F9D
:101B9000652F542F432F322F22270850F4CF220FC6
:101BA000331F441F551F661F771F881F991F0A95F3
:101BB000B2F70F91089597FB10F8169400080F9351
:101BC000083098F00850232F342F452F562F672FB9
:101BD000782F892F902DF4CF059497958795779539
:101BE000679557954795379527950A95AAF70F91C9
:101BF00008952A0D3B1D4C1D5D1D6E1D7F1D801F10
:101C0000911F08950024A7FD00942A0F301D401D48
